:020000040000FA
:10000000A80B002015140000F93B00004514000067
:10001000451400004514000045140000451400007C
:100020000000000000000000000000005D12000061
:10003000451400000000000015120000F73A00000F
:10004000D5130000D5130000D5130000D513000010
:10005000D5130000D5130000D5130000D513000000
:10006000D5130000D5130000D5130000D5130000F0
:10007000D5130000D5130000D5130000D5130000E0
:10008000D5130000D5130000D5130000D5130000D0
:10009000D5130000D5130000D5130000D5130000C0
:1000A000D5130000D5130000D5130000D5130000B0
:1000B000D5130000D5130000D5130000D5130000A0
:1000C000D5130000D5130000D5130000D513000090
:1000D000D5130000D5130000D5130000D513000080
:1000E000D5130000D5130000D5130000D513000070
:1000F000D5130000D5130000D5130000D513000060
:10010000D5130000D5130000D5130000D51300004F
:10011000D5130000D5130000D5130000D51300003F
:10012000D5130000D5130000D5130000D51300002F
:10013000D5130000D5130000D5130000D51300001F
:10014000D5130000000000000000000000000000C7
:10015000000000000000000000000000000000009F
:10016000000000000000000000000000000000008F
:10017000000000000000000000000000000000007F
:10018000000000000000000000000000000000006F
:10019000000000000000000000000000000000005F
:1001A000000000000000000000000000000000004F
:1001B000000000000000000000000000000000003F
:1001C000000000000000000000000000000000002F
:1001D000000000000000000000000000000000001F
:1001E000000000000000000000000000000000000F
:1001F00000000000000000000000000000000000FF
:10020000DEE61E284CBBCE8F025B00003C000000E7
:10021000008000000100000000000000000000005D
:10022000FFFF02910000000000000000000000003D
:1002300000000000000000000000000053B94AB9AF
:10024000002908BF00281CBF4FF0FF314FF0FF30DE
:1002500000F06CB9ADF1080C6DE904CE00F006F8C1
:10026000DDF804E0DDE9022304B070472DE9F04732
:10027000089D04468846002B7DD18A4217463FD907
:10028000B2FA82F242B1C2F120009140974024FAC2
:1002900000F0944040EA01084FEA174C230C1FFA83
:1002A00087FEB8FBFCF60CFB168106FB0EF043EA5A
:1002B0000143984205D9FB1802D2984200F22481EA
:1002C000013E191AA3B2B1FBFCF00CFB101100FBAC
:1002D0000EFE43EA0144A64505D93C1902D2A645C3
:1002E00000F20F81013840EA0640A4EB0E0400261C
:1002F0001DB1D4400023C5E900433146BDE8F08775
:1003000002B9FFDEB2FA82F2002A50D1CB1B4FEACB
:10031000174E1FFA87F80126210CB3FBFEFC0EFBDB
:100320001C300B4608FB0CF941EA004189450AD90B
:1003300079182CBF01230023894502D9002B00F036
:10034000D9800CF1FF3CA1EB0901A3B2B1FBFEF097
:100350000EFB101108FB00F843EA0144A04505D943
:100360003C1902D2A04500F2C9800138A4EB080470
:1003700040EA0C40BCE78B4209D9002D00F0B18067
:100380000026C5E9000130463146BDE8F087B3FAE2
:1003900083F6002E46D18B42C0F0A680824240F206
:1003A000A3803046002DA8D0C5E90048A5E79740B6
:1003B000C2F1200301FA02F04FEA174ED94024FAA5
:1003C00003F31FFA87F894400343B1FBFEF01E0CC1
:1003D0000EFB101100FB08FC46EA01418C4509D9CF
:1003E00079182CBF012600268C4502D9002E00F07A
:1003F00093800138A1EB0C019BB2B1FBFEF60EFB22
:10040000161106FB08FC43EA01418C4505D9791811
:1004100002D28C4500F28780013EA1EB0C0346EA34
:10042000004679E7C6F1200703FA06F402FA06FC53
:1004300001FA06FEFA4020FA07F8F94000FA06F33E
:10044000224348EA0E044FEA12484FEA144E1FFABC
:1004500082F9B1FBF8FA08FB1A110AFB09F04EEA1F
:10046000014E70450AD912EB0E0E2CBF012100215E
:10047000704501D9002952D00AF1FF3AAEEB000EC7
:10048000A4B2BEFBF8F008FB10EE00FB09F944EA49
:100490000E4EF14505D912EB0E0E01D2F14538D8BA
:1004A000013840EA0A40AEEB090EA0FB0C89CE45AC
:1004B00041464C4602D306D1434504D20138B8EB3D
:1004C0000C0169EB020415B35A1A6EEB040EF240EC
:1004D0000EFA07F72EFA06F300261743C5E9007354
:1004E0000BE72E46284608E7841A61EB030101203A
:1004F000884657E7ACF1020C394424E702383C4403
:1005000034E702383C44EEE6023E3B44D9E62E4650
:10051000F3E602389644C4E7023839446AE7AAF1A0
:10052000020A9644AAE7023E394476E7704700BFC4
:100530002DE9E04F2746A046A146A246A346A44681
:100540002DED108B4FF0000545EC185B45EC195A6A
:1005500045EC1A5A45EC1B5A45EC1C5A45EC1D5A01
:1005600045EC1E5A45EC1F5AF1EE105A4FF66076D4
:10057000C0F6FF763540E1EE105A84F30088254638
:100580002646A447BDEC108BBDE8E08F0B68013315
:100590000B60014B1B681847000000202DE9F04F4D
:1005A0002DED028B83B00E9C9A46012CB8BF01241E
:1005B000012B0CBF302320231546064608EE103AC7
:1005C00001274FF00A080022DFF874B0B5FBFBF9F1
:1005D0000AB9AB4520D809F130000091B04701229B
:1005E000013700990A2308F1FF38B8F1010F0BFB1E
:1005F0001955BBFBF3FBE9D105F130000091B04781
:10060000BAF1030F009902D1E41B002C11DC03B0F6
:10061000BDEC028BBDE8F08F4445E3DBBAF1020F7D
:10062000E0D818EE100ACDE900120137B047019A60
:10063000D7E720200091013CB0470099E5E700BFD3
:1006400000CA9A3B2DE9F04F002705468B464FF034
:10065000FF39B8461C468DB0531E0393002605E0B3
:100660006EB9252800F071815946A847039B13F8FD
:10067000010F03930028F3D10DB0BDE8F08F7A2865
:100680000AD8622810D8302854D045D8252800F040
:100690005A812D2800F05F8159462520A8475946E8
:1006A000039B1878A847D9E7A0F16303172BF3D869
:1006B00001A252F823F000BF3F09000083070000A9
:1006C00099060000990600009906000065070000E1
:1006D00083070000990600009906000065070000E6
:1006E0009906000099060000990600002508000000
:1006F00099060000990600000F0900009906000005
:10070000F307000099060000990600002107000089
:10071000990600006507000039281AD95828BBD16E
:10072000039B1B78702B40F0888054F8043B002218
:10073000069390E0B9F1000F0EDAB8F1000F00F067
:100740000D81A0F13009B8F1000F08BF4FF0020889
:100750008CE7B9F1000FF4DB0A2303FB0909A9F1C7
:100760003009F0E7682803D1682F06D148277DE7D4
:100770006C2802D16C2F00F0F480002F8CD107463A
:1007800074E77A2F02D154F8046B21E06C2FFAD071
:100790004C2FF8D1073424F00704F4E80223CDE904
:1007A0000423049B4FF0FF3013F10041059B089197
:1007B00043F1000109910021DDE90823994208BFB6
:1007C000904204D25946284603F00BF846E7049EAF
:1007D000002E05DA59462D20A847764209F1FF3947
:1007E00043463246CDF8009059462846FFF7D6FEDC
:1007F00034E77A2F02D154F8042B0FE06C2FFAD093
:100800004C2FF8D100214FF0FF30073424F00704BB
:10081000F4E80223994208BF9042D3D34346CDF86F
:100820000090E1E759463020A84759467820A8476C
:100830004FF008094FF0010872E76C2F3FF475AFD5
:100840004C2F7FF472AFE31D23F007031C4654F8CE
:10085000082B06925A68002110234FF0400A049199
:100860000791AAF1040A0699CAF1200EAAF1200CF8
:1008700021FA0AF002FA0EFE40EA0E0022FA0CFCFF
:1008800040EA0C0010F00F0007D1079911B9BAF136
:10089000000F25D14FF0300C05E009288CBF4FF038
:1008A000570C4FF0300C6044594640B20A920793FF
:1008B000A847049B0A9A01330493079BBAF1000FDF
:1008C00023D1B8F1030F7FF4C9AE049BC3EB4906F3
:1008D000002E7FF7C3AE59462020A847013EF7E718
:1008E000591E99450A9107DBB8F1010F06D1594607
:1008F00030200B92A8470B9A0A9BB2E7B8F1020F7F
:10090000FAD1594620200B92F4E70796A9E754F84C
:10091000046BB24653461AF8010B68B9B8F1030FDD
:1009200021D19E1BA9EB0606002E7FF797AE5946F4
:100930002020A847013EF7E75946A847EAE759466D
:1009400054F8040BAEE65946ACE63746B0464FF0D5
:10095000FF3901268AE64FF0030887E64FF00108C9
:1009600084E64C2782E6064680E600BF07B50B46C4
:10097000002102460191034801A9FFF763FE03B07D
:100980005DF804FB8D0500004FF02002EFF31183AA
:1009900082F31188BFF36F8F0121044AC2F840151A
:1009A00083F31188BFF36F8F0020704700900350CE
:1009B00020B1034B800143F001031847704700BF8B
:1009C00090420000F8B50C24114F0546FB6804FB6B
:1009D0000034012363724FF02003EFF3118183F39E
:1009E0001188BFF36F8F23682BB166681A68B34212
:1009F000226008BF626081F31188BFF36F8F03B973
:100A0000F8BD2946D3E901623846B047E3E700BFA5
:100A10007000002008B5114B1A686AB14FF05022DF
:100A2000D2F80423D10707D500221A600C4BDB68EB
:100A3000587A08B9FFF7C6FF0A4B1A6862B14FF03F
:100A40005022D2F80423920706D5002201201A6012
:100A5000BDE80840FFF7B6BF08BD00BF0051005019
:100A60007000002004510050821C084B22F07F428D
:100A7000C3F84025D3F80425904200D17047D3F83D
:100A80000405821C22F07F42F2E700BF00500150B3
:100A90000022064B1A60064AD3F800041368C01AF5
:100AA00020F07F400344136001F046BF40510150E5
:100AB0002801002038B5144801F046F900B38368D6
:100AC000002401211B6898474FF400120F4D104B72
:100AD000C5F808451C600F4B0121C3F880214FF475
:100AE00080332246C5F80433152000F0D7FB1520CB
:100AF00000F0C4FB01232046074A13602B6038BD79
:100B00004FF0FF30FBE700BFB2460000005001503D
:100B10004051015000E100E008500150F8B52C4B65
:100B20002C4CD3F804252C4BB0F1FF3F08BF2046D6
:100B30001968521A22F07F43120236D4013820EA93
:100B4000E070A042A8BF204601331844A04294BFE1
:100B50000C180C194FF4803000271D4B1F4EC3F8A2
:100B60000803D3F80415D3F8402521F07F45521A25
:100B700022F07F42012A3760C3F840551D46C3F872
:100B8000440303D10F2003F0F4F937604FF400124F
:100B9000134BC3F88021D5F80405231A23F07F43B3
:100BA000012B04D1FFF760FF0BE00020CCE724F01D
:100BB0007F43C5F84035D5F80405241A023C2302CA
:100BC000F0D44FF48032024BC3F80423F8BD00BFC9
:100BD00000500150FFFF7F002801002040510150CC
:100BE00000E100E04FF02002EFF3118382F311885F
:100BF000BFF36F8F064AD2F80405064A1268801ABE
:100C000020F07F4083F31188BFF36F8F704700BFE0
:100C10000050015028010020F7B500281C460D4661
:100C200014BF4FF400534FF40043204E954232D38B
:100C300002FB03F0013A4B4300901D4802F0DFFD38
:100C40001C4B14F0100F1C491C4808BF194602F039
:100C5000D6FD14F0040F14BF72212D21184802F0A4
:100C6000CEFD14F0020F14BF77212D21144802F09D
:100C7000C6FD14F0010F0CBF2D217821104802F0A1
:100C8000BEFD6C210E4802F0BAFD0E4803B0BDE86F
:100C9000F04002F0B4BD28B105F5E07746F82740F2
:100CA0000135C3E705F5C077F8E700BF0030005015
:100CB0001145000005450000FC440000904600007E
:100CC0002B4500005F48000008B543B2002B0CDB49
:100CD000012200F01F018A405B091049203341F8CE
:100CE0002320BFF34F8FBFF36F8F830003F1A04327
:100CF00003F540533128D3F8002806D0002A07DA3C
:100D000002F00302023A012A02D8054AC3F8002879
:100D1000002102F042FF002008BD00BF00E100E01A
:100D20000001008030B54FF440444CF2040585B01A
:100D30004FF440412C4802F062FD21682B4802F03C
:100D40005EFD29682A4802F05AFD102200216846FB
:100D500002F0E1FF236868460093029400F044FE2D
:100D6000012000F071FE002000F05AFE002000F08B
:100D70007FFE0121002000F099FE00F08DFE2C681E
:100D80001C4802F03CFD0820FFF79EFF24F0010400
:100D9000BFF34F8FBFF36F8F640864002046214676
:100DA00022462346B7EE000AF7EE000AB7EE001A15
:100DB000F7EE001AB7EE002AF7EE002AB7EE003A77
:100DC000F7EE003AB7EE004AF7EE004AB7EE005AE7
:100DD000F7EE005AB7EE006AF7EE006AB7EE007A57
:100DE000F7EE007AFFF7A4FB2E4500004545000012
:100DF0005A450000784500002DE9F8433B4802F0D1
:100E0000FEFC002140F2171308460122FFF704FF01
:100E100040F20713202201210020FFF7FDFE344895
:100E200002F0EDFC334B344AC3F3C431C3F30E0379
:100E3000C3F50043C3F34313C2F80015C2F80435E9
:100E4000D2F80015D2F804252C48520102F0D7FC44
:100E5000274802F0D4FC02F050FE014610B12848A9
:100E600002F0CDFC0024274802F0C9FC40F2171321
:100E7000082200210120FFF7CFFE1F4D40F207138B
:100E8000202208210120FFF7C7FE194802F0B7FC15
:100E9000C5F880441C4802F0B2FC1C4FC5F8C044A1
:100EA000DFF87C801A4DDFF87C906E792146002EA9
:100EB00014BF3B46434648462A6802F0A0FC66B988
:100EC0001448013402F09BFC1A2C05F10805ECD102
:100ED0000748BDE8F84302F092BC2879FFF7F4FE1A
:100EE00008B10D48EDE70D48EBE700BFAE45000047
:100EF0005F480000E07F000000300050D245000055
:100F000018460000484600006A460000A34500005D
:100F1000AC420000934600009A460000A246000042
:100F2000094500008646000010B500284BD0002A75
:100F300049D0264B99423CD9541803F61D239C42B4
:100F40003AD802F0BDFE0020BDE81040714672465E
:100F50007346B7EE000AF7EE000AB7EE001AF7EE96
:100F6000001AB7EE002AF7EE002AB7EE003AF7EEC5
:100F7000003AB7EE004AF7EE004AB7EE005AF7EE35
:100F8000005AB7EE006AF7EE006AB7EE007AF7EEA5
:100F9000007A8EF3008C10B4F1EE10CA4FF6607434
:100FA000C0F6FF740CEA040CE1EE10CA10BCF44663
:100FB0007447074B994203D9064B54189C42C0D939
:100FC0004FF0FF30C0E76FF01500BDE70302FF00F0
:100FD0002F01FF003801FF002DE9F04F81460E463A
:100FE00085B0002954D04FF00008DFF8B8B0DFF822
:100FF000B8A001AF5BF8045B9AE807004D4487E8AE
:1010000007000C223946284602F033FE044608B990
:10101000002D40D108F10108B8F1050FEAD16FF0B9
:101020000D04204605B0B7EE000AF7EE000AB7EE51
:10103000001AF7EE001AB7EE002AF7EE002AB7EE14
:10104000003AF7EE003AB7EE004AF7EE004AB7EE84
:10105000005AF7EE005AB7EE006AF7EE006AB7EEF4
:10106000007ABDE8F04F714672467346F7EE007A9B
:101070008EF3008C10B4F1EE10CA4FF66074C0F617
:10108000FF740CEA040CE1EE10CA10BCF44674477D
:101090006FF01504C5E73C222946304602F010FEE9
:1010A000BFE700BF7C43000060420000014801F040
:1010B000ADBE00BF9043000008B530B143683BB1FE
:1010C000006801F037F8002008BD6FF4E040FBE74E
:1010D0000048F9E7EA8FFFFF38B5044618B90B4B13
:1010E0000B485B689847656855B115F002052068A4
:1010F00007D10146074800F07BFF256000236360AD
:1011000038BD1422002102F006FEF7E7440000205B
:10111000A34700002C01002010B5044618B9144B59
:1011200014485B6898476368CBB92368BBB94FF034
:10113000FF324FF0FF3321460F4800F027FF08B978
:1011400023681BB90A4B0D485B689847142200219D
:10115000206802F0E0FD636843F0020363602068EA
:1011600002F042FE636843F00103636010BD00BFFC
:1011700044000020A34700002C010020C9470000C4
:1011800008B568B1436873B100684FF0FF334FF0A2
:10119000FF3200F057FF054B002818BF184608BD66
:1011A0006FF4E040FBE70248F9E700BFE98FFFFF7B
:1011B000EA8FFFFF08B5064940231422054802F0D4
:1011C000F8FDBDE808400449044801F057BE00BFDF
:1011D000480100202C010020A84300009843000093
:1011E000094A0A4993680968D866196708494B682B
:1011F00043F080534B60002383F31188BFF36F8F5C
:101200009368186F704700BF44070020F843000040
:1012100000ED00E00F498A684FF030001044EFF312
:10122000098C80E8F01F202080F31188BFF36F8FB6
:10123000094F4FF000664A6A8A603E60D06E002314
:10124000D36680F3118802F1300090E8F01F8CF330
:10125000098870474407002004ED00E01EF0040FE9
:101260000CBFEFF30880EFF30980816911F8021CCD
:101270000229FFD001B502F0BBFC01BD43B2002B37
:1012800008DB012200F01F0002FA00F0024A5B09AD
:1012900042F82300704700BF00E100E043B2002B9A
:1012A00001F10101ACBF03F16043064B4FEA41116C
:1012B000C9B2ABBF03F5614300F00F0083F8001320
:1012C0001954704714ED00E0C0E918120A44203A9E
:1012D00022F007021360009B07495360019B21F035
:1012E00001019360029B9161D3604FF08073D361E1
:1012F00000230265C366704719380000F8B51D4623
:1013000006460C4617460023E1EE103A00F0F4F9C9
:10131000084BE21922F007049E60284684F30988EE
:10132000002163B681F31188BFF36F8F0022002381
:1013300002F072FA44070020014910220A60704747
:1013400010ED00E072B6404080F31188BFF36F8F5C
:10135000BFF34F8F30BF62B6BFF36F8F704700BFD0
:1013600030BFFFF7FDBF00BF174A08B5174B22F08B
:101370007F029A60BFF34F8FBFF36F8FD3F888203F
:1013800022F47002C3F88820D3F8882042F4A00227
:10139000C3F888200E4A536823F040435360BFF3DC
:1013A0004F8FBFF36F8F0023E1EE103AEFF31483FA
:1013B00023F0040383F3148800F004FD00F00CFD17
:1013C00000F068F900F03AFD0000000000ED00E0D8
:1013D00030EF00E001B572B60B4A106A00281EBF5C
:1013E0000021116202F0E3FC62B6EFF30580A0F188
:1013F00010004FEAC0000549014409C99847BDE8FB
:101400000140034908470000440700205440000001
:101410005516000002F0B5FA202080F31188084824
:101420004FF40061401880F30988EFF31480022123
:10143000084380F31488BFF36F8FFFF795FF000018
:10144000E80C0020EFF30880EFF30981724601B544
:1014500000F06CF801BD00BF0C4B9A6A9A6A9A6A58
:10146000920708D55A6B9A6A120604D518B19A6A7F
:1014700022F080029A620020044B9A6A9A6A9A6A61
:101480009A6A42F0FF029A620870704700ED00E02D
:101490000D4B9A6A9A6A9A6A920508D59A6B9A6A6B
:1014A000120404D518B19A6A22F400429A6200200C
:1014B000054B9A6A9A6AD20558BF9A6A9A6A42F4A8
:1014C0007F429A620870704700ED00E0074B0020F1
:1014D0009A6A9A6A9A6A9A6A9A6A9A6A9A6A9A6AEC
:1014E0006FEA02426FEA12429A62704700ED00E032
:1014F0000D4B9A695A695A69D0070FD45A699107F6
:101500000CD45A69520709D45A69100706D45A698B
:10151000D10603D45A69920658BF5A695A6942F0F3
:10152000FF025A61704700BFD0ED00E0F0B5414BBB
:1015300000255B688BB0C3F3080385F31188BFF304
:101540006F8F02F07F44B4F17F4F1ED112F001047F
:101550001AD0560602F0080467D482F00402C2F3DF
:10156000800564B1EFF389860022033B8DF80720E4
:10157000042B4BD8DFE803F00B4C50414800EFF34D
:101580008886F1E70E46EFE725462E46ECE7294B25
:10159000DA6A92073AD4DC6A14F0804408D028331F
:1015A0001B78EBB101200DF10701FFF755FF044651
:1015B0009DF8073093B92022314602A802F080FB43
:1015C000099B6DB3C3F3080222B96FEA53236FEA94
:1015D00043230993204602A902F008FB0BB0F0BD9B
:1015E000154B1B782BB101200DF10701FFF750FFC0
:1015F000DDE7124B1F88BFB217B1FFF767FFD6E7D1
:101600000F4B5C69002CD3D0FFF772FF0024CFE7AB
:1016100000200DF10701C8E700200DF10701E5E703
:1016200023F4FF7323F00103D3E7002CAAD106466D
:10163000012599E700ED00E029ED00E02AED00E04A
:10164000D0ED00E0024A536943F010035361704744
:1016500000ED00E0044B9968586A884203D00349C2
:101660004FF080520A6070474407002004ED00E00C
:10167000BFF34F8F0549064BCA6802F4E06213437B
:10168000CB60BFF34F8F00BFFDE700BF00ED00E070
:101690000400FA05002320210348C2180133412B1E
:1016A00082F80013F9D1704700E100E038B5044634
:1016B0004FF02003EFF3118583F31188BFF36F8F91
:1016C00000F0F8FE0A4B9B68A3420BD1094B5A6805
:1016D000C2F3080212B92846FFF782FD5A6842F0A9
:1016E00080525A602846BDE8384002F08FBB00BFE8
:1016F0004407002000ED00E010B50E4B88B00293C7
:101700000D4B0E4C03930E4B0E4A049302AB019308
:1017100001A82346012100F007F9002307930A4B93
:101720000121E41A05A80593069400F007F908B012
:1017300010BD00BF000000200000000000000120DC
:1017400006000100000000200801002010B50B6811
:101750000C7A23F01F0204F01F031A43CB686409BC
:1017600023F01F03044943EA440343F00103886064
:10177000CA600B6110BD00BF90ED00E02DE9F04F95
:1017800007468846144600264A4D85B046450BDA82
:1017900057F82630D3F80490B9F1000F3AD0B9F1D8
:1017A0001F0F05D86FF01504204605B0BDE8F08F77
:1017B00019F01F0FF6D1D3F800A01AF01F0FF1D1C6
:1017C000504602F040FA834609EB0A00013802F065
:1017D0003AFA8345E6D11BF1160FE3D0631E5B4551
:1017E000E0DBC5F808B0E868C5F808B02B6957F821
:1017F000261020F01F0043F01F0AD1E900321A44DE
:10180000984202F1FF3918D1CA4505D15FFA8BF031
:1018100002F0F9F90136B9E7C5F808B0EB6822F033
:101820001F0203F01F031A43EA60E0B202F0EBF973
:1018300010F1160FB6D0441CECE7C5F808B02A69C1
:10184000013B23F01F0302F01F021343CA45E0B21D
:101850002B61EBD002F0D7F910F1160FA2D0C5F82A
:1018600008B0EA689DF808300AF1FF3A62F3040311
:101870008DF808302B699DF808205B0863F3471248
:1018800057F826308DF80820D3E900130B44009355
:1018900023F01F0301305344A3EB0903C0B223F02C
:1018A0001F030F2803933FF67DAF6946FFF74EFFF6
:1018B000C1E700BF90ED00E00522034B5A60BFF383
:1018C0004F8FBFF36F8F704790ED00E0BFF35F8FD6
:1018D0000022014B5A60704790ED00E038B50E4C85
:1018E0002568102D14D8FFF7F1FF00200B4B0C4A90
:1018F0001A63854205D10B4B1D70FFF7DDFF0020F9
:1019000038BD616801EB0011FFF720FF0130F0E7FF
:101910004FF0FF30F4E700BFBC43000090ED00E063
:10192000AAFF4400A007002010B5034C2278FFF75F
:1019300025FF207010BD00BFA00700202DE9F74F44
:10194000264D8A4606464FF00008AB46244FD04548
:101950001BDAD6F80490B9F1000F39D03168084687
:10196000019102F070F90199044609EB0100013878
:1019700002F069F984424FF014021A4B08D06FF05C
:10198000150302FB08F84BF8083003B0BDE8F08FF0
:1019900014F1160F2C60F8D01978A142F5DD02FB86
:1019A00008B0BC60BC60FC6800F10801007B64F317
:1019B0000400087138690C79400860F347140C7111
:1019C000F96821F01F016960396921F01F0129615F
:1019D00008F1010814350C36B9E700BF48060020AD
:1019E00090ED00E0A007002082680C4B9A6003682D
:1019F00083F38888436883F38988027B02F00101BE
:101A0000EFF3948323F00303920748BF43F00203EC
:101A100009B143F0010383F39488704700ED02E0BD
:101A2000084AD36848B123F400531B041B0C43F04D
:101A3000BF6343F40033D36070479BB243F4005359
:101A4000F5E700BF00ED00E0084AD36840B19BB263
:101A500043F4804343F0BF6343F40033D3607047E3
:101A600023F480431B041B0CF4E700BF00ED00E0EF
:101A7000084AD36840B19BB243F0080343F0BF6308
:101A800043F40033D360704723F008031B041B0C9E
:101A9000F4E700BF00ED00E0034AD2F88C3043F4D5
:101AA0004063C2F88C30704700ED00E0084B1A68C4
:101AB00018B142F001021A60704722F001021A6068
:101AC0001A6811B142F00202F5E722F00202F2E7D1
:101AD000D0ED00E02DE9F0430025214C214E54F8D3
:101AE000048CDFF8889085B0A84503D8002005B0A5
:101AF000BDE8F083636A96E807001F6801AB83E8DE
:101B000007000C221946384602F0B3F890B98FB19D
:101B1000636A21691B681A6991420BD19A69A169AC
:101B2000914207D8E169914204D962695B6932EA5E
:101B300003030AD0276A67B10B4801F060FE4040FA
:101B400080F311884FF0040002DFE36801351C4484
:101B5000CAE7484601F053FE636A1F60F5E700BF1D
:101B60003C0200006C420000054800002E480000C6
:101B7000064B1868043B1B68092B05D10138012866
:101B80008CBF002001207047002070473401FF0007
:101B9000054B1868043B1B68092B03D1431E5842B0
:101BA00058417047002070473401FF004E4A08B585
:101BB000136843F002031360FFF7DAFF30B14FF010
:101BC00050230022C3F81421C3F81821FFF7E0FFC7
:101BD00030B10123454A1360A2F63822C2F87835A5
:101BE000434B1B68092B07D1424B1B68022B02BFDA
:101BF0000122414BC3F87825FFF7CAFF10B10E222E
:101C00003E4B1A60FFF7B4FF20B100223C4B1A6034
:101C100001225A600022D30003F57F03D3F800139A
:101C2000013108D0D3F800130132D3F80433B2F5F0
:101C3000807F0B60EFD1334BDA69D1073BD5324B54
:101C40001946D3F80024012AFBD1C3F80425D1F8A2
:101C50000034012BFBD12B4BDA69D20708D5DA69A6
:101C6000294922F00102DA61D1F80024012AFBD1CE
:101C70001A6A01320AD11A6A22F0FF0242F02002E7
:101C80001A62214AD2F80034012BFBD100221E4BEC
:101C9000C3F80425D3F80024012AFBD1BFF34F8FEA
:101CA0001A491B4BCA6802F4E0621343CB60BFF3CE
:101CB0004F8F00BFFDE71B6A0133C0D0134BD3F831
:101CC0008C2042F44062C3F88C20D3F8882042F480
:101CD0007002C3F88820BFF34F8FBFF36F8F0D4B97
:101CE0000D4A1A6008BD00BFD0ED00E0384A005030
:101CF0003001FF003401FF0000400050E4AE03500B
:101D00000C4700500080FF000090035000ED00E001
:101D10000400FA05240000200090D003F8B5002745
:101D2000084B53F82040013053F82060A64200D8F9
:101D3000F8BDD4E900352846984708B105B1AF6031
:101D40000834F3E7E44300000F4B70B505461E4628
:101D50000E4C9C4204D10D4CB44208D1002410E03A
:101D6000A26812B12268AA420BD01034F1E7A3682E
:101D70000BB91034F0E72846216801F06EFF002807
:101D8000F7D1204670BD00BFA000002070000020E9
:101D900008B50B4D4FF02002EFF3118382F3118849
:101DA000BFF36F8F02F0FDF8012104460228D8BF6F
:101DB000084602F006F92C62FFF7C4FAEAE700BF12
:101DC000440700200248034A0021121A01F0A3BF71
:101DD00008010020A407002008B50648064A074964
:101DE000121A01F06DFFBDE80840054A0549064892
:101DF00001F066BF000000200401002078480000C8
:101E0000000000007848000000000020012208B512
:101E1000084B02201A70FFF781FF0320FFF77EFFB7
:101E200000F074FC01F0D4FC034A137B23F001039F
:101E3000137308BDA1070020D00600202DE98048BB
:101E4000DFF8F890A5B089F308880024E023344D2A
:101E50004FF0010B85F82230EC772C766C76AC765F
:101E6000EC766B6A2F4E43F4E0236B626B6ADFF80B
:101E7000D0A043F400236B62AC63FFF7E3FBFFF7F2
:101E80005BFA4FF0FF33AB62EB6240F20113264D79
:101E9000ADF8283007ABAB602046CDE91F44FFF713
:101EA0003DFF0120FFF73AFFDFF8988000F0F6FBD6
:101EB0001E4B6E624FF48062414630460593CDE979
:101EC000034B5346CDE90144009400F0F9FB737BCA
:101ED000304623F00403737301F0B8FF0F23144F4F
:101EE0004FF4A0723846CDE902431249124BCDE9B6
:101EF00004B4CDE9004400F0E3FB7B7B4FF4806247
:101F000023F004037B7305F11803C5E9063341464A
:101F100053463046EF602C75C5F80490FFF7EEF994
:101F200000ED00E0D0060020440700206C480000CF
:101F30005C060020A80B0020911D0000E814002082
:101F40000D1E0000A807002070B50E4B0E4CA342DA
:101F500001D3002070BDD3E9030141EA000212F071
:101F600003020BD19D685A61AA4201D11C33EEE7EE
:101F70005E6901320E6059610144F5E76FF01500AA
:101F8000E8E700BFA0000020A0000020D3B50C4669
:101F900016461F464FF02003EFF3118183F311889B
:101FA000BFF36F8F43695BB123601B684361836933
:101FB00001338361002081F31188BFF36F8F11E03B
:101FC00056EA070203D16FF00B002360F3E70246E5
:101FD000CDE90067044800F009FB18B9034B9B6882
:101FE0005B69236002B0D0BDA20700204407002037
:101FF00070B504460D464FF02003EFF3118683F3CE
:102000001188BFF36F8F01F087FF58B100212A6854
:102010000167426101F01AFF3146BDE8704008488F
:1020200001F0E9BE2B6862691A602B686361A369DD
:10203000013BA36186F31188BFF36F8F70BD00BFB2
:10204000A20700202DE9F341044616461F464FF033
:102050002003EFF3118883F31188BFF36F8FC368F8
:10206000324A6BB180689168884219D056EA0703FA
:1020700018D188F31188BFF36F8F6FF00F000CE059
:10208000916891F90E100133E36093682161A360B8
:1020900088F31188BFF36F8F002002B0BDE8F08194
:1020A0002169F0E790F90E3091F90E109942A8BF1E
:1020B000194621EAE1718B422CDD00F0ABFA0546AE
:1020C00022464146CDE90067194800F08FFA002802
:1020D000E3D04FF02003EFF3118683F31188BFF3B1
:1020E0006F8F236821699C4207D033B193F90E307A
:1020F0009942A8BF194621EAE171A06890F90E3013
:10210000994209D16DB13146094801F074FE6FF072
:102110000A00C2E70025D3E700F07CFA0028F2D1DC
:10212000F0E786F31188BFF36F8FF0E744070020D4
:10213000A207002038B583680446002B36D01E4A1B
:102140009268934235D1DA7B013ADA73C368012B86
:1021500005D0013BC36000F0C3F8002038BD4FF04C
:102160002003EFF3118583F31188BFF36F8F0169AB
:10217000806890F90E30994201D000F04BFA204669
:1021800001F0CAFEA06058B190F90E202261002231
:10219000026701F05BFE2946084801F02CFEDAE7F1
:1021A000E06085F31188BFF36F8FD4E76FF01500FF
:1021B000D4E74FF0FF30D1E744070020A20700200A
:1021C00010B5084C23685BB1FEF70CFD2268064988
:1021D00010440861BDE810400021104601F0F1BE36
:1021E00010BD00BF7C07002044070020F8B50C4656
:1021F0004FF02003EFF3118583F31188BFF36F8F46
:102200004FF4004140F2E73600270022E1FB00676F
:10221000094B30461A6139464FF47A720023FEF7B3
:102220000DF8064B1860064B1C60FFF7C9FF85F3DD
:102230001188BFF36F8FF8BD440700207C07002092
:10224000780700204FF02003EFF3118183F311880A
:10225000BFF36F8F044B9A68D37B013BD37381F339
:102260001188BFF36F8F704744070020094B03F1BB
:102270002802824205D19B688B4202D14B7BDB0650
:1022800006D1D1E9003213605A600023C1E900335E
:10229000704700BF4407002070B5104C064604F19B
:1022A000280001F0C9FD0546A368597B880644BF94
:1022B00041F00801597305B9E5684EB95A7BD20659
:1022C00006D1AA6922B9DA897F2A01D9636270BD71
:1022D000AB4201D0FFF774FF6562F8E744070020C6
:1022E00010B54FF02003EFF3118483F31188BFF38F
:1022F0006F8F084B00209A68D37B0133D373FFF7AD
:10230000CBFF84F31188BFF36F8FBDE8104001F05D
:1023100089BD00BF4407002070B4437BDB062AD18F
:10232000836943BB154A114651F8284F8C4218BFA8
:102330002346002B38BF0023D46AB3B190F90E6056
:1023400093F90E50AE4203DBA3420ED01B68F4E7B4
:102350005A68C0E9003210605860437B63F07F0325
:10236000437370BC0020FFF797BFC0E90014D36A25
:102370001860D062F1E770BC704700BF44070020CE
:1023800010B54FF02002EFF3118482F31188BFF3F0
:102390006F8F427B510704D484F31188BFF36F8F92
:1023A00010BD22F004024273FFF7B6FF2146BDE8DC
:1023B0001040014801F01FBDA20700200146F8B5FA
:1023C0004FF02003EFF3118483F31188BFF36F8F75
:1023D00090F90D30002B02DA1948FFF747FF194A30
:1023E000104650F8283FD56A834208BF0023002BCF
:1023F00038BF0023EBB191F90E7093F90E60B7422C
:1024000003DB9D4215D01B68F4E75868C1E9003032
:10241000016059604B7B906863F07F034B73431AF4
:1024200058425841FFF738FF84F31188BFF36F8F8C
:10243000F8BDC1E90005D36A1960D162EAE700BFBF
:102440006C0700204407002038B5154A154B146866
:1024500001469868A0421C4603D1BDE83840FFF70A
:10246000AFBE00251560104A1268B2B1C2897F2A3A
:1024700013D80E4A90F90E50126895420DDB0C4AA3
:1024800090420AD0826942B91A698A4202DCFFF797
:1024900095FFE2E7521A1A6138BD00232361FBE77A
:1024A00074070020440700207C07002078070020E4
:1024B0005C060020836D2DE9F041044603B1984786
:1024C00004F1180001F057FD4FF02003EFF31186DF
:1024D00083F31188BFF36F8F637BD80623D1A26982
:1024E0000ABB190607D521461E48FFF7BFFE637BCE
:1024F00003F07F0363731C4B9868021B50425041EA
:10250000FFF7CAFE0027637B04F1280843F00803A5
:102510006373A56A454500D095B986F31188BFF36A
:102520006F8FBDE8F0819B07ECD52146A068FFF7CF
:102530009DFE637B23F0020363730023A360E1E746
:1025400005F1180001F017FDA8682946FFF78EFE77
:102550006B7B284623F002036B73AF602F67FFF796
:10256000DBFED6E76C0700204407002008B590F991
:102570000D300146002B06DA0748FFF777FE4B7B4C
:1025800003F07F034B73054B9868431A5842584138
:10259000BDE80840FFF780BE6C070020440700201C
:1025A0002DE9F041064614461D464FF02003EFF397
:1025B000118783F31188BFF36F8F01F082FC87F3DB
:1025C0001188BFF36F8F6B1C08BFB4F1FF3F08D0B9
:1025D00022462B4606F118000349BDE8F04100F001
:1025E00031B9BDE8F08100BF6D3E000010B50C466A
:1025F000064B11469868064B1860DDE90223FFF789
:10260000CFFF2046BDE81040FEF7EABD440700209A
:10261000740700202DE9F04104464FF02003EFF34A
:10262000118883F31188BFF36F8F437B4EB2DB06B3
:102630002ED1856965BB184F214607F12800FFF7A9
:1026400015FEBB6AFA6A834218BF1D46002D38BFCB
:102650000025A673B5B195F90E10B14203DCAA426C
:1026600010D02D68F6E76A68C4E9005214606C6007
:102670000120FFF711FE012088F31188BFF36F8F4F
:10268000BDE8F081C4E90002FB6A1C60FC62EFE770
:102690000020A673F0E700BF440700200021044B90
:1026A000084603F12802C3E90A22FFF79FBD00BFD5
:1026B00044070020014B9868704700BF4407002082
:1026C000F0B500F12805C0E90A5504254573002539
:1026D000044687B0DDE90F67CDE9036786730E9E78
:1026E000C0E9065502960D9E077301960C9EC573B0
:1026F0000096FEF7E9FD044BC4E915559B6803B14C
:102700009B6EA36607B0F0BD440700202DE9F04F93
:10271000DFF8B4902B4DC84687B04D4505F1300425
:102720000DD3FFF78FFD4FF40049264CDFF89CA036
:10273000444521D307B0BDE8F04FFFF7D1BD54F8B1
:10274000043C059354F8103C049354F8143C039350
:1027500054F8183C029354F81C3C019354F8203C64
:10276000009354E90A2354E90C01FFF7A9FF54F838
:10277000303C5D652546D0E7616A4B1C17D040F2BE
:10278000E73B4FF0000C21EAE171C9FB01BC0023DB
:102790004FF47A7258466146FDF750FD0027064611
:1027A00056EA0703256804D12846FFF7E9FD3034CF
:1027B000BEE702463B46514605F1180000F042F8DC
:1027C000F5E700BFA0000020A00000206D3E000043
:1027D000034B1B680BB9FEF705BA0020704700BF1A
:1027E00080070020036840B1074A5268904204D035
:1027F0001BB19A6881680A449A60426813605A6003
:102800000023C0E900337047280000200B4B10B5AF
:102810001C689C4208BF0024FFF7DAFF54B1A3688C
:10282000181A20EAE070064B1B6913B19842A8BF42
:10283000184610BD6FF00040F5E700BF28000020EB
:10284000440700202DE9F74F019119464B1C08BFA2
:10285000B2F1FF3F824661D06FF001034FF0FF3BC2
:10286000541C41F10005B3EB04086BEB0509B8F10A
:10287000000F79F100030FDBFFF7AAFF6FF00103F0
:102880002B4AD2E9001C5B1A6BEB0C021E1B62EB9D
:102890000507341A67EBE075019BCAF80C304FF05E
:1028A0002003EFF3118683F31188BFF36F8FFFF7D7
:1028B0008FFF012C75F10003B8BF01241D4B20448C
:1028C0001A68CAF808009A4201D05C6852B95A687E
:1028D000CAF80030CAF804205A68C2F800A0C3F849
:1028E00004A00DE09068DAF80810884219DD411A5A
:1028F00091605168CAE90021C1F800A0C2F804A0A3
:102900001A689A4206D0924504D1FFF77FFF002152
:10291000FEF704F986F31188BFF36F8F03B0BDE8AB
:10292000F08F091A9442CAF80810D0D01268CDE787
:1029300008010020280000202DE9F0470646FFF797
:1029400083FD4FF02003EFF3118483F31188BFF36D
:102950006F8FDFF884801F4DC146DFF880A02E60A6
:10296000DAF800002A685045D8E9006705D020B1A0
:102970008368934213DD9B1A8360B61847EBE277B6
:10298000C9E9006700262E60FFF740FF3146FEF7D9
:10299000C5F884F31188BFF36F8FBDE8F087F61890
:1029A00047EBE377D31A2B6000238360C8E9006705
:1029B000FFF718FF84F31188BFF36F8FC368984740
:1029C0004FF02003EFF3118483F31188BFF36F8F6F
:1029D000C6E700BF80070020080100202800002073
:1029E00038B5064C064DAC4201D3002038BD204618
:1029F000D4E9011201F000FB1434F4E7A000002038
:102A0000A000002001F045B90A46002101F083B979
:102A100010B5114800F048F800B110BD0F4800F0A3
:102A200043F80028F9D10E4C204600F03DF800286C
:102A3000F3D10C4B0C481C6000F036F8014600281E
:102A4000EBD100F02DF8044608B1204610BD00F08F
:102A500051F82046FAE700BF3C000020300000207B
:102A600038000020400000203400002008B508484D
:102A700000F024F8074800F021F8074800F01EF89D
:102A8000064800F01BF8BDE8084000F00BB800BF96
:102A90003C000020300000203800002034000020DE
:102AA00000207047704700BF08B5034B02681B68E1
:102AB00010689847002008BD4C00002008B5034B63
:102AC00002685B6810689847002008BD4C00002031
:102AD0000268024B10689B68184700BF4C0000203A
:102AE00008B5034B0268DB6810689847002008BDF2
:102AF0004C00002070B5094C094D2069AB6898471F
:102B000018B1084B08485B6898470021074AEB68F2
:102B100011602069BDE87040184700BF5C000020CC
:102B20004C00002044000020FC43000084070020EB
:102B3000F8B51A4C1A4D0746AB6820699847E8B9B2
:102B4000184E33687FB93BB90120174A1749C2F8BC
:102B500000050A68002AFCD101333360EB68206964
:102B600098470020F8BD002BF8D0012B08D0013B7E
:102B700033602069EB6898470020F3E70C48F8BD04
:102B80000A4A1368002BFCD1074A6FF07E40C2F856
:102B9000003500F021F83368E9E700BF5C00002051
:102BA0004C0000208407002000008450101984503D
:102BB000E98FFFFF0020704700207047430503D5D1
:102BC0004FF0FF32024B1A60024B1860704700BF93
:102BD00008118450081A8450014B1860704700BFD8
:102BE000041A845008B100F003B84FF47500704720
:102BF0000246074803681342FCD021B1054B064842
:102C00001B680B600360054B00201A60704700BF13
:102C1000001A84500411845008118450081A8450FA
:102C200000F0A0B830B129B1002301440370013095
:102C30008142FBD1704700BF2DE9F041ADF51A7D0F
:102C40000F4605920021144612A84FF408721E4642
:102C500001F061F8002308A819462822069301F024
:102C60005AF8002F3CD0002E3AD0002C38D0042146
:102C700006A8FFF7C9FE08A82821FFF7C5FE08A887
:102C800000F032F878B14FF0FF3512A84FF4087118
:102C9000FFF7C8FF06A80421FFF7C4FF28460DF57B
:102CA0001A7DBDE8F08112AB0DF11C080390CDE94F
:102CB0000163024605AB08A9CDF8008006A800F024
:102CC000E9FC0028DFD13368A342DCD3D8F8001038
:102CD0000546083138462246FFF794FE3460D4E7B3
:102CE0004FF0FF35DAE700BF1C2330B583B002A9EF
:102CF00041F8043D044600F0B1F90546D8B9019BFE
:102D00001C2B1BD1D4E9003201210033E16118BF33
:102D100001230AB143F00203A26832B9E268AAB9FA
:102D2000C4E908323BB90D4D09E0E26843F0040301
:102D300062B9C4E90832284603B030BD084D2046C8
:102D40001C21FFF761FE284603B030BD0022284653
:102D500043F00803C4E9083203B030BD0E0CF000A4
:102D6000370CF00010B50C4C236813B10B4B1B68EB
:102D70006BB900F031F938B10138062896BF084B1D
:102D8000084853F8200010BD0122044B1A600123AB
:102D90000020236010BD00BF880700208C070020A2
:102DA0001C440000FE8FFFFF10B5094C23681BB1C7
:102DB00001230020236010BD00F07CF80028F7D02C
:102DC0000138062896BF034B034853F8200010BD76
:102DD000880700201C440000FE8FFFFFBFF34F8FC9
:102DE0000549064BCA6802F4E0621343CB60BFF3A7
:102DF0004F8F00BFFDE700BF00ED00E00400FA05C3
:102E0000014B5B68184700BF44000020024BD0E92B
:102E10000012C3E90012704744000020704700BF51
:102E200010B5044620B1BFF35F8F0020206010BDB5
:102E30000348FFF7E5FFBFF35F8F0020206010BD60
:102E40005C44000010B5044610B10023236010BD9F
:102E50000248FFF7D5FF0023236010BD384400006F
:102E600050B10122D0E8EF3FC0E8E12F0029F9D1AD
:102E7000012BF7D0BFF35F8F0020704770B40B4B6E
:102E80000668C268D0E90154C3E90242C3E900659B
:102E9000D1E903020E68064BD1E90154C3E900658C
:102EA000C3E902401A6170BC704700BF4C000020AB
:102EB0005C00002010B5FFF77DFE70B9FFF7A8FD9C
:102EC00080B9FFF735FE80B9114B1B681B0EF02B44
:102ED0000DD00624FFF770FE00E00324FFF7C6FDC7
:102EE000204610BD0424204610BD0024F2E7094A04
:102EF000094B12689A4201D00724EBE70120FFF743
:102F000017FE0028F1D1054B04461860E8E700BF22
:102F100028198450241A84500000E0200C1A845090
:102F200030B5ADF5157D4FF4087200210CA800F006
:102F3000F2FE002302A819462822019300F0EBFEBE
:102F400002A8FFF7D1FE18B105200DF5157D30BDA3
:102F50001C4D4FF0FF312868FFF7BAFD0446F0B969
:102F60000020FFF7E5FDB0B90CAA02A901A800F006
:102F7000D5FB04460120FFF7DBFDF0B92868FFF719
:102F8000AFFD10B11048FFF73BFF2046002CDBD10E
:102F90000DF5157D30BD0D48FFF732FFE4E70C4815
:102FA000FFF72EFF012CDBD12868FFF799FD0028E1
:102FB000CAD00548FFF724FFC6E70648FFF720FF01
:102FC000DCE700BF4000002094440000AC44000057
:102FD0007C440000CC44000008B5FFF7EBFD18B1BD
:102FE000FFF744FD032008BDFFF712FD68B9FFF7A6
:102FF0009FFD60B9154B1B681B0EF02B12D0FFF71D
:10300000DBFDFFF733FD062008BD042008BDFFF7F8
:10301000D3FDFFF72BFDFFF783FF00280CBF002037
:10302000052008BD0A4A0B4B12689A4205D0FFF7EB
:10303000C3FDFFF71BFD072008BD0120FFF778FD4A
:103040000028E4D1044B1860E5E700BF281984503C
:10305000241A84500000E0200C1A845018B111B1D9
:103060000B681C2B01D0012070474FF47F033A4AB4
:10307000D3F8101C91425AD0D3F8102C013256D0FC
:10308000D3F8102C4FF47F030260D3F8141C334A9A
:1030900091425ED0D3F8142C01325AD0D3F8142CBC
:1030A0004FF47F034260D3F8182C12F5947F4DD073
:1030B000D3F8182C013249D0D3F8182C4FF47F03E1
:1030C0008260D3F81C1C264A91423CD0D3F81C2CB9
:1030D000013238D0D3F81C2C4FF47F03C260D3F8F0
:1030E000002C70322DD0D3F8002C013229D0D3F827
:1030F000002C4FF47F030261D3F8042CAF321ED0B2
:10310000D3F8042C01321AD0D3F8042C4FF47F03E7
:103110004261D3F8081C134A91420BD0D3F8082C13
:10312000013207D0D3F8083C83610020704740F695
:10313000FC02A7E740F23733836100207047512239
:10314000E4E79022D5E742F60412C5E740F6D862DC
:10315000B4E742F2D002A3E7FCF8FFFFD020FFFF64
:103160000429FFFF37F3FFFFA8B32DE9F0414C1E00
:10317000B4F5047F2CD25BB352B34FF0000CC900FE
:10318000E646654664464F1E03F1FF380CE0AB424D
:1031900016D08E4501D10CF1010CA84516D0013492
:1031A000BC4205F1010518D8610950F8211004F05E
:1031B0001F06F1401F2E18BF01F00101002CE6D1BF
:1031C0000025A8458E464FF0010CE8D16245E6D2B5
:1031D0000348BDE8F081024870470020BDE8F08157
:1031E000370CF1002DE9F04F8FB00D46DDE91941A4
:1031F0008346002957D12969039100211C60189B3F
:103200001960002A00F02281814A824B11686A6AA3
:103210001B689A4257D10A2955D19BF8033006936F
:103220000399042308467C4A0293A2FB00029208F9
:10323000CB0002EB420204F10800A1EB4202013B89
:10324000DFF8D091DFF800A2049000920593189B5C
:10325000039C1C60002C00F0CC800026049F00F032
:10326000A9FA00230793069BBBF1000F3AD0002D6B
:1032700034D053BB5B000693BBF1000F36D0002D5A
:1032800034D0E3B106A9284600F084FA002800F003
:103290007D81624B984212D0009000F08BFA00982A
:1032A0000FB0BDE8F08F4FF47F01D1F80C0C013066
:1032B0000CBF4FF40471D1F80C1C03919DE72B6AED
:1032C00073B95648E8E75648E6E706A9284600F0ED
:1032D00061FA68B1534B9842DED0069B082BC9D1E6
:1032E0005148D9E7082BFBD05B0006934F48D3E742
:1032F0002946069800F030FA0028EBD1069B082BEF
:1033000000F00E81042B00F03181A3F10203B3FA27
:1033100083F35B09019301231946454A136042F880
:10332000843C434B19606B6AC9F80030D9F800201F
:103330006B6A9A42F5D14FF000084FF0FF30CAF89F
:103340000080FFF73BFC3B4A3B4B40461A60FFF7CF
:1033500043FC0A22019839492D4B08601A602A69FA
:10336000A8F15538A8FB02126B6A120903EB43035C
:10337000DB0303FB02F3324A9B0913600123CAF803
:1033800000300699DBF800200B0243EA016322F0CB
:103390007F421343CBF8003007A800F0CDF9002896
:1033A00098D1284BA8FB04281A681433089253F8C4
:1033B000102CB6EB980F099253F80C2C0A9253F884
:1033C000082C0B9253F8042C0C921B680D9301D11E
:1033D000009B9BB93846182208A9FFF713FB183C3D
:1033E00018370136002C7FF43AAF049B002B40F0D5
:1033F0009A800023189A1360069B6FE71A46384696
:1034000008A9E41AFFF7FEFA009B1F44E9E700BF92
:103410003811845030118450ABAAAAAA310CF100A3
:10342000300CF100020CF100320CF100350CF1000F
:10343000C4118450FEFFFF0F001184500C11845002
:10344000D8118450141184502C118450BBF1000FFA
:103450003FF44CAF002D3FF449AF01230EA941F8D2
:10346000203DCBF80020284600F094F900287FF496
:1034700013AF2946069800F06FF900287FF40CAFCF
:10348000069F082F00F0EB80042F00F0EA80A7F1E0
:103490000207B7FA87F77F0901221646734B744972
:1034A0001A6018460A60943B06606A6A1A601968D6
:1034B0006A6A9142F8D14FF000086E4B4FF0FF302E
:1034C000C3F80080FFF77AFB6B4B6C4A40461A60EA
:1034D000FFF782FB0A226A496A4B0F601A601A9949
:1034E0002B6901296A6A00F0B1806749A1FB0313C7
:1034F0001B09012102EB4202D20303FB02F3634AE0
:103500009B0913605B4B19600699DBF800200B02E6
:1035100043EA016322F07F421343CBF800307FE699
:1035200003230193F7E6039BB3F5047F3FF661AFF6
:10353000DDE9047C204623466E6904E00120013366
:103540006345144615D85A0957F8222003F01F0185
:10355000CA401F2918BF02F00102002BEED0A24280
:10356000ECD101308642EAD149480BE002230193B5
:10357000D1E64FF48063DDE90310AA69FFF7F4FD9B
:1035800000285DD00023189A1360A3E62946069808
:1035900000F0E2F800287FF47CAE069C082C51D0A5
:1035A000042C51D0A4F10204B4FA84F46409012378
:1035B0001E4619462D4A136042F8843C2B4B196075
:1035C0006B6AC9F80030D9F800206B6A9A42F5D1CD
:1035D00000274FF0FF30CAF80070FFF7EFFA264BD4
:1035E000264A38461A60FFF7F7FA0A222449254B83
:1035F0000C601A602A6924496B6AA1FB021203EB72
:1036000043031209DB0303FB02F3204A9B09136007
:10361000CAF80060069BDBF800101A0242EA036356
:1036200021F07F421A43130A03F47F03134323F06C
:103630007F43CBF80030029B013B02937FF407AE3F
:10364000002029E60324B2E70224B0E74FF47F0309
:10365000D3F80C1C013106D0D3F80C3C45E7032706
:103660001AE7022718E7162343E700BFC411845066
:10367000401184502C11845000118450FEFFFF0F24
:103680000C11845038118450ABAAAAAAD8118450C6
:10369000360CF1002DE9F0431B4C85B00746DDE9FF
:1036A0000D56884620684FF0FF319146FFF710FA1B
:1036B00028BB0020FFF73CFAE8B90023CDE900560B
:1036C00002934A46414638460C9BFFF78BFD054660
:1036D0000120FFF72DFA50B92068FFF701FA10B169
:1036E0000A48FFF78DFB284605B0BDE8F08308487F
:1036F000FFF786FBF0E70748FFF782FBDDE70648A8
:10370000FFF77EFBD5E700BF400000209444000097
:10371000CC440000AC4400007C44000010B50124FF
:1037200086B005ABCDE901240093002204ABFFF77E
:1037300059FD06B010BD00BF08B501464FF48060CA
:10374000FFF750FA00230249024A0B60136008BDDC
:10375000C81184502C1184500138072815D8DFE88F
:1037600000F0100C140814141404CB6800204B62F1
:1037700070478B6800204B6270474B6800204B629B
:1037800070470B6800204B6270470148704700BFCC
:10379000310CF1000B6802E0082B0B6006D8026ABE
:1037A00013424FEA4303F7D00020704700487047A8
:1037B000310CF10000230449044A0B604FF480608F
:1037C0001360FFF7FBB900BF2C118450C411845063
:1037D00008B5FDF711FBBDE80840FDF7A3BA0020CE
:1037E000704770B50D4604464520A0472946522033
:1037F000A04729462346BDE87040522018470FB421
:1038000007B504A951F8040B0191FDF7AFF803B017
:103810005DF804EB04B07047044608B5084611464D
:103820001A46A047FEF746FFFDF740FF036803EB8B
:10383000C1018368B3F5004F2CBF51F8220031F865
:103840001200704710B50468806804EBC101B0F540
:10385000004F2CBF41F8223021F8123010BD2DE965
:10386000F041044600220D46FFF7E0FFE268A3683E
:103870001040B3F5004FB0FA80F234BF00200120B1
:103880006368C0F11F00801A03EBC0014A68561C30
:103890004E60A2B9012202FA00F162690A43626134
:1038A000294643F8305002222B462046FFF7CAFF34
:1038B000032229462046BDE8F041FFF7C3BF53F875
:1038C0003070022239462046FFF7B0FF0646034615
:1038D000022229462046FFF7B5FF3B460322294630
:1038E0002046FFF7AFFF032231462B462046FFF765
:1038F000A9FF02223946DDE7F8B58B1847F6FF72BB
:10390000CC1D24F0070423F007031B1BDB08B3F5D1
:10391000004F2CBF6FF0004111460460002093421D
:10392000E16094BF00210121B3FA83F61746844673
:10393000C1F1200104F11805891B21F06041C4E99F
:1039400001530331246060612161A268BA4294BFCF
:1039500000220122C2F11F02921B90420ADD204682
:103960005B1A0022FFF76EFF20462169BDE8F84090
:10397000FFF775BFC5F804C0013045F808CBE4E790
:103980007047FEF713B90C22C368C9B202FB0131BC
:103990004B7A23B9087AB0FA80F0400970470220C8
:1039A000704770B5C9B24468C5684FF02003EFF3A3
:1039B000118683F31188BFF36F8F0C224A43AB1833
:1039C000187A90B10138C0B2187288B904EB81013D
:1039D000A850CA78012102F1502258601160587233
:1039E00086F31188BFF36F8F70BD6FF04400F7E767
:1039F0000020F5E72DE9F8434668D0F80CE0CFB297
:103A00004AB10C237B435EF803309A4252D013B183
:103A10001B68002BF9D14FF02003EFF3118C83F3D7
:103A20001188BFF36F8F0C257D430EEB05031C7AC5
:103A30000134E4B21C728CF31188BFF36F8F5AB358
:103A40004FF0502C4FF00308CCF8088393F809C0CE
:103A5000BCF1000F15D14FF02008EFF3118988F366
:103A60001188BFF36F8FC2F800C0D3F80480B8F19B
:103A7000000F1BD15A604EF8052089F31188BFF35F
:103A80006F8F4FF050230325C3F80453BCF1000F90
:103A900002D0D2E901329847012C05D106EB870606
:103AA000B37803F150231C60002005E0C8F8002023
:103AB0005A60E2E76FF00F00BDE8F8830022FFF7DD
:103AC00099BF10B50022044601210520FDF7E6FB51
:103AD0000520FDF7D3FB4FF050230222C3F8182531
:103AE00003220020C3F80423E368C3E90000E3686D
:103AF000C3E9030010BD70477047002307B501A854
:103B00008DF80430FFF78CF803B05DF804FB9029C2
:103B100008B5134639D10A4601460020FFF78CF854
:103B2000BDE80840714672467346B7EE000AF7EEEC
:103B3000000AB7EE001AF7EE001AB7EE002AF7EE09
:103B4000002AB7EE003AF7EE003AB7EE004AF7EE79
:103B5000004AB7EE005AF7EE005AB7EE006AF7EEE9
:103B6000006AB7EE007AF7EE007A8EF3008C10B49C
:103B7000F1EE10CA4FF66074C0F6FF740CEA040C44
:103B8000E1EE10CA10BCF44674476FF01500C7E7A9
:103B9000FEE70021012000F029B843B2A9B1002BB3
:103BA00012DB01215B099B0003F1604303F56143D4
:103BB000D3F8802200F01F0001FA00F022EA000092
:103BC000C3F88002D3F880327047002BFCDB01225F
:103BD0005B099B0003F1604303F56143D3F8801256
:103BE00000F01F0002FA00F00843E9E700F0C3B854
:103BF0000146006800F0BFB808B5FDF7B1FBBDE8AD
:103C00000840FDF727BD30B54B680C6885B00A89C0
:103C10008D7A0094013B24F01F04234402F01F021C
:103C200042EA451223F01F030F2804468DF80820AE
:103C3000039305D86946FDF789FD204605B030BDE0
:103C40006FF01504F9E740E800F0C3B210F4803FCC
:103C500014BF18466FF0150070470138013910F88D
:103C6000013F11F8012F934201D1002BF7D1981A8F
:103C7000704710B55AB10139841810F8012B11F8AA
:103C8000013FA04201D09A42F7D0D01A10BD104691
:103C9000FCE7431A934210B500EB020308D3024637
:103CA00001399A420BD011F8014F02F8014BF8E7A5
:103CB0000A4412F8014D8A4203F8014DF9D110BDB2
:103CC000F0B581EA0004A50703460BD0013B0A4486
:103CD00091421BD1F0BD002AFCD011F8014B013AF2
:103CE00003F8014B9C07F6D122F003041D1F960830
:103CF0000F19B94205D16FF00305234405FB0622D5
:103D0000E4E751F804CB45F804CFF2E711F8014B92
:103D100003F8014FDCE7034670B5C9B29C0711D127
:103D200041EA012422F0030644EA04451E449408B3
:103D3000B3420DD16FF0030505FB04221A449342F0
:103D400009D170BD002AFCD003F8011B013AE5E758
:103D500043F8045BECE703F8011BF0E7002008B52B
:103D6000FDF786FC08B5FDF7A1F9FDF723FABDE8DC
:103D70000840FFF719B873B5054601914FF02003CD
:103D8000EFF3118683F31188BFF36F8FFEF792FC78
:103D9000019904462846FFF7E1FF86F31188BFF337
:103DA0006F8F204602B0BDE87040FDF77FBCFFF783
:103DB000A3BE30B50024846141EA020414F0030478
:103DC000C0E9023201610CD14461A34203D1C0E9D0
:103DD0000000002030BD456901340D60416111448F
:103DE000F3E76FF01500F5E70023C0E90000C0E934
:103DF00002331846704721B9EFF3058008B9FDF783
:103E0000EFB981F31188BFF36F8F7047034620B974
:103E1000EFF305820AB9FDF7E3B983F31188BFF325
:103E20006F8F70474FF02003EFF3118083F31188F9
:103E3000BFF36F8FFFF7EABF0368984204D0002BEF
:103E400038BF0023184670470020704710B54FF068
:103E50002003EFF3118483F31188BFF36F8FFEF714
:103E60005BFA84F31188BFF36F8F10BD38B550F83B
:103E7000103C0446A0F11801C3B14FF02003EFF34A
:103E8000118583F31188BFF36F8F50F8100CFEF784
:103E9000EDF914F80B3C23F0020304F80B3C00236B
:103EA00044F8103C85F31188BFF36F8F14F80B3C76
:103EB000084623F0140304F80B3CBDE83840FFF734
:103EC000C5BF38B504460D46FEF750FB637B43F093
:103ED00002036373C5B12B68A5609D4208BF002330
:103EE000002B38BF002383B194F90E1093F90E20F4
:103EF000914204DB6A689A4207D01B68F3E75A686C
:103F0000C4E9003214605C6038BD6B682560636092
:103F10006B681C606C60F7E738B54FF02003EFF377
:103F2000118283F31188BFF36F8FFFF785FF04467B
:103F300082F31188BFF36F8FC8B14FF02003EFF306
:103F4000118583F31188BFF36F8F01468068FEF7F8
:103F50008DF9637B23F0020363730023A36085F371
:103F60001188BFF36F8F04F1180000F004F82046A9
:103F700038BDFCF71DBD10B54FF02002EFF31184E2
:103F800082F31188BFF36F8F03683BB1FEF72AFC01
:103F9000002084F31188BFF36F8F10BD6FF0150000
:103FA000F7E710B54FF02003EFF3118483F3118886
:103FB000BFF36F8FFEF72AFC84F31188BFF36F8F76
:103FC00010BD37B5044601914FF02003EFF3118582
:103FD00083F31188BFF36F8FFEF718FC012805DD0E
:103FE000A042019902DD2046FCF798FD85F3118877
:103FF000BFF36F8F03B030BD10B400F10C04C0E903
:1040000003445DF8044BFFF777BC704760C2FF7F45
:10401000010000008909000000000000491F0000A5
:1040200000000000E129000000000000DD18000091
:1040300000000000C33A000070000020B50A000034
:1040400080000020653D000090000020D51A00008F
:104050000000000000000000933B00000000000092
:10406000933B000000000000933B000000000000B4
:10407000933B000000000000933B000000000000A4
:10408000150A000000000000933B00000000000043
:10409000933B000000000000933B00000000000084
:1040A000933B000000000000933B00000000000074
:1040B000933B000000000000933B00000000000064
:1040C000933B000000000000933B00000000000054
:1040D000933B000000000000933B00000000000044
:1040E000933B000000000000933B00000000000034
:1040F000933B000000000000933B00000000000024
:10410000910A000000000000933B00000000000046
:10411000933B000000000000933B00000000000003
:10412000933B000000000000933B000000000000F3
:10413000933B000000000000933B000000000000E3
:10414000933B000000000000933B000000000000D3
:10415000933B000000000000933B000000000000C3
:10416000933B000000000000933B000000000000B3
:10417000933B000000000000933B000000000000A3
:10418000933B000000000000933B00000000000093
:10419000933B000000000000933B00000000000083
:1041A000933B000000000000933B00000000000073
:1041B000933B000000000000933B00000000000063
:1041C000933B000000000000933B00000000000053
:1041D000933B000000000000933B00000000000043
:1041E000933B000000000000933B00000000000033
:1041F000933B000000000000933B00000000000023
:10420000933B000000000000933B00000000000012
:10421000933B000000000000933B00000000000002
:10422000933B000000000000933B000000000000F2
:10423000933B000000000000933B000000000000E2
:10424000933B000000000000933B000000000000D2
:10425000933B000000000000933B0000FFFFFFFFC6
:10426000DEE61E284CBBCE8F025B0000DEE61E2879
:10427000EAAC45B8025B0000DEE61E284CBBCE8FE0
:10428000025B0000000000000000000000000000D1
:104290000338FDD870470000BD3A0000A339000084
:1042A000F53900000000000087390000A746000033
:1042B00042010000AE46000005010000B8460000C3
:1042C00014010000C146000015010000CA460000AC
:1042D00039010000D346000009010000DE4600005D
:1042E0000A010000E94600000A010000F346000050
:1042F0000B010000FD4600000F0100000847000010
:104300001001000013470000110100001E470000CB
:104310000E01000028470000210100003147000085
:10432000220100003A47000023010000434700003B
:10433000240100004C470000180100005447000011
:104340002A0100005C4700003A01000064470000B9
:104350002C0100006C4700001C01000075470000A4
:104360001D0100007E470000170100008847000083
:10437000310100009447000004010000000000002B
:10438000000200000004000000080000001000000F
:1043900000000000913B000019110000D91000003E
:1043A00081110000B91000001C0000200400002052
:1043B00014000020000000000C000020020000009B
:1043C000C443000000000000F647000006000000A3
:1043D000E0FF0F0000000020FE4700002100000069
:1043E000E0FF0020144000003C400000444000007A
:1043F0005440000054400000F5FFFFFF436F756C10
:1044000064206E6F74206C6F636B20706F776572C1
:104410002073617665206D7574657800FF8FFFFFEE
:10442000FF8FFFFFFE8FFFFFFE8FFFFFFD8FFFFF60
:10443000FC8FFFFFFC8FFFFF43616E277420696EC6
:10444000697469616C697A65206D757465782C2072
:10445000776173204E554C4C0D0A000043616E2766
:104460007420756E6C6F636B206D757465782C208D
:10447000776173204E554C4C0D0A00004661696C03
:1044800020746F2061637175697265206D75746544
:10449000780A00004661696C20746F2072656C6553
:1044A000617365206D757465780A00004661696CFA
:1044B00020746F20696E63726561736520504D20B2
:1044C000636F756E7465720A000000004661696C66
:1044D00020746F20646563726561736520504D20A0
:1044E000636F756E7465720A0000000100040401B8
:1044F000080C7379735F636C6F636B00536563754E
:1045000072650909004E6F6E2D53656375726509FA
:104510000025303275202530327520307825303531
:1045200078203078253035782009002563005350F5
:104530004D3A204E5320696D6167652061742030CB
:104540007825780A0053504D3A204E53204D535051
:1045500020617420307825780A0053504D3A204E5F
:104560005320726573657420766563746F72206181
:104570007420307825780A0053504D3A20707265C7
:104580007061726520746F206A756D7020746F2081
:104590004E6F6E2D53656375726520696D61676539
:1045A0002E0A004E6F6E2D53656375726500466C62
:1045B00061736820726567696F6E730909446F6D76
:1045C00061696E09095065726D697373696F6E7305
:1045D0000A004E6F6E2D7365637572652063616CA2
:1045E0006C61626C6520726567696F6E2030207047
:1045F0006C6163656420696E20666C61736820720B
:104600006567696F6E202564207769746820736917
:104610007A652025642E0A00436F756C64206E6FE6
:104620007420696E697469616C697A652073656369
:10463000757265207365727669636573202865728B
:1046400072202564292E0A005352414D207265675D
:10465000696F6E0909446F6D61696E090950657271
:104660006D697373696F6E730A0050657269706863
:104670006572616C0909446F6D61696E0909537453
:10468000617475730A002530327520252D3231731F
:1046900025730009534B49500A00094552524F52A5
:1046A0000A00094F4B0A004E52465F5030004E52EE
:1046B000465F434C4F434B004E52465F525443308B
:1046C000004E52465F52544331004E52465F4E56A2
:1046D0004D43004E52465F554152544531004E52B3
:1046E000465F554152544532004E52465F54574939
:1046F0004D32004E52465F5350494D33004E5246A4
:104700005F54494D455230004E52465F54494D4525
:104710005231004E52465F54494D455232004E527E
:10472000465F5341414443004E52465F50574D301F
:10473000004E52465F50574D31004E52465F505723
:104740004D32004E52465F50574D33004E52465F39
:10475000574454004E52465F495043004E52465F04
:10476000564D43004E52465F465055004E52465FEE
:1047700045475531004E52465F45475532004E522F
:10478000465F4450504943004E52465F4750494FA0
:10479000544531004E52465F524547554C41544FA7
:1047A0005253006D757465785F696E69742063613A
:1047B0006C6C65642077697468204E554C4C207091
:1047C0006172616D6574657200436F756C64206E13
:1047D0006F7420616C6C6F63617465206D757465B6
:1047E00078206265666F726520696E697469616CB4
:1047F000697A696E6700464C4153485F30005352F6
:10480000414D5F30004552524F523A2043616E6E27
:104810006F742066756C66696C6C204558545F41F6
:10482000504920726571756573742E0D0A005741E9
:10483000524E494E473A204F7074696F6E616C203A
:104840004558545F415049207265717565737420F5
:104850006E6F742066756C66696C6C65642E0D0AEB
:104860000048575F43433331305F30006D61696EFC
:104870000000000000000000DF370000B40000204E
:1048800001000000C800002001000000DC00002042
:1048900001000000F0000020010000000090D003A3
:1048A0002800002028000020600000206C0000206C
:1048B000640000205C0000203800002000000000A0
:1048C000DD2D0000452E00001D2E0000612E000091
:1048D000212E00009C070020900700209807002050
:1048E0000000000094070020B2460000EA440000E7
:1048F0009842000010010020F24400000000000077
:1049000000000000000000006148000000000000FE
:104910000000000000000000A0000020A000002017
:1049200000000000000000000F000000B4000020A4
:10493000B400002000000000000000000F00000094
:10494000C8000020C8000020000000000000000097
:104950000F000000DC000020DC0000200000000050
:10496000000000000F000000F0000020F000002018
:1049700000000000000000000F000000FFFFFFFF2C
:104980000000000000000000000000000000000027
:104990000000000000000000000000000000000017
:1049A0000000000000000000000000000000000007
:1049B00000000000000000000000000000000000F7
:107FE0007FE97FE9F8F7A0BF7FE97FE9F8F7F4BF01
:107FF0007FE97FE9FBF78BBD000000000000000077
:10C00000C0CF022099330100A5330200C9330100DB
:10C01000C9330100C9330100C9330100C93301002C
:10C02000000000000000000000000000B13001002E
:10C03000C9330100000000000D300100DD320200B4
:10C0400059330100593301005933010059330100BC
:10C0500059330100593301005933010059330100AC
:10C06000593301005933010059330100593301009C
:10C07000593301005933010059330100593301008C
:10C08000593301005933010059330100593301007C
:10C09000593301005933010059330100593301006C
:10C0A000593301005933010059330100593301005C
:10C0B000294D01004B48020059330100593301005A
:10C0C000593301005933010059330100593301003C
:10C0D000593301005933010059330100593301002C
:10C0E00059330100593301006948020059330100F6
:10C0F000593301005933010059330100593301000C
:10C1000059330100593301005933010059330100FB
:10C1100059330100593301005933010059330100EB
:10C1200059330100593301005933010059330100DB
:10C1300059330100593301005933010059330100CB
:10C140005933010000000000000000000000000062
:10C1500000000000000000000000000000000000DF
:10C1600000000000000000000000000000000000CF
:10C1700000000000000000000000000000000000BF
:10C1800000000000000000000000000000000000AF
:10C19000000000000000000000000000000000009F
:10C1A000000000000000000000000000000000008F
:10C1B000000000000000000000000000000000007F
:10C1C000000000000000000000000000000000006F
:10C1D000000000000000000000000000000000005F
:10C1E000000000000000000000000000000000004F
:10C1F000000000000000000000000000000000003F
:10C20000DEE61E284CBBCE8F025B00003C00000027
:10C2100074E101000100000000C0000000C0000047
:10C22000FFFF02910000000000000000000000007D
:10C23000000000000000000000000000FFFFFFFF02
:10C2400081F0004102E000BF83F0004330B54FEAC7
:10C2500041044FEA430594EA050F08BF90EA020F34
:10C260001FBF54EA000C55EA020C7FEA645C7FEAC7
:10C27000655C00F0E2804FEA5454D4EB5555B8BFEA
:10C280006D420CDD2C4480EA020281EA030382EA5B
:10C29000000083EA010180EA020281EA0303362DED
:10C2A00088BF30BD11F0004F4FEA01314FF4801CC0
:10C2B0004CEA113102D0404261EB410113F0004FD2
:10C2C0004FEA03334CEA133302D0524263EB430389
:10C2D00094EA050F00F0A780A4F10104D5F1200E27
:10C2E0000DDB02FA0EFC22FA05F2801841F1000182
:10C2F00003FA0EF2801843FA05F359410EE0A5F156
:10C3000020050EF1200E012A03FA0EFC28BF4CF086
:10C31000020C43FA05F3C01851EBE37101F000453C
:10C3200007D54FF0000EDCF1000C7EEB00006EEB49
:10C330000101B1F5801F1BD3B1F5001F0CD34908D3
:10C340005FEA30004FEA3C0C04F101044FEA44522A
:10C3500012F5800F80F09A80BCF1004F08BF5FEAB1
:10C36000500C50F1000041EB045141EA050130BD91
:10C370005FEA4C0C404141EB0101013C28BFB1F5A3
:10C38000801FE9D291F0000F04BF01460020B1FAEE
:10C3900081F308BF2033A3F10B03B3F120020CDAC1
:10C3A0000C3208DD02F1140CC2F10C0201FA0CF09F
:10C3B00021FA02F10CE002F11402D8BFC2F1200C04
:10C3C00001FA02F120FA0CFCDCBF41EA0C019040BA
:10C3D000E41AA2BF01EB0451294330BD6FEA040403
:10C3E0001F3C1CDA0C340EDC04F11404C4F12002EE
:10C3F00020FA04F001FA02F340EA030021FA04F300
:10C4000045EA030130BDC4F10C04C4F1200220FA56
:10C4100002F001FA04F340EA0300294630BD21FA94
:10C4200004F0294630BD94F0000F83F4801306BF5A
:10C4300081F480110134013D4EE77FEA645C18BF4E
:10C440007FEA655C29D094EA050F08BF90EA020FE5
:10C4500005D054EA000C04BF1946104630BD91EADD
:10C46000030F1EBF0021002030BD5FEA545C05D1E0
:10C470004000494128BF41F0004130BD14F580041F
:10C480003CBF01F5801130BD01F0004545F0FE4193
:10C4900041F470014FF0000030BD7FEA645C1ABFC8
:10C4A000194610467FEA655C1CBF0B46024650EAFF
:10C4B000013406BF52EA033591EA030F41F400212B
:10C4C00030BD00BF90F0000F04BF0021704730B5B1
:10C4D0004FF4806404F132044FF000054FF0000186
:10C4E00050E700BF90F0000F04BF0021704730B547
:10C4F0004FF4806404F1320410F0004548BF40421C
:10C500004FF000013EE700BF42004FEAE2014FEA70
:10C5100031014FEA02701FBF12F07F4393F07F4F4B
:10C5200081F06051704732F07F4208BF704793F04E
:10C530007F4F04BF41F40021704730B54FF4607461
:10C5400001F0004521F000411CE700BF50EA010264
:10C5500008BF704730B54FF000050AE050EA01020D
:10C5600008BF704730B511F0004502D5404261EB7D
:10C5700041014FF4806404F132045FEA915C3FF4BE
:10C58000D8AE4FF003025FEADC0C18BF03325FEA5B
:10C59000DC0C18BF033202EBDC02C2F1200300FA0C
:10C5A00003FC20FA02F001FA03FE40EA0E0021FA31
:10C5B00002F11444BDE600BF53B94AB9002908BFCF
:10C5C00000281CBF4FF0FF314FF0FF3000F06CB976
:10C5D000ADF1080C6DE904CE00F006F8DDF804E0DA
:10C5E000DDE9022304B070472DE9F047089D0446B9
:10C5F0008846002B7DD18A4217463FD9B2FA82F293
:10C6000042B1C2F120009140974024FA00F09440DA
:10C6100040EA01084FEA174C230C1FFA87FEB8FBCB
:10C62000FCF60CFB168106FB0EF043EA0143984230
:10C6300005D9FB1802D2984200F22481013E191A52
:10C64000A3B2B1FBFCF00CFB101100FB0EFE43EAA1
:10C650000144A64505D93C1902D2A64500F20F8136
:10C66000013840EA0640A4EB0E0400261DB1D44078
:10C670000023C5E900433146BDE8F08702B9FFDE7B
:10C68000B2FA82F2002A50D1CB1B4FEA174E1FFAA2
:10C6900087F80126210CB3FBFEFC0EFB1C300B4679
:10C6A00008FB0CF941EA004189450AD979182CBFE9
:10C6B00001230023894502D9002B00F0D9800CF119
:10C6C000FF3CA1EB0901A3B2B1FBFEF00EFB101180
:10C6D00008FB00F843EA0144A04505D93C1902D201
:10C6E000A04500F2C9800138A4EB080440EA0C40E0
:10C6F000BCE78B4209D9002D00F0B1800026C5E9C6
:10C70000000130463146BDE8F087B3FA83F6002ECB
:10C7100046D18B42C0F0A680824240F2A3803046D0
:10C72000002DA8D0C5E90048A5E79740C2F1200335
:10C7300001FA02F04FEA174ED94024FA03F31FFA28
:10C7400087F894400343B1FBFEF01E0C0EFB101162
:10C7500000FB08FC46EA01418C4509D979182CBF39
:10C76000012600268C4502D9002E00F09380013866
:10C77000A1EB0C019BB2B1FBFEF60EFB161106FB02
:10C7800008FC43EA01418C4505D9791802D28C4551
:10C7900000F28780013EA1EB0C0346EA004679E7F0
:10C7A000C6F1200703FA06F402FA06FC01FA06FEB7
:10C7B000FA4020FA07F8F94000FA06F3224348EA63
:10C7C0000E044FEA12484FEA144E1FFA82F9B1FBE9
:10C7D000F8FA08FB1A110AFB09F04EEA014E7045FF
:10C7E0000AD912EB0E0E2CBF01210021704501D990
:10C7F000002952D00AF1FF3AAEEB000EA4B2BEFB04
:10C80000F8F008FB10EE00FB09F944EA0E4EF14582
:10C8100005D912EB0E0E01D2F14538D8013840EAA5
:10C820000A40AEEB090EA0FB0C89CE4541464C46B2
:10C8300002D306D1434504D20138B8EB0C0169EBB1
:10C84000020415B35A1A6EEB040EF2400EFA07F703
:10C850002EFA06F300261743C5E900730BE72E46B0
:10C86000284608E7841A61EB03010120884657E750
:10C87000ACF1020C394424E702383C4434E7023876
:10C880003C44EEE6023E3B44D9E62E46F3E602384F
:10C890009644C4E7023839446AE7AAF1020A96448A
:10C8A000AAE7023E394476E7704700BF70B54FF003
:10C8B000FF0C4CF4E06C1CEA11541DBF1CEA13552C
:10C8C00094EA0C0F95EA0C0F00F0DEF82C4481EA94
:10C8D000030621EA4C5123EA4C5350EA013518BFB4
:10C8E00052EA033541F4801143F4801338D0A0FBA1
:10C8F00002CE4FF00005E1FB02E506F00042E0FB4E
:10C9000003E54FF00006E1FB03569CF0000F18BF53
:10C910004EF0010EA4F1FF04B6F5007F64F54074FB
:10C9200004D25FEA4E0E6D4146EB060642EAC6218E
:10C9300041EA55514FEAC52040EA5E504FEACE2EFB
:10C94000B4F1FD0C88BFBCF5E06F1ED8BEF1004FFE
:10C9500008BF5FEA500E50F1000041EB045170BD7A
:10C9600006F0004646EA010140EA020081EA0301BE
:10C97000B4EB5C04C2BFD4EB0C0541EA045170BDBA
:10C9800041F480114FF0000E013C00F3AB8014F134
:10C99000360FDEBF002001F0004170BDC4F100047D
:10C9A000203C35DA0C341BDC04F11404C4F12005FE
:10C9B00000FA05F320FA04F001FA05F240EA020059
:10C9C00001F0004221F0004110EBD37021FA04F68F
:10C9D00042EB06015EEA430E08BF20EAD37070BD49
:10C9E000C4F10C04C4F1200500FA04F320FA05F0A8
:10C9F00001FA04F240EA020001F0004110EBD370AA
:10CA000041F100015EEA430E08BF20EAD37070BD19
:10CA1000C4F1200500FA05F24EEA020E20FA04F3F2
:10CA200001FA05F243EA020321FA04F001F00041A1
:10CA300021FA04F220EA020000EBD3705EEA430E12
:10CA400008BF20EAD37070BD94F0000F0FD101F041
:10CA50000046400041EB010111F4801F08BF013C7A
:10CA6000F7D041EA060195F0000F18BF704703F0B8
:10CA70000046520043EB030313F4801F08BF013D3F
:10CA8000F7D043EA0603704794EA0C0F0CEA1355FB
:10CA900018BF95EA0C0F0CD050EA410618BF52EAB5
:10CAA0004306D1D181EA030101F000414FF00000BB
:10CAB00070BD50EA410606BF1046194652EA4306C9
:10CAC00019D094EA0C0F02D150EA013613D195EA3D
:10CAD0000C0F05D152EA03361CBF104619460AD185
:10CAE00081EA030101F0004141F0FE4141F470018F
:10CAF0004FF0000070BD41F0FE4141F4780170BD7F
:10CB000070B54FF0FF0C4CF4E06C1CEA11541DBFE3
:10CB10001CEA135594EA0C0F95EA0C0F00F0A7F8E5
:10CB2000A4EB050481EA030E52EA03354FEA013112
:10CB300000F088804FEA03334FF0805545EA131325
:10CB400043EA12634FEA022245EA111545EA1065ED
:10CB50004FEA00260EF000419D4208BF964244F184
:10CB6000FD0404F5407402D25B084FEA3202B61AA3
:10CB700065EB03055B084FEA32024FF480104FF477
:10CB8000002CB6EB020E75EB030E22BFB61A7546EB
:10CB900040EA0C005B084FEA3202B6EB020E75EB7E
:10CBA000030E22BFB61A754640EA5C005B084FEAE6
:10CBB0003202B6EB020E75EB030E22BFB61A7546B3
:10CBC00040EA9C005B084FEA3202B6EB020E75EBBE
:10CBD000030E22BFB61A754640EADC0055EA060E7F
:10CBE00018D04FEA051545EA16754FEA06164FEAC2
:10CBF000C30343EA52734FEAC2025FEA1C1CC0D16E
:10CC000011F4801F0BD141EA00014FF000004FF0FA
:10CC1000004CB6E711F4801F04BF01430020B4F1BB
:10CC2000FD0C88BFBCF5E06F3FF6AFAEB5EB030C73
:10CC300004BFB6EB020C5FEA500C50F1000041EB70
:10CC4000045170BD0EF0004E4EEA113114EB5C043D
:10CC5000C2BFD4EB0C0541EA045170BD41F4801110
:10CC60004FF0000E013C90E645EA060E8DE60CEA18
:10CC7000135594EA0C0F08BF95EA0C0F3FF43BAF35
:10CC800094EA0C0F0AD150EA01347FF434AF95EAEC
:10CC90000C0F7FF425AF104619462CE795EA0C0FD0
:10CCA00006D152EA03353FF4FDAE1046194622E79D
:10CCB00050EA410618BF52EA43067FF4C5AE50EA77
:10CCC00041047FF40DAF52EA43057FF4EBAE12E767
:10CCD0004FF0FF3C06E000BF4FF0010C02E000BF48
:10CCE0004FF0010C4DF804CD4FEA410C7FEA6C5C2B
:10CCF0004FEA430C18BF7FEA6C5C1BD001B050EACE
:10CD0000410C0CBF52EA430C91EA030F02BF90EAB8
:10CD1000020F0020704710F1000F91EA030F58BF77
:10CD2000994208BF90422CBFD8176FEAE37040F0D9
:10CD3000010070474FEA410C7FEA6C5C02D150EA77
:10CD4000013C07D14FEA430C7FEA6C5CD6D152EA32
:10CD5000033CD3D05DF8040B704700BF84461046F7
:10CD600062468C461946634600E000BF01B5FFF7F6
:10CD7000B7FF002848BF10F1000F01BD4DF808EDC6
:10CD8000FFF7F4FF0CBF012000205DF808FB00BF97
:10CD90004DF808EDFFF7EAFF34BF012000205DF8F1
:10CDA00008FB00BF4DF808EDFFF7E0FF94BF01203E
:10CDB00000205DF808FB00BF4DF808EDFFF7CEFF3F
:10CDC00094BF012000205DF808FB00BF4DF808ED7E
:10CDD000FFF7C4FF34BF012000205DF808FB00BF4F
:10CDE0004FEA410C7FEA6C5C02D150EA013C0AD167
:10CDF0004FEA430C7FEA6C5C02D152EA033C02D159
:10CE00004FF0000070474FF0010070474FEA4102B9
:10CE100012F5001215D211D56FF47873B3EB62528C
:10CE200012D94FEAC12343F0004343EA505311F0B3
:10CE3000004F23FA02F018BF404270474FF0000045
:10CE4000704750EA013005D111F0004008BF6FF083
:10CE5000004070474FF00000704700BF10F8012BF2
:10CE600011F8013B012A28BF9A42F7D0D01A704727
:10CE7000034613F8012B002AFBD1181A013870471A
:10CE80002DE9F04F456A04462DED028B95B057EC25
:10CE9000106BDDF88080059109920F93CDE9026750
:10CEA0003DB9102014F022FF60620560C560C0E942
:10CEB0000155636A196851B15A68012320469340AD
:10CEC0004A608B6019F07FF9636A00221A603B1E8A
:10CED000B7BF23F00043002301220393A8BFC8F883
:10CEE0000030DDF80C90B64BB8BFC8F8002033EA2C
:10CEF00009031BD142F20F730F9A1360C9F3130396
:10CF0000334300F07285219B63B9AE4B25E0AE4BF5
:10CF100000930833219A1360009815B0BDEC028B82
:10CF2000BDE8F08FA74B00930333F3E79DED027B41
:10CF30000022002351EC170B8DED0A7BFFF71EFF3B
:10CF4000804660B101230F9A1360219B002B00F0F3
:10CF500049859E4B219A1360013B0093DCE7C9F39E
:10CF60000A5512AA13A920469DED0A0B19F06DFB74
:10CF70008246002D7CD00B9BA5F2FF35CDF840807A
:10CF8000C3F31303DDE90A6743F07F5747F4401703
:10CF900000228F4B30463946FFF756F982A3D3E97A
:10CFA0000023FFF783FC82A3D3E90023FFF74EF9A8
:10CFB00006460F462846FFF795FA7FA3D3E90023DC
:10CFC000FFF774FC02460B4630463946FFF73EF940
:10CFD00006460F46FFF71AFF00228146002330461F
:10CFE0003946FFF7D5FE48B14846FFF77BFA32468F
:10CFF0003B46FFF7C3FE08B909F1FF39B9F1160F37
:10D0000055D8744B03EBC903DDE90A01D3E90023CA
:10D01000FFF7BEFE00284CD009F1FF3900230E9324
:10D02000129B5D1B6B1E049345BF0023C5F10108D5
:10D030004FF000080493B9F1000F3CDB049BCDF8DE
:10D0400034904B44049300230693059B092B00F274
:10D050009980052BC5BF043B002501250593059B41
:10D06000023B032B00F29A80DFE803F02D7E7C8ADE
:10D07000DDE912531D4405F23243202BC6BFC3F134
:10D08000400305F21240C3F1200305F1FF35C5BF8F
:10D0900009FA03F326FA00F006FA03F01843FFF743
:10D0A00011FA01230646A1F1F877109370E70123E6
:10D0B000B5E70E90B4E7C9F10003A8EB09080693A1
:10D0C00000230D93C1E700230893099B002B00F375
:10D0D00085804FF0010B5B46CDF804B0CDF824B04D
:10D0E0000022666A7260042202F11400716898429C
:10D0F0007AD9204619F033F8636A30601B680093D0
:10D10000019B0E2B00F2F580002D00F0F280B9F1AA
:10D11000000F7DDD09F00F032E4A19F4807F4FEADE
:10D12000291702EBC30393ED007BB0EE478AF0EEC4
:10D13000678A5DD0284B07F00F070325D3E9082342
:10D14000DDE90A01FFF7DCFCCDE90201224E002FE8
:10D1500050D1DDE9020153EC182BFFF7D1FCCDE9EA
:10D1600002016FE00123AFE700230893099B09EB5D
:10D17000030B0BF10103012B0193B8BF0123AFE7B0
:10D180000123F2E701250023089505934FF0FF3BAB
:10D1900000221223CDF804B00992A1E701230893DD
:10D1A000F4E700BFAFF3008061436F63A787D23F0E
:10D1B000B3C8608B288AC63FFB799F501344D33F86
:10D1C0000000F07FE9980200E0980200467D02002E
:10D1D0000000F83F606D0200386D0200DDF824B0F9
:10D1E0005B46CDF804B07BE70131520071607BE70C
:10D1F0000225ABE7F90708D5013551EC180BD6E944
:10D200000023FFF753FB41EC180B7F1008369EE715
:10D2100000F0AB80C9F10006AA4BAB4F022506F027
:10D220000F02361103EBC203DDE90A01D3E9002343
:10D23000FFF73CFB0023CDE90201002E40F08A807D
:10D24000002B8CD10E9B002B00F0918000229F4B75
:10D25000DDE9026730463946FFF79AFD002800F005
:10D260008680019B002B00F08280BBF1000F3CDD2B
:10D2700009F1FF3301350022304607933946944BBC
:10D28000FFF714FBCDF830B0CDE90201DDE902670C
:10D290002846FFF727F932463B46FFF707FB8D4B41
:10D2A0000022FEF7D3FFA1F15073CDE902010393F1
:10D2B0000C9B002B60D10022874B30463946FEF78D
:10D2C000C3FF06460F46DDE90223FFF77FFD002876
:10D2D00040F097823046DDE9022101F100433946F2
:10D2E000FFF756FD002840F08982DDE90A23CDE9E9
:10D2F0000223139B002BC0F25B81B9F10E0F00F3E8
:10D300005781704B03EBC90393ED007B099B002B06
:10D31000B0EE478AF0EE678A80F2E280019B002B34
:10D3200000F3DE8040F06A8200226B4B51EC170B59
:10D33000FFF7BCFADDE90223FFF73EFD019E374609
:10D34000002840F04082009D312309F1010905F8D1
:10D35000013B3CE2F20705D50135D7E90023FFF791
:10D36000A5FA01237610083767E702256AE7019BD3
:10D37000CDF81C900C9389E700990C980C9A014405
:10D38000504B9DED027B03EBC20302910899B0EE76
:10D39000478AF0EE678A53E90223002945D000202E
:10D3A0004E49FFF7ADFB53EC182BFEF74DFF009DE8
:10D3B00041EC180B39463046FFF728FD0C90FFF77B
:10D3C00091F802460B4630463946FEF73DFF0C9B6E
:10D3D00006460F46303305F8013B53EC182BFFF798
:10D3E000D7FC002864D132463B4600203749FEF77F
:10D3F0002BFF53EC182BFFF7CBFC002840F0B88034
:10D40000029B9D423FF471AF0022314B51EC180B4F
:10D41000FFF74CFA00222E4B41EC180B30463946F0
:10D42000FFF744FA06460F46C4E751EC170BFFF727
:10D430003DFA029B009D0C9341EC180B3946304697
:10D44000FFF7E4FC1190FFF74DF802460B4630461B
:10D450003946FEF7F9FE119B06460F46303300228F
:10D4600005F8013B029B9D4225D11C4B51EC180B4A
:10D47000FEF7ECFE02460B4630463946FFF7A6FCA7
:10D48000002875D10020154953EC182BFEF7DCFE5F
:10D4900002460B4630463946FFF77AFC00283FF437
:10D4A00024AF0C9D6B1E0C9315F8013C302BF8D06B
:10D4B000DDF81C904AE0064BFFF7F8F906460F46E8
:10D4C000BCE700BF606D0200386D02000000F03F55
:10D4D0000000244000001C40000014400000E03F19
:10D4E000DDE90267009D3046394653EC182BFFF703
:10D4F00007FBFFF78BFC8046FEF7F4FF53EC182B7D
:10D50000FFF7D4F90246304608F130060B4639469B
:10D51000FEF79AFE05F8016B009E0246019F0B463E
:10D52000AE1BB74237D1FEF791FE06460F4653ECCD
:10D53000182BFFF74BFCC8B93046394653EC182B73
:10D54000FFF71CFC10B118F0010F0FD12046514617
:10D5500018F039FE002309F101002B700F9B1860B1
:10D56000219B002B3FF4D8AC1D60D5E4CDF81C9076
:10D570002B461D4613F8012D392A08D1009A9A42EC
:10D58000F7D1079A00990132079230220A701A786F
:10D5900001321A708CE700229C4BFFF787F90022BA
:10D5A000002306460F46FFF7E9FB00289BD0CDE796
:10D5B000089A002A00F0C480059A012A00F3A98085
:10D5C000109A002A00F0A18003F23343069E4546DC
:10D5D000049A0121204698441A44049218F099FEB6
:10D5E0000746002D0BDD049B002B08DDAB42049A9F
:10D5F000A8BF2B46A8EB0308ED1AD31A0493069B89
:10D60000FBB1089B002B00F09F80002E11DD3946F6
:10D610003246204614F072FB524601460746204629
:10D6200018F080FE51460790204618F0CCFD079B6D
:10D630009A46069B9A1B04D05146204614F05EFB86
:10D6400082460121204618F064FE0D9B0646002B01
:10D650007CDD1A460146204614F050FB059B064629
:10D66000012B76DD00230693336906EB83031869EB
:10D6700018F0FFFDC0F12000049B184410F01F00BB
:10D6800000F08680C0F12003042B7FDDC0F11C0078
:10D69000049B8044054403440493B8F1000F05DD66
:10D6A00051464246204618F0D8FE8246049B002B85
:10D6B00005DD31461A46204618F0CFFE06460E9B81
:10D6C000002B67D03146504618F026FF002861DA5B
:10D6D000002351460A22204618F08CFD089B09F1D0
:10D6E000FF398246002B00F08781394600230A2249
:10D6F000204618F07FFDBBF1000F074600F38E8037
:10D70000059B022B40F38A804CE0129BC3F1360349
:10D710005CE7019B5E1E069BB342B7BF069B9E1B48
:10D720000696F21ABFBF0D9B00269B180D93019B16
:10D73000002BB5BFA8EB030545460023019B47E737
:10D74000069E4546089F4CE7069A75E7059B012B08
:10D7500018DC029BB3B9039BC3F31303A3B9039B68
:10D7600023F000431B0D1B052BB1049B08F101089E
:10D7700001330493012306930D9B002B7FF474AFB8
:10D78000012079E70023F6E7029BF4E785D01846ED
:10D790001C307DE7019B002B3ADC059B022B37DD1B
:10D7A000DDF804B0BBF1000F0DD131465B46052218
:10D7B000204618F01FFD01460646504618F0ACFE04
:10D7C00000283FF7C0AD099B009D6FEA03094FF0A9
:10D7D00000083146204618F0F6FC002F3FF4B6AEA4
:10D7E000B8F1000F05D0B84503D04146204618F0E7
:10D7F000EAFC3946204618F0E6FCA7E60026374644
:10D80000E1E70C9EDDF81C9037469CE500002440C3
:10D81000089BDDF804B0002B00F0F580002D05DD3D
:10D8200039462A46204618F018FE0746069B002B6C
:10D8300055D07968204618F092FC3A69054607F100
:10D840000C0102320C30920018F04CF901222946EA
:10D85000204618F002FE009BB846074601330193AC
:10D86000009B5B440793029B03F001030693019B1B
:10D870003146504603F1FF3B18F06CFB034641462E
:10D88000029050463033089318F046FE3A46049012
:10D890003146204618F05CFEC2680546089B02BB74
:10D8A0000146504618F038FE089B0246294620469D
:10D8B000CDE9083218F087FC059B099A019D43EADF
:10D8C0000201069B0B43089B0DD1392B27D0049AEC
:10D8D000002A01DD029B31338BF8003079E73846AE
:10D8E000B9E70122E2E70499002904DB0598014326
:10D8F0000698014320D1002AEEDD51460122204640
:10D90000019318F0AAFD3146824618F005FE002862
:10D91000019B02DCE0D1DA07DED5392BDAD13923DD
:10D920008BF800302B461D46013B15F8012C392A97
:10D9300050D001321A704CE7002A03DD392BEED0AB
:10D940000133C9E7019A079902F8013C8A422AD0BB
:10D95000514600230A22204618F04CFCB845824666
:10D960004FF000034FF00A024146204607D118F05D
:10D9700041FC80460746019B0133019377E718F08D
:10D9800039FC3946804600230A22204618F032FC32
:10D990000746F0E7BBF1000F009A4FF00008CCBF3C
:10D9A0005D4601251544514601222046019318F099
:10D9B00054FD3146824618F0AFFD0028B2DC02D19A
:10D9C000019BDB07AED42B461D4613F8012D302AF0
:10D9D000FAD0FEE6009A9A42A5D1312309F1010955
:10D9E0001370F6E6124BFFF7B8BA219B002B7FF4B9
:10D9F0008EAA104BFFF7B1BABBF1000F03DC059BF9
:10DA0000022B3FF7CFAE009D3146504618F0A2FAE8
:10DA1000009A00F1300305F8013BAA1A9345B9DDDD
:10DA2000514600230A22204618F0E4FB8246EBE729
:10DA3000457D0200E09802000749D1E8EF3F43F03E
:10DA40000102C1E8E02F0028F7D1DB0703D4034827
:10DA5000083917F027BD7047E0130220F4130220A5
:10DA600038B5144B144C154DE41AE408A4011448BD
:10DA700044F0030114F0BDFF28684FF4005114F086
:10DA8000D3FB28688368DB6913B100220D499847EE
:10DA90004FF48071286814F0DBFB00F0A1FA014616
:10DAA00030B144F001020848BDE8384014F0B0BF7E
:10DAB00038BD00BF006C0200006C0200F0130220B1
:10DAC0004C760200E413022056760200054A064B0B
:10DAD0000146D21AD2089201044842F0010214F021
:10DAE00097BF00BF006C0200006C0200717602005C
:10DAF00010B5274811F07AFD264C206058B9BDE8D2
:10DB000010402549254B2648C91AC908890141F00A
:10DB1000010114F06EBF4FF4887114F099FB0146B7
:10DB200058B11D4A1D4B1F48D21AD208920142F02B
:10DB30000102BDE8104014F06BBF1B491B4B20686D
:10DB40004B6040238B608368DB6963B10122984797
:10DB5000014658B1104A114B1548D21AD208920109
:10DB600042F00102E5E76FF08501F3E720684FF42A
:10DB7000103114F059FB014640B1074A074B0D48DC
:10DB8000D21AD208920142F00102D2E710BD00BFC2
:10DB90008E760200F0130220006C0200006C02007E
:10DBA00095760200A7760200E413022039DA00001D
:10DBB000BF760200DD76020038B51C4B1C4C1D48B8
:10DBC000E41AE408A40144F0030114F012FF08F081
:10DBD000F5FB014630B1184844F00102BDE8384079
:10DBE00014F016BF154808F02DFC0821144817F052
:10DBF000E1F9014618B1134844F00102EEE700F0E4
:10DC0000EFF9054620B1014644F001020E48E5E770
:10DC10000E234FF400620D490D4812F05DFD0D4BCF
:10DC20000D4A1D60C3E9012538BD00BF006C02002C
:10DC3000006C0200FE7602000F77020080080220CE
:10DC4000D01302203777020056760200C09C0220D3
:10DC5000F4130220D813022061DA0000F8B505465B
:10DC600008460E46FFF704F904462846FFF700F978
:10DC7000844217D100230C4FA34201DB0120F8BDE1
:10DC8000E95CCA5D02F00302022AF25C08BF203997
:10DC9000B85C00F00300022808BF203A914201D18D
:10DCA0000133E9E70020EAE773970200F8B506467A
:10DCB00008460F46FFF7DCF804463046FFF7D8F871
:10DCC000844223D800251348A5420DDB3046FFF7D8
:10DCD000CFF80234A0421BD9705D00F0FD00A0F126
:10DCE0003D0358425841F8BD725D135C03F00303D5
:10DCF000022B7B5D08BF203AC15C01F003010229C1
:10DD000008BF203B9A4201D10135DDE70020EAE758
:10DD10000120E8E7739702002DE9F8430D4690468D
:10DD20000746A8B1A2B1B3EB410F4FEA41060FDBA2
:10DD30000024DFF82490A54202DC3046BDE8F883D9
:10DD40003A5D08EB4400494613F0D4FB0134F2E796
:10DD50006FF01506F1E700BF5877020070B5037841
:10DD6000062B62D8DFE803F0040D209F6161BB0041
:10DD7000604B186817F0FBFABDE870405E4812F07F
:10DD800075BB5C4B186817F0F2FA5B4812F06EFB3B
:10DD9000BDE8704059495A4B5A48C91AC908890107
:10DDA00041F0030114F025BE574D43682A681B78E3
:10DDB000541C222B2C6023D07F2B01D0082B24D184
:10DDC00002B1013A022C38BF022400204F49023C24
:10DDD00088542C604E49097839BB4E49097802298C
:10DDE00052D034D9032957D0444A454B4A48D21A15
:10DDF000D208920142F00102BDE8704014F008BE62
:10DE00004348017881F00101017040F68C26B4424C
:10DE10000CD93B49394A4148521AD2089201194655
:10DE200042F0010214F0F4FD2E6070BD64B9344B71
:10DE3000324A2146D21AD2089201394842F00102F0
:10DE400014F0E6FD2C60F0E730498B54C2E7354A08
:10DE5000525C9A42E9D1344B186814F05CFA3349A9
:10DE6000D1E8EF3F43F00102C1E8E02F0028F7D1ED
:10DE7000DB0703D42E48083917F014FB2A682D4B12
:10DE80001A6000232B60D0E720490A4412F8012CC5
:10DE9000002ACAD00A2BDDE71C490A4412F8012CDB
:10DEA0000D2AC2D1F6E7204B234C186821788368ED
:10DEB000224D012229441B699847014648B10F4A67
:10DEC0000F4B1F48D21AD208920142F0020214F0FE
:10DED0009FFD2378013303F007032370A5E7074A6A
:10DEE000074B0179D21AD2089201164842F0020279
:10DEF00082E700BFDC14022008070220106C020039
:10DF0000006C02005D770200C814022066780220CF
:10DF10007F8D0220808D0220A677020068770200A4
:10DF200088770200067B0200D8140220D414022055
:10DF3000BC6C0220C41402207E8D0220818D022040
:10DF4000C3770200D7770200F8B507460D464FF0B9
:10DF5000FF324FF0FF331B4812F0AEFA284611F0A3
:10DF600057FD194E0446306070B91849184B1948CE
:10DF7000C91AC908890141F0020114F03AFDBDE84F
:10DF8000F840104812F072BA2A46394617F0AAFD36
:10DF9000114B1868836821465F682A464FF0FF33AB
:10DFA000B847014668B10A4B084A0C48D21AD20851
:10DFB000920142F0020214F02BFD306817F0D7F9FD
:10DFC000DDE7F8BD08070220DC140220106C020017
:10DFD000006C0200E7770200D8140220F5770200F7
:10DFE0002DE9FF480322704B1A70704811F0FEFAB9
:10DFF0006F4C206080B96F4B6F4A6C49D21AD208BF
:10E0000092016E4842F0010214F002FD6FF0150417
:10E01000204604B0BDE8F08817F0E2FB4FF47A76B2
:10E020000B46A0FB060106FB0311C70B47EA41475D
:10E03000206883681B6A002B00F09D809847054686
:10E04000002800F0988017F0CBFBA0FB06BC06FB75
:10E0500001CC4FEADB3242EA4C42D21BB2F5FA7FE6
:10E06000E6D9544B544A2946D21AD2089201544850
:10E0700042F0010214F0CCFC6FF00404C8E7012563
:10E080002068009329460669039503AAB0474D4BC3
:10E0900020681D7083684C49DC682A464FF0FF33C6
:10E0A000A047014638B1444A424B4848D21AD208E8
:10E0B00092012A4372E0464907F060FD044658B1D8
:10E0C0003C4B3D4A0146D21AD2089201414842F0E7
:10E0D000010214F09DFC9BE701F02EFD014640B1CA
:10E0E000354A344B3C48D21AD208920142F0010220
:10E0F00054E002F051F8014640B12F4A2D4B374809
:10E10000D21AD208920142F0010247E002F05AFB13
:10E11000014640B1284A274B3148D21AD208920111
:10E1200042F001023AE014F039F9014640B1224AC6
:10E13000204B2C48D21AD208920142F001022DE065
:10E1400003F0E4FA044648B11B4A1A4B0146D21ABE
:10E15000D2089201244842F001021FE0234B244AD6
:10E160001860C3E90120234812F080F907212248F2
:10E17000FFF7EAFE4CE72068002283681F491B680E
:10E180009847034600283FF47AAF0A490A4A1C48D8
:10E19000521A1946D208920142F0010214F038FCDA
:10E1A0006FF00D0434E700BF808D02200878020074
:10E1B000D8140220006C0200106C02000F780200DC
:10E1C0001F7802007E8D0220818D02206D78020072
:10E1D0001D23020082780200A0780200C3780200AA
:10E1E000E57802000679020028790200CC140220AA
:10E1F00021E3000008070220497902005DDD0000EC
:10E20000557802001FB514F096F8014648B1394A16
:10E21000394B3A48D21AD208920142F0020214F065
:10E22000F7FB14F0B9F8014648B1324A324B344892
:10E23000D21AD208920142F0020214F0E9FB02F075
:10E24000CFFA014648B12B4A2B4B2E48D21AD2089E
:10E25000920142F0020214F0DBFB02F0DBFD01460A
:10E2600048B1244A244B2848D21AD208920142F0DD
:10E27000020214F0CDFB14F0C1F8014648B11D4A6A
:10E280001D4B2248D21AD208920142F0020214F029
:10E29000BFFB1F49002007F0BBFC014648B1154AEF
:10E2A000154B1C48D21AD208920142F0020214F017
:10E2B000AFFB194C206814F02EF8002140F6CD4039
:10E2C00012F0AEF805230393002320680093012188
:10E2D000046903AAA047014648B1064A064B0F4805
:10E2E000D21AD208920142F0020214F091FB04B05B
:10E2F00010BD00BF106C0200006C020051790200DA
:10E30000767902009A790200BD790200E179020073
:10E310001D230200047A0200D8140220217A020090
:10E3200040F68B22924B70B51B68924C934228BFEB
:10E330001346002294B020468F49E254FFF7B6FC02
:10E3400020B10F218D48FFF7FFFD28E020468C49C2
:10E35000FFF7ACFC0546002847D00A218648FFF7A6
:10E36000F3FD02218748FFF7EFFD09218648FFF7FB
:10E37000EBFD02218348FFF7E7FD08218048FFF706
:10E38000E3FD02217F48FFF7DFFD01F0B3FB01F061
:10E39000E7FE02F0FBF902F01BFD03F09BF90421FC
:10E3A0007A48FFF7D1FD002140F6CD4012F038F851
:10E3B0000122774B1A70774B186883687649DC68BE
:10E3C0004FF0FF33A047014600284FD0734B744AEB
:10E3D0007448D21AD208920142F0010214F018FBDC
:10E3E0000D217148FFF7B0FD40E020466649FFF778
:10E3F0005DFC002858D0294620466C4A16F089FD5D
:10E40000061E0DDA664A654B3146D21AD2089201D1
:10E41000674842F0010214F0FBFA07216548C0E7A3
:10E42000204616F079FD0128044628D15F48ADF852
:10E43000105016F0B6FE012811D921465B4804AAF7
:10E4400016F067FE00280ADA544B55495A48C91A93
:10E45000C908890141F0010114F0CBFADDE7BDF8EC
:10E4600010302BB9FFF7CEFEFFF742FB14B070BDA2
:10E47000012BE9D1FFF7C6FE13F0F7FE8FE7032863
:10E480000ED1012329464022CDE9005304A84B4B6D
:10E4900017F07FFC04A8FEF7EBFC014604A852E746
:10E4A000002E3FF47CAFB8E7204601F0E7FA0028E1
:10E4B0003FF475AF8630B0D1204601F023FE00282E
:10E4C0003FF471AF8630A8D1204601F0BDFF00288F
:10E4D0003FF465AF8630A0D1204602F03DFC002815
:10E4E0003FF45DAF863098D1224803F097F80028BA
:10E4F0003FF455AF863090D1314940F68C221D480B
:10E500000DF10F0307F07CFA011E0DDA234B244AAC
:10E510002C48D21AD208920142F0010214F078FA83
:10E5200001238DF80F3078E79DF80F30032B3FF66D
:10E530003AAF01A252F823F049E500001BE40000C5
:10E5400055E5000069E500001D48FEF791FC014615
:10E550001B48F8E61C4B00910021182204A817F074
:10E5600018FC411C04A81CE7184B0091F4E700BFFD
:10E57000C4140220667802203A7A0200457A02002A
:10E580005A7A020059850200637A0200557A020025
:10E590007E8D0220D8140220818D0220006C0200A2
:10E5A000106C0200DD7A0200F07A0200D013022023
:10E5B0006D7A0200F67A02008B7A02009E7A0200DF
:10E5C000F2820220B27A0200C77A0200D27A0200F6
:10E5D000802370B5BCB005465022002108A80293E4
:10E5E00017F08DFA01239D420A9304D06FF01504B1
:10E5F00020463CB070BD404816F0D3FD0128F5D947
:10E6000029463D4802AB1CAA16F0A8FD0446002886
:10E61000EED1029B3CAA134403F8800C1CA8FEF721
:10E6200027FCC1B21CA813F067FE064650B1334B5D
:10E6300033493448C91AC908890141F0010114F06D
:10E64000D8F9D3E7214603AB08AA1CA814F01CFD97
:10E650000446D8B1294B2A4A0146D21AD20892015F
:10E66000294842F0010214F0D3F96342314640F6E2
:10E670008C2200932548264B17F08BFB2348FEF78E
:10E68000F7FB01462148FFF75FFCB1E7039BBBB9ED
:10E690001A4B1B491F48C91AC908890141F00101D9
:10E6A00014F0A7F91C49194817F09AFB1748FEF710
:10E6B000DFFB01461548FFF747FC6FF0010497E7C1
:10E6C0009969043104AE32461023284605F02AFB2E
:10E6D00040F68C222146114B00960C4817F059FB4E
:10E6E0000A48FEF7C5FB01460848FFF72DFC0398D2
:10E6F00014F0CCFC7CE700BFD0130220006C0200B9
:10E70000A86C0200097B02001E7B0200DA6D022069
:10E71000367B02009D7B02004A7B0200657B020083
:10E7200008B50123074A49BA1380518001460432D3
:10E73000184614F05BFD012814BF6FF0150000208F
:10E7400008BD00BFF4140220F0B5044617460126A8
:10E750009BB050220D4606A8002117F0D0F92046A4
:10E76000002101AB06AACDE9086714F08DFC044630
:10E7700060B1164A164B0146D21AD20892011548CA
:10E78000324314F045F920461BB0F0BD019B63B93C
:10E790000F4B0E491048C91AC908890141F00101FF
:10E7A00014F027F96FF00104EDE79B690B495B68F2
:10E7B0006DBA4B600E804D801023304602AA0431A2
:10E7C00005F0B0FA019814F061FCDCE7A86C0200D7
:10E7D000006C0200797B0200967B0200F414022098
:10E7E00038B504460D46FEF743FBC1B2204613F090
:10E7F00083FD90B129462046FFF792FF044650B1B1
:10E80000094A0A4B0146D21AD2089201084842F03E
:10E81000010214F0FDF8204638BD022229462046A8
:10E82000FFF792FFEAE700BFA86C0200006C02004D
:10E83000B07B020030B50128044687B005D003281C
:10E8400000F0A7806FF0150469E0584B1A681D4668
:10E85000002A0ADA5649574B5748C91AC90889018C
:10E8600041F0010114F0C5F8ECE75B6843B1504991
:10E87000504B5248C91AC908890141F00101F1E71A
:10E880004F4816F08EFC0228DCD921464C4802AADB
:10E8900016F03FFC0446002841D1022148480DF102
:10E8A0000A0216F036FC0446002838D1BDF80830BC
:10E8B000012B37D1424816F074FC0328C2D902213B
:10E8C0003F4803AA16F037FC044640BBBDF80A20B7
:10E8D000042A03D0142A06D0022A58D139493A48CA
:10E8E00017F07EFA4BE000230593039B28680493FE
:10E8F00008230121009304AB14F096FC041E0EDAE9
:10E900002C4A2B4DAD1AED0814F09BFDAD0145F0DE
:10E9100001052A4601682D48494214F079F820463D
:10E9200007B030BD002BFAD1BDF80A30042BD5D08A
:10E93000142B01D0022BD0E708232868039303ABE4
:10E9400000931422012104AB14F057FC044668B173
:10E95000184A174DAD1A14F074FDED080168AD01A9
:10E9600045F001052A461A484942D6E7049B01466C
:10E97000009340F68C22174B134817F00AFA1248FE
:10E98000FEF776FA01461048FFF7DEFAC7E71249AC
:10E99000A5E70024012340F68C22CDE9004321465F
:10E9A0000E4B094817F0F5F9E9E700BFE014022023
:10E9B000A86C0200006C0200C17B0200D77B020041
:10E9C000D0130220E47B0200DA6D0220FB7B020000
:10E9D0002F7C0200467C0200127C02005C7C02005C
:10E9E00073B51E4E05463068002835DD14F05FFB18
:10E9F000041E12DA1A4A1B4CA41A14F022FDE40871
:10EA00000168A40144F0020422461748494213F069
:10EA1000FFFF14F016FD046864424FF0FF33B06846
:10EA20003360002801DD14F042FB00214FF0FF337A
:10EA300040F68C22C6E901130C480D4B0095317449
:10EA400017F0A7F90948FEF713FA01460748FFF740
:10EA50007BFA204602B070BD0024FAE7E0140220E1
:10EA6000006C0200A86C0200857C0200DA6D0220B6
:10EA7000987C02008023F0B5ADF5397D02AF3B6193
:10EA80004FF41073FB81794B06461A681C46002A26
:10EA90000FDA7749774B7848C91AC908890141F0DC
:10EAA000010113F0A6FF6FF0150007F53777BD469B
:10EAB000F0BDDB6823F48073112B08D06C496D4BDB
:10EAC0006E48C91AC908890141F00101E9E7012826
:10EAD000E9D16B4816F065FB0228E4D907F1180567
:10EAE0002A463146664807F1100316F037FB002826
:10EAF000DBD13B690221E85407F10C02604816F0B3
:10EB000008FB0028D1D15E4816F04BFB03283BD808
:10EB10000823FA892846B9897A607B61FFF760FE8D
:10EB2000002807F114067A68BFDB2068554B019670
:10EB3000009307F19801002314F03FFB051E40DA13
:10EB40004C4A4B4CA41A14F07CFCE4080168A40164
:10EB500044F0010422464C48494213F059FF14F096
:10EB600070FC03680B2B18D014F06BFC0368742B3B
:10EB700013D014F066FC00684042FFF731FF14F038
:10EB800060FC0068404290E703213D4807F10E0217
:10EB900016F0BFFA0028BBD087E714F052FC0368D8
:10EBA00040F68C225B42002100933848384B17F026
:10EBB000F0F83648FEF75CF901463448FFF7C4F92F
:10EBC000DDE7A9B207F19800796013F05EFB044617
:10EBD000002833D06B00DA1D22F007026C46ADEB43
:10EBE000020D02AD79682A469BB207F19800FFF743
:10EBF00093F8011E17DD28467960FFF7A5F97968BB
:10EC000040F68C2201910021224B00911F4817F001
:10EC1000C0F81E48FEF72CF901461C48FFF794F98E
:10EC20000020A54641E7134B114A1B48D21AD208CF
:10EC3000920142F0010213F0EBFEF1E7294607F1E1
:10EC40009800FFF781F9012340F68C2221460093BA
:10EC50000E48104B019517F09CF80C48FEF708F988
:10EC600001460A48FFF770F920461EE7E01402202B
:10EC7000A86C0200006C0200C17B0200AF7C0200A5
:10EC8000D0130220F4140220C07C0200DA6D0220AE
:10EC9000D57C0200E47C0200FB7C0200F0B5ADF5FF
:10ECA000157D5D4B0246D3E90001012902AF13D166
:10ECB0009868431C10D1594B59495A48C91AC90878
:10ECC000890141F0010113F094FE6FF01504204614
:10ECD00007F51377BD46F0BD002307F10801CDE924
:10ECE000003314F06AFA051E37DA4C4A4C4CA41A69
:10ECF00014F0A7FBE4080168A40144F002042246D2
:10ED00004948494213F084FE14F09BFB03680B2B27
:10ED10000FD014F096FB0368742B0AD014F091FB0B
:10ED200000684042FFF75CFE14F08BFB046864420D
:10ED3000CDE714F086FB036840F68C225B4200218D
:10ED400000933A483A4B17F024F83848FEF790F809
:10ED500001463648FFF7F8F8E6E709D130492F4B6E
:10ED60003448C91AC908890141F0020113F041FE73
:10ED7000A9B207F10800796013F087FA0446002869
:10ED800033D06B00DA1D22F007026E46ADEB020DA8
:10ED900002AD2A4679689BB207F10800FEF7BCFF76
:10EDA000041E16DD21462846FFF7CEF80194002404
:10EDB00040F68C222146204B1C48009416F0E9FFB7
:10EDC0001A48FEF755F801461848FFF7BDF8B54652
:10EDD0007DE7124B124A2146D21AD20892011748F7
:10EDE00042F0010213F014FEF1E7294607F1080092
:10EDF000FFF7AAF80123214640F68C2200930195E3
:10EE00000D4B0A4816F0C5FF0848FEF731F80146D9
:10EE10000648FFF799F85AE7E0140220006C020058
:10EE2000A86C0200117D0200267D0200DA6D02202E
:10EE3000D57C0200377D0200477D0200FB7C02008A
:10EE40004FF4107313B5ADF80630134B04461B7C1A
:10EE500063B91249124B1348C91AC908890141F014
:10EE6000010113F0C6FD6FF015000AE00128FAD188
:10EE70000D4816F096F9012805D8BDF80600FFF7F1
:10EE80000DFF02B010BD214607480DF1060216F035
:10EE900040F90028F1D0F4E7E0140220A86C020049
:10EEA000006C02005A7D0200D01302202DE9F347C6
:10EEB00017461E46FFF794FC041E47DB00254FF063
:10EEC0000809DFF8D480DFF8D4A0AE422DD9D8F8F5
:10EED00000000023CDE900A9721B791914F042F952
:10EEE000041E4BDC264A274CA41A14F0AAFAE408A4
:10EEF0000168A40144F0010422462348494213F06A
:10EF000087FD14F09EFA03680B2B23D014F099FAB6
:10EF10000368742B1ED014F094FA00684042FFF787
:10EF20005FFD14F08EFA0468644240F68C220021E2
:10EF3000164B1748009516F02CFF1548FDF798FF63
:10EF400001461348FFF700F804EAE474204602B0D3
:10EF5000BDE8F08714F075FA036840F68C225B4236
:10EF6000002100930A480B4B16F013FF0848FDF7E9
:10EF70007FFF01460648FEF7E7FFD2E72544A4E7F6
:10EF8000006C0200A86C02006C7D0200807D020013
:10EF9000DA6D0220D57C0200E0140220F414022075
:10EFA000F0B5ADF5337D3C4B05461A6800AF002A3D
:10EFB0000FDA3A493A4B3B48C91AC908890141F06E
:10EFC000010113F016FD6FF0150007F53377BD460C
:10EFD000F0BDDB6823F48073112B08D02F49304B30
:10EFE0003148C91AC908890141F00101E9E701283E
:10EFF000E9D12E4816F0D5F80428E4D9802307F18A
:10F0000008047B602246294628483B1D16F0A6F8D6
:10F010000028DAD17B683A46E0540221234816F0F2
:10F0200078F80028D1D103212048BA1C16F071F8D5
:10F030000028CAD14FF4107304217B601B483B1D8C
:10F0400007F1880216F08AF80028BED17B8879681B
:10F05000D3B901EBD1735B10DA1D22F007026D46C4
:10F06000ADEB020D6A469BB289B207F1880013F03E
:10F070001FF900286E4605DD0346324620463988D2
:10F08000FFF714FFAD46A0E70B462046398807F18D
:10F090008802FFF70BFF98E7E0140220A86C02003B
:10F0A000006C0200C17B0200AF7C0200D013022082
:10F0B0003A4B2DE9F743D3E90072012A80460E4608
:10F0C00068D19F687B1C65D1354B36493648C91AD3
:10F0D000C908890141F0010113F08BFC6FF01500A4
:10F0E00003B0BDE8F08314F0ACF9036840F68C225D
:10F0F0005B42002100932D482D4B16F04AFE2B4811
:10F10000FDF7B6FE01462948FEF71EFF2CE0254418
:10F11000AE422DD900233846CDE90099721B08EB89
:10F12000050114F01FF8041EF1DA1D4A1D4CA41A43
:10F1300014F087F9E4080168A40144F001042246B0
:10F140001C48494213F064FC14F07BF903680B2B54
:10F15000C9D014F076F90368742BC4D014F071F997
:10F1600000684042FFF73CFC14F06BF9046864420D
:10F1700040F68C220021104B0C48009516F009FE39
:10F180000A48FDF775FE01460848FEF7DDFE04EA71
:10F19000E470A5E700242546A146B9E7E014022063
:10F1A000006C0200A86C0200117D0200DA6D0220E2
:10F1B000D57C02008F7D0200A17D020090B54FF446
:10F1C0001073ADF5137D00AF7B60254B04461B7CAF
:10F1D0007BB92449244B2548C91AC908890141F043
:10F1E000010113F006FC6FF0150007F51377BD461B
:10F1F00090BD0128F7D11E4815F0D3FF0228F2D99F
:10F2000021461B48BA1C15F084FF0028EDD10221CD
:10F2100017483B1D07F1080215F0A0FF0028E4D1B4
:10F220007B887968BBB901EBD1735B10DA1D22F0E2
:10F2300007026C46ADEB020D6A469BB289B207F13C
:10F24000080013F035F8002803DD01466846FFF793
:10F250002FFFA546C9E707F10800FFF729FFC4E71C
:10F26000E0140220A86C0200006C02005A7D02002B
:10F27000D0130220F0B54E4B044618681E460028F5
:10F2800089B00CDA4B494C4B4C48C91AC908890162
:10F2900041F0010113F0ADFB6FF0150046E05A6834
:10F2A000012A08D04349444B4548C91AC908890175
:10F2B00041F00101EEE7DB68062B0BD0B3F5817F4F
:10F2C00008D03C493C4B3F48C91AC908890141F064
:10F2D0000101DFE7012C07D0022CDDD1B3685A1CF5
:10F2E00060D00093384B4EE008230393374903AABC
:10F2F00013F026FF051E1BDA2F4B2E4CE41A14F0D8
:10F30000A0F8E4080168A40144F0010423462A4659
:10F3100049422F4813F093FB14F093F800684042E1
:10F32000FFF75EFB14F08DF80068404209B0F0BDB5
:10F3300004AF10233A462046264904F0F3FC78B97E
:10F340001D4A1C4CA41A14F07CF8E4080168A401BE
:10F3500044F0020422462048494213F059FB9BE73F
:10F360001E4B40F68C2200211D48009716F011FD1F
:10F370001B48FDF77DFD01461948FEF7E5FD194BD9
:10F38000B5603474009540F68C220021144816F0C4
:10F3900000FD1348FDF76CFD01461148FEF7D4FD52
:10F3A0000020C3E710490E4816F01AFDF1E700BF30
:10F3B000E0140220A86C0200006C0200C17B020075
:10F3C000D77B0200AF7C0200137E0200F4140220FF
:10F3D000AE7D0200F8140220C57D0200E67D020029
:10F3E000DA6D0220047E0200257E0200294B0146D0
:10F3F000186810B500281C460CDA2749274B284806
:10F40000C91AC908890141F0010113F0F2FA6FF03D
:10F41000150039E05A68012A08D01F491F4B2148BE
:10F42000C91AC908890141F00101EEE7DB68062B22
:10F430000BD0B3F5817F08D01749184B1A48C91A69
:10F44000C908890141F00101DFE70129DFD113F08B
:10F4500067FE002819DA114A0F4CA41A13F0F1FFC5
:10F46000E4080168A40144F00104224649420F481F
:10F4700013F0CEFA13F0E5FF00684042FFF7B0FA50
:10F4800013F0DFFF0068404210BD4FF0FF33002053
:10F49000A360F9E7E0140220A86C0200006C0200EF
:10F4A000C17B0200D77B0200AF7C0200367E0200E7
:10F4B000802370B5A2B001934A4B05461A681E46D8
:10F4C000002A0CDA4849494B4948C91AC908890138
:10F4D00041F0010113F08DFA6FF0150448E05C680B
:10F4E00044B14149414B4348C91AC908890141F017
:10F4F0000101EFE7012806D00228EDD11B7C002B8B
:10F500006ED03D4961E03D4815F04BFE0228E3D93D
:10F5100029463A4801AB02AA15F020FE044638BB42
:10F52000019B22AA134403F8800C022133480DF1F9
:10F53000020215F0EEFD0446D0B902A8BDF8024063
:10F54000FDF796FCC1B202A812F0D6FE98B1214692
:10F5500002A8FFF7E5F8044698B1234A234B014679
:10F56000D21AD2089201264842F0010213F050FA52
:10F57000204622B070BD2A46214602A8FFF7E4F8D3
:10F58000E9E7306808221F4913F0B8FD002819DAAE
:10F59000164A154CA41A13F054FFE4080168A4019C
:10F5A00044F0010422464942174813F031FA13F09F
:10F5B00048FF00684042FFF713FA13F042FF046867
:10F5C0006442D5E7012311493374114816F008FC51
:10F5D0000F48FDF74DFC01460D48FEF7B5FCC7E7A7
:10F5E0000C49F2E7E0140220A86C0200006C020053
:10F5F000C17B0200D77B02006E7E0200D013022086
:10F60000B07B0200F41402204A7E02005F7E0200FA
:10F61000DA6D02207D7E020030B54A4D04462B682B
:10F6200085B0002B0CDA4849484B4948C91AC9082B
:10F63000890141F0010113F0DCF96FF0150028E0B9
:10F640000128FAD1434815F0ACFD0128F5D921462F
:10F6500040480DF1060215F05CFD002819DBBDF8ED
:10F6600006203D48130243EA1223ADF80840ADF8E6
:10F670000A3006F039FF014668B1334A334B374848
:10F68000D21AD208920142F0010213F0C1F94FF0F0
:10F69000FF3005B030BD3248FDF7EAFB50B92A49CA
:10F6A0002A4B3048C91AC908890141F0010113F0F9
:10F6B000A0F9ECE7C1B22A4812F01EFE40B9224977
:10F6C000224B2948C91AC908890141F00101EEE716
:10F6D0002349204603AA13F089FD01280FD01B4AB5
:10F6E000194CA41A13F0ADFEE4080168A40144F01B
:10F6F000010422461D48494213F08AF99DE7286813
:10F7000008220DEB020113F0E7FC0028C1D00F4ADC
:10F710000D4CA41A13F095FEE4080168A40144F00E
:10F72000010422464942124813F072F913F089FE8F
:10F7300000684042FFF754F913F083FE006840422E
:10F74000A7E700BFE0140220A86C0200006C0200D2
:10F75000C17B0200D0130220800802208C7E0200B0
:10F76000920B0220B37E0200C97E0200DF7E0200FF
:10F77000017F02002DE9F041022804468AB000F022
:10F780002081032800F03B81012846D1AA4815F0CA
:10F7900008FD012841D92146A7480DF11A0215F0AC
:10F7A000B8FC0446002840F0BC80BDF81A30012B9C
:10F7B00040F0F4804FF0FF339F48089315F0F1FCC0
:10F7C00003282AD902219C480DF11E0215F0A1FC44
:10F7D0000446002840F0A5800321974807AA15F0A9
:10F7E00098FC0446002840F09C80934815F0D9FC12
:10F7F000042804D90421904808AA15F09CFC8F4DD8
:10F800002B68002B0CDD8E498E4B8F48C91AC90816
:10F81000890141F0020113F0ECF86FF0150480E06B
:10F820009DF81E609DF81C80012E089F56D17A1C01
:10F830004AD106223146304602F0A6FF0623286050
:10F84000EB602B68002B27DA7E4A7D4CA41A13F05C
:10F85000F8FDE4080168A40144F00104224649428D
:10F860007A4813F0D5F813F0ECFD036840F68C22CB
:10F870005B42002100937648764B16F08AFA744872
:10F88000FDF7F6FA01467248FEF75EFB0023EB60D7
:10F8900013F0D7FD04686442781C68D0B8F1010FFA
:10F8A000099742D16C496A4816F09AFA6848FDF700
:10F8B000DFFA01466648FEF747FB286813F0F7FBBE
:10F8C0004FF0FF332B602AE04FF48172314630460F
:10F8D00002F05AFF4FF481732860B1E7022E13D172
:10F8E0007B1C07D111223146012002F04DFF11236C
:10F8F0002860A5E740F211123146012002F044FFD2
:10F9000040F2111328609BE74D4A4E4B3146D21A04
:10F91000D2089201514842F0010213F079F86FF0D9
:10F92000850420460AB0BDE8F0812868042301223E
:10F9300000934FF48D7109AB13F076FC0446B0B11F
:10F94000404A3F4CA41A13F07CFDE4080168A4016E
:10F9500044F0010422464248494213F059F828680D
:10F9600013F0A5FB13F06DFD04686442D9E7EB6862
:10F9700040F68C22CDE902832B68002100933448A5
:10F98000384B0196C5F8048016F003FA3048FDF7AD
:10F990006FFA01462E48FEF7D7FAC2E7002BC0D116
:10F9A000264B1B68002B08DA2549264B2E48C91A1E
:10F9B000C908890141F002012DE7FFF711F804465B
:10F9C000AFE71E4B1A68511C14D0596820480291A9
:10F9D000DB680021CDE9002340F68C22234B16F092
:10F9E000D8F91B48FDF744FA01461948FEF7ACFA6E
:10F9F000002496E71E49164816F0F2F9F1E70024B4
:10FA0000012302222146CDE90232CDE9044340F62A
:10FA10008C22CDE900430E48164B16F0BAF90C487B
:10FA2000FDF726FA01460A48FEF78EFA1249084801
:10FA300016F0D6F9AAE700BFD0130220E014022086
:10FA4000A86C0200006C0200137F0200497F0200D4
:10FA5000DA6D0220D57C02005D7F02002C7F02005F
:10FA6000857F02009D7F0200B87F0200D17F0200E7
:10FA7000E87F0200F67F02001D8002002DE9F041C0
:10FA8000174E05460024374628467168FEF70EF9E2
:10FA9000F0B100212846134A15F03BFA014668B13F
:10FAA000114B124A1248D21AD208920142F00102B6
:10FAB00012F0AEFF6FF01500BDE8F081284615F09A
:10FAC0002BFA0C2303FB0474A368BDE8F04118472C
:10FAD00001340B2C06F10C06D6D16FF08500EBE754
:10FAE000286E0200D0130220006C0200A86C0200F5
:10FAF0006D7A0200F7B500240C4D0D4F0D4E6B686A
:10FB000040F68C220021009330463B4616F041F926
:10FB10003046FDF7ADF9013401463046FEF714FAE0
:10FB20000B2C05F10C05EAD103B0F0BD286E0200E4
:10FB3000747B0200DA6D022000204FF0FF32034B8D
:10FB4000C3E900209A601874D8607047E01402205E
:10FB500080232DE9F0430128A5B00446029305D087
:10FB60006FF01504204625B0BDE8F083744815F009
:10FB700018FB0328F4D92146714802AB04AA15F0FA
:10FB8000EDFA041EEEDB0025029B24AA1344022199
:10FB90006A466B4803F8805C15F0BBFA041EE1DB93
:10FBA000032167480DF1020215F0B3FA041ED9DBF8
:10FBB000634815F0F6FA042829D90421604801AAFF
:10FBC00015F0A7FA041ECDDB5D4815F0EAFA05280A
:10FBD00020D905215A480DF1060215F09AFA041EA3
:10FBE000C0DBBDF80080BDF80290B8F5007FBDF81D
:10FBF0000460BDF8067011DD5249534B5348C91AD1
:10FC0000C908890141F0010112F0F3FE15E0ADF8D9
:10FC10000450D9E70023ADF80630E2E74C4806F07F
:10FC200063FC011E0CDA474A474B4A48D21AD208F5
:10FC3000920142F0010212F0EBFE4FF0FF3491E727
:10FC40004548FDF715F940B93E493F4B4348C91AAD
:10FC5000C908890141F00101D6E700223E4811465A
:10FC600003AB13F011FA044660B1364A364B014635
:10FC7000D21AD20892013A4842F0010212F0C8FEAC
:10FC800064426FE7039B374D024601462B600390A9
:10FC900003AB04A813F0F8F90446C8B12A4B294A6B
:10FCA0000146D21AD208920142F001022E4812F007
:10FCB000AFFE2E492E4816F093F82D48FDF7D8F8E0
:10FCC00001462B48FEF740F9286813F0DFF9D7E723
:10FCD000039B2A686B6092689B689A4210D01A4B0B
:10FCE00018492448C91AC908890141F0010112F0D4
:10FCF00080FE686813F0CAF9286813F0C7F99CE71A
:10FD0000002E08BF0126002F4FF47A7318BF3B4620
:10FD1000C5E9028918492E616B61D1E8EF3F43F0D4
:10FD20000102C1E8E02F0028F7D113F001057FF4AC
:10FD300019AF1248083915F0B5FB2C4612E700BF81
:10FD4000D0130220506C0200006C0200AF80020051
:10FD5000800802208C7E0200920B0220B37E0200FB
:10FD6000CA80020008150220E5800200018102001D
:10FD7000DA6D02201E81020004150220F413022015
:10FD80002DE9F04F9E4DADF5177DAB6800241C3377
:10FD90001FFA83FB5BBAADF81A304FF4A07345220B
:10FDA000CDE90844ADF820302B680A949B6907948C
:10FDB0005B68142109936B6806A89B69ADF818204D
:10FDC0005B68ADF822400A9312F0B8FA08230A26BD
:10FDD0008C49ADF830400A7889460132D2B28DF8AC
:10FDE00032400A70ADF82200ADF82C308DF8332087
:10FDF0000DAC0395ABF11401994240DC4FF0000AC1
:10FE00000BA8ADF82EA012F099FAADF82E0013F061
:10FE100018FB002200237C4DC0F800A0C5E9002398
:10FE200015F0DEFC4FF47A730A46A0FB030103FBD6
:10FE30000211764EC30B43EA4143CA0BC6E90032B6
:10FE40000321524605200DF0A9FC714C714BB0F115
:10FE50000008A4EB03042F464FEAD40419DA13F088
:10FE6000F0FAA401016844F001046B4822464942BB
:10FE700012F0CEFD28680DF5177DBDE8F08FD7187C
:10FE8000B7FBF6F006FB1070303004F8010B0133BD
:10FE9000B2E753465A4606A90DF0BCFC00280FDC19
:10FEA00013F0CFFAA401016844F0010422465B4834
:10FEB000494212F0ADFD40460DF082FC3868DAE7A9
:10FEC0000121039B04A8DA68CDF81080ADF8141066
:10FED0000DF076FD021E1BDD4FEA841ADFF860B1DB
:10FEE0004AF0030A00234FF41072404606A90DF0B1
:10FEF000C7FC051E25DC13F0A4FAA401016844F038
:10FF0000010423462A464648494212F098FDD2E7AA
:10FF1000039213F096FAA401016844F001044148E9
:10FF200049422346039A12F08AFD3F493F4815F0A3
:10FF300057FF3E48FCF79CFF01463C48FEF704F89B
:10FF4000B9E7132D05DC52462946584612F060FDEC
:10FF5000C8E79DF82130012BC4D115F041FC4FF4C6
:10FF60007A7A0B46A0FB0A010AFB0311C20B42EA94
:10FF70004142CB0BD6E90001B2EB000B63EB010170
:10FF8000C7E900B10BA8A5F11401C6E9002312F0DE
:10FF9000D5F9014650B1A201254842F0020212F003
:10FFA00037FD00220023C7E9002384E79DF83300D2
:10FFB00099F80020904207D00146A3011D4843F064
:10FFC000020312F03CFDECE79DF81A309DF81B602F
:10FFD00006EB0326AE4206D0A3012A463146164858
:10FFE00043F00203EDE7BBFBFAF20AFB12B30F4842
:10FFF000CDE9002340F68C22104B15F0CAFE98E79D
:020000040001F9
:1000000008150220898D022068110220701102203B
:10001000506C0200006C0200468102005C8102000C
:10002000A38102007481020091810200DA6D022036
:10003000DB810200E88102000582020018820200D2
:10004000C08102002DE9F74F00274FF4004A3E46D9
:100050003C46284DD5E900982B69BB422FDC012E88
:1000600019D904EB5604B4FBF6F64FF47A74B6FBD8
:10007000F4F304FB1366002140F68C22CDE9003630
:100080001D481E4B15F085FE1B48FCF7F1FE01468E
:100090001948FDF759FF484612F0F8FF404612F0A4
:1000A000F5FF1749144815F09BFE1348FCF7E0FED6
:1000B0000146114803B0BDE8F04FFDF745BFFFF71B
:1000C0005FFE08B10136044440F2E73B4FF0000CFC
:1000D0006B694FF47A7223EAE371CAFB01BC002317
:1000E00058466146FCF768FA002110F099F901378B
:1000F000B2E700BF08150220DA6D02202A82020052
:10010000557A020010B511490446FDF7CFFDD0B174
:10011000002120460E4A14F0FCFE011E0CDA0D4BA5
:100120000D4A0E48D21AD208920142F0010212F092
:100130006FFC6FF0150010BD204614F0EDFEBDE819
:100140001040FFF705BD6FF08500F4E74482020020
:10015000D0130220006C0200506C02006D7A020085
:1001600013B50A4B0A4C40F68C220021009320461E
:10017000084B15F00EFE2046FCF77AFE014620469D
:1001800002B0BDE81040FDF7DFBE00BF44820200B0
:10019000DA6D0220747B02000020034B034A1860D2
:1001A000C3E90120704700BFFC1402204500010094
:1001B00030B500241C4D85B028680394431C1CD026
:1001C0000423082200934FF4017103AB0DF0BCFB34
:1001D0000446A8B1154A164CA41A13F032F9E408E3
:1001E0000168A40144F0010422461248494212F079
:1001F0000FFC13F026F904686442204605B030BDB8
:100200000D4B18680FF05CFF28680DF0D9FA0B4908
:100210000B48AC7115F0E4FD0948FCF729FE0146D6
:100220000748FDF791FEE8E720150220006C020068
:10023000486C020052820200E01502206F82020028
:10024000DA6D02202DE9F041714D724C2F4686B0D7
:100250000023D8226F4928680DF012FB002829DC02
:100260006D4A6E4CA41A13F0ECF8E4080168A4017E
:1002700044F0010422464942694812F0C9FB13F0D8
:10028000E0F8036840F68C225B4200210093654849
:10029000654B15F07EFD6348FCF7EAFD01466148B9
:1002A000FDF752FE28680DF08BFA0023AB7106B003
:1002B000BDE8F0812378012B39D1EB79002B46D1B1
:1002C00018461E461946DFF84CC1BCF84620013AD4
:1002D00092B21F2A0DD89CF85020013612F0010F5F
:1002E0001CBF0130C0B2120748BF0133F6B248BF8D
:1002F000DBB201310C290CF10C0CE6D1DFF84481A2
:1003000098F80020B24222D040F68C220021CDE99C
:1003100001030096454B434815F03BFD4148FCF76F
:10032000A7FD01463F48FDF70FFE88F800602378DF
:10033000012B0CD0022B8BD1FB79002B88D03C48B1
:10034000FCF796FD01463A48FDF7FEFD80E794F87C
:100350004430DB077FF57CAFD4E90223CDE90223EB
:100360000021D4E904232F48CDE9002340F68C2254
:10037000304B15F00EFD2B48FCF77AFD014629485D
:10038000FDF7E2FD94F82E3040F68C22059394F8A8
:100390002D300021049394F82C302248039394F8D4
:1003A0002B30029394F82A300193238D0093224B33
:1003B00015F0EFFC1B48FCF75BFD01461948FDF703
:1003C000C3FDFE79002E7FF443AF15F009FA4FF418
:1003D0007A720B46A0FB020102FB0311C30B43EA36
:1003E000414316490F4809685B1A93FBF2F3314603
:1003F00040F68C220093124B15F0CBFC0948FCF719
:1004000037FD01460748FDF79FFD0123FB711FE7FC
:100410002015022078110220006C0200486C0200B6
:100420007A820200DA6D02208D8202009982020037
:1004300080110220C0820200D982020050120220E4
:10044000018302008A8D0220F0B5B7498DB00446C1
:10045000FDF72CFC002800F0638100212046B34A00
:1004600014F057FD011E0CDAB14AB24BB248D21A51
:10047000D208920142F0010212F0CAFA6FF015049C
:100480000AE1204614F048FD0228044600F02C81C1
:10049000032800F043810128F0D1A44814F081FE24
:1004A0000128EBD92146A14809AA14F032FE041E06
:1004B000C0F2F280BDF82430012B40F003819B484C
:1004C00014F06FFE022807D902219C4A974814F0C5
:1004D00020FE041EC0F2E080994DAB7953B19449DF
:1004E000944B9848C91AC908890141F0020112F0D9
:1004F00080FAD1E00127ADF826300B93AB884FF49A
:10050000017202213846ADF82870ADF82A300DF09E
:1005100045F90028286033DA864A854CA41A12F07F
:1005200090FFE4080168A4013C4322468648494202
:1005300012F06EFA6FF0150428680DF041F97D4B4A
:100540007B4A2146D21AD2089201804842F0010229
:1005500012F05EFA40F68C227D4B002100947D481B
:1005600015F017FC7B48FCF783FC01467948FDF742
:10057000EBFC0023AB7112F064FF046864428BE073
:1005800002264FF40171324600960DF126030DF05C
:10059000DBF9044678B1674A654EB61AF60812F0E0
:1005A00050FFB60146F00106324601686A484942EA
:1005B00012F02EFAC0E700963A464FF4017128680F
:1005C0000AAB0DF0C1F9044668B15A4A584EB61A42
:1005D00012F037FFF6080168B60146F00106324610
:1005E0005E484942E4E7009604224FF4017128680E
:1005F0000DF12A030DF0A8F9044668B14D4A4C4E9E
:10060000B61A12F01EFFF6080168B60146F00106A0
:10061000324653484942CBE70423009307224FF464
:10062000017128680BAB0DF08FF9044668B1414A9F
:100630003F4EB61A12F005FFF6080168B60146F003
:100640000106324647484942B2E7474E306830B368
:100650000FF0A0FC0123AB71AB8840F68C22002187
:1006600000933C48414B15F094FB3A48FCF700FCE2
:1006700001463848FDF768FC15F0B2F84FF47A737C
:100680000D46A0FB030103FB0511394AC30B43EAE6
:100690004143C90BC2E9003120460DB0F0BD002234
:1006A0000023CDE906230E234FF48062CDE90243F7
:1006B000CDE900442F4B3049304804940FF07EFFC1
:1006C0003060C7E7002BE7D11D4B9B7943B9184930
:1006D000184B2B48C91AC908890141F0020106E7E5
:1006E000FFF766FD0446D7E7154B9A798AB19B88D8
:1006F00040F68C22009300211C4B164815F049FB54
:100700001448FCF7B5FB01461248FDF71DFC002418
:10071000C2E71C490F4815F063FBF1E71A49F9E7F6
:100720006FF08504B8E700BF14830200D0130220E5
:10073000486C0200006C02006D7A02002415022051
:10074000201502201C8302002B830200EC83020090
:100750008D820200DA6D02204B8302007383020057
:100760009E830200C0830200E0150220DE830200A7
:100770005012022045020100C0A4022028150220C8
:10078000018402006F8202001484020013B50A4B38
:100790000A4C40F68C22002100932046084B15F0AD
:1007A000F8FA2046FCF764FB0146204602B0BDE89B
:1007B0001040FDF7C9BB00BF14830200DA6D0220B0
:1007C000747B02004FF0FF311F220020024BC3E96F
:1007D0000012024B1860704720150220E01502201D
:1007E00010B5064C236833B1FFF7E2FC206803F034
:1007F0003DF800232360002010BD00BFE01502205B
:100800002DE9F04387B00B780D46CC6904AF052B7A
:1008100008D8DFE803F003041C078DA614B10022FA
:100820005D4B1A7001942B7840F68C2200210093C6
:100830005A485B4B15F0ADFA5848FCF719FB0146D6
:100840005648FDF781FB0C37BD46BDE8F0834A6989
:10085000B2F5107F00F29C80524913F0EFFC041EA9
:10086000E0DBA98A4F4811F010FD696904460028B1
:100870003AD04B00DA1D22F007026E46ADEB020DB6
:100880000DF11008424647489BB289B2FDF744FA81
:10089000041E01DAB546C5E74FF000090294AB68C3
:1008A00040F68C2249460193CDF800903E4B3B48E0
:1008B00015F06FFA3948FCF7DBFA01463748FDF7C7
:1008C00043FBD5E90101FDF73FFB02213748FDF766
:1008D0003BFB21464046FDF737FB02213348FDF73D
:1008E00033FB4C46B5469DE70291AB6840F68C223F
:1008F000019301230146009328482B4B15F049FA38
:100900002648FCF7B5FA01462448FDF71DFBD5E95A
:100910000101FDF719FB02212448FDF715FB696968
:100920002048FDF711FB02212048FDF70DFB79E778
:10093000002C7FF477AF8B881D48391DBB8013F0E6
:1009400017FB044600283FF46DAF1A4A1A4B0146C4
:10095000D21AD2089201194842F0010212F058F856
:1009600060E7002C7FF45EAF8B881148391DBB8097
:1009700013F025FB044600283FF454AF0D4A0E4BFC
:100980000146D21AD20892010D4842F00102E5E771
:100990006FF0790446E700BF1C170220DA6D0220D1
:1009A000928402008B8D022033840200598502005C
:1009B0009C160220806C0200006C02004984020038
:1009C0006D84020070B52A4B2A4C2B4DE41AE408C2
:1009D0004FF0FF324FF0FF3328480FF06DFD284EE7
:1009E0003378002BF4D0274813F0EDFB02460121A9
:1009F000284601F0EFFE00280ADA12F022FDA601D7
:100A000046F00106324601681F4812F001F8DFE7A0
:100A10001C4813F0B1FB014638B110F10B0F04D0A4
:100A2000A2011A4842F00102EFE7EB88D9070ED580
:100A3000144813F0DFFB014648B1A201144842F00C
:100A4000010211F0E5FF0F4813F082FBC0E7EB88CD
:100A50001A0706D5A1010F4841F0010111F0C9FFA5
:100A6000F1E79B06BCD5A1010B4841F00101F5E778
:100A7000006C0200806C0200A0000220200702200F
:100A80001C1702209C160220A5840200B4840200D8
:100A9000C8840200DD840200E58402008023F0B5F2
:100AA0000128A7B00446009304D0032828D06FF093
:100AB000150023E0194814F074FB0228F7D106AEA4
:100AC0006B4632462146154814F048FB002815DBDA
:100AD0000027009D26AB2B4403F8807C03AB0193D9
:100AE000ADF8084003F0F8FA01A9ADF80A000C4887
:100AF000CDE903658DF8147013F0D8FA27B0F0BD76
:100B00000849094815F06CF90748FCF7B1F90146A6
:100B10000548FDF719FA0020F0E700BFD0130220C6
:100B20009C160220EE840200DA6D02208023F0B5CC
:100B30000128A9B00446029304D0032835D06FF0F1
:100B4000150030E01F4814F02CFB0328F7D108AD46
:100B50002A4621461B4802AB14F000FB002822DB8A
:100B6000029B28AA13440022022103F8802C154876
:100B70000DF1060214F0CDFA002814DB05ABBDF828
:100B80000660029F0393ADF8104003F0A5FA022E11
:100B9000ADF81200D3D80C4803A9CDE905578DF85C
:100BA0001C6013F05CFA29B0F0BD0849084815F044
:100BB00017F90748FCF75CF901460548FDF7C4F949
:100BC0000020F0E7D01302209C16022005850200C9
:100BD000DA6D022080224FF410732DE9F041ADF55B
:100BE0003A7D012800AF0446C7E9022305D0032857
:100BF00000F09D806FF0150451E0534814F0D1FAD5
:100C00000628F7D107F1280521462A464E4807F164
:100C1000080314F0A3FA041E41DB0026BB6802217E
:100C20004948BA1DEE5414F074FA041E37DB032150
:100C3000454807F10C0307F1A80214F08FFA041ECF
:100C40002DDBFB6807F1A802D65404213E48BA1CEC
:100C500014F05FFA041E22DB05213B483A1D14F014
:100C600058FA041E1BDBFB88F968002B3AD14B08AD
:100C7000DA1D22F007026E46ADEB020D6A469BB20A
:100C800089B207F1A800E84611F012FB30B17B8869
:100C9000BA88022BB96808D96FF01504B54620460A
:100CA00007F53A77BD46BDE8F081012A3B76F3D8D7
:100CB00097F82630C7E9045162F3410387F82630DC
:100CC000C7E9078003F008FA97F82630B8846FF375
:100CD00000031E4807F1100187F8263013F003F9CE
:100CE0000446DBE77B88BA88022BB86882D8012AE1
:100CF0003B763FF67FAF97F82630C7E9045062F3A2
:100D0000410387F8263007F1A803C7E9073103F04C
:100D1000E3F997F82630B8846FF300030B4807F126
:100D2000100187F8263013F0DEF80446B7E70849CB
:100D3000084815F055F80748FCF79AF801460548A9
:100D4000FDF702F90024AAE7D01302209C16022026
:100D500025850200DA6D02202DE9F041174E054687
:100D60000024374628467168FCF7A0FFF0B1002147
:100D70002846134A14F0CDF8014668B1114B124AC7
:100D80001248D21AD208920142F0010211F040FE3C
:100D90006FF01500BDE8F081284614F0BDF80C2373
:100DA00003FB0474A368BDE8F04118470134042C28
:100DB00006F10C06D6D16FF08500EBE7AC6E0200B1
:100DC000D0130220006C0200806C02006D7A0200D9
:100DD000F7B500240C4D0D4F0D4E6B6840F68C227C
:100DE0000021009330463B4614F0D3FF3046FCF719
:100DF0003FF8013401463046FDF7A6F8042C05F112
:100E00000C05EAD103B0F0BDAC6E0200747B0200A9
:100E1000DA6D022000204FF0FF32024B1865024BC2
:100E20001A6070479C160220A000022080224023F6
:100E30002DE9F0470228ACB00446CDE9092300F0C3
:100E40004181032800F06981012804D1B84814F0D9
:100E5000A8F9012802D86FF015040AE12146B44828
:100E60000DF1220214F055F9041EC0F20281BDF802
:100E70002230012B40F00181AD4814F092F9042892
:100E8000E9D9AC4E3778002F40F04C81CC2239465E
:100E9000304614F034FE0221A5480AABB21C14F00F
:100EA0005DF9041E06F10205C0F2E3800A9B0321EE
:100EB00033449F709E4809AB06F1430214F04EF98B
:100EC000041E06F14308C0F2D4800022099B0421CD
:100ED000334483F84320964805F1C20214F02BF9FD
:100EE000041EC0F2C680924814F05BF906280AD1AD
:100EF00005218F4805F1C60214F01DF9041EC0F249
:100F0000B8800123737031780791002940F00D817A
:100F1000894812F08BFF5022079918A814F0EFFDB2
:100F200001230799CDE91A3318AA84480BAB12F0B4
:100F3000ABF8834F834A0146BF1AFF0800283AD016
:100F4000BA01814842F0010211F062FD7A4C7F4BF8
:100F50007F4823657F4BA5646366FBF789FF042206
:100F600084F87A207C4A0023A2664FF410727B49F1
:100F7000E266C4E91C1272782546C4E91533E064C0
:100F8000002A6AD00222C4E90C330123E262744AC7
:100F9000A363C4E90F2884F82430674812F05FFF88
:100FA000044600285CD00146BA016E4842F00102B6
:100FB00011F02EFD5DE04FEA87190B9CDFF8D4A1FC
:100FC00049F00109DCB1616908291CD10120A3693C
:100FD0005E495B68D6F8C4204B60C2F3072343EA3E
:100FE000022308804B802E230CAA043102F09AFEC3
:100FF000BA015D4842F003020CA911F009FD0B98FB
:1010000012F044F8A2E718291ED1A36957491A1D06
:10101000143352F8040B9A4241F8040BF9D1022020
:10102000D6F8C4204949C2F3072343EA02230880C3
:101030004B802E230CAA043102F074FEBA014C48F6
:1010400042F003020CA9D8E7182308225046ADF855
:10105000009011F00DFD2468B4E784F824209CE78B
:10106000444AAB6A136001239380337042480FF007
:10107000FDF920462CB0BDE8F087002BF9D12D4BAF
:101080001B78002B00F088802B4812F0BFFF04462D
:1010900050B12B4A2B4B0146D21AD2089201374845
:1010A00042F0010211F0B4FCFFF7B4FE002CE0D0D6
:1010B000234A244B2146D21AD2089201304842F0EA
:1010C000010275E71B4B59781A78D3F8C450981C65
:1010D00003F14304B1B1D3F8C8300021CDE9035383
:1010E000CDE901040092274B40F68C22264814F0EB
:1010F00050FE2548FBF7BCFE01462348FCF724FFC1
:101100000024B6E7CDE90020CDE9024540F68C2267
:101110001E4B1D4814F03DFEEBE71D491A4814F024
:101120005FFEE6E76FF07E04A3E76FF07604A0E7CA
:10113000D01302201C1702209C1602205F170220E9
:10114000806C0200006C0200797B0200986D022026
:101150001E17022001080100CB8F02200B920220F3
:10116000E4170220A98502005C8502009C6D022024
:101170006D850200A000022020070220C085020029
:10118000DA850200F8850200DA6D02201886020076
:10119000358602007E8502006FF07F0469E700BF9C
:1011A0008023B0B5ADF5347D2B4800AFBB6013F0A4
:1011B000F8FF022805464CDD07F110042246022103
:1011C000254807F1080313F0C9FFA0BBBB68042D35
:1011D000E0543BDD03212048BA1D13F09AFF50BBB9
:1011E0004FF410730421FB601B4807F10C0307F157
:1011F000900213F0B3FFF0B9FB68FA8899B2F2B924
:1012000003EBD3735B10DA1D22F007026D46ADEBE2
:10121000020D6A469BB207F1900011F049F80028D0
:1012200004DD82B26946204605F0B2FFAD46E238E1
:1012300018BF4FF0FF3007F53477BD46B0BD0A4602
:1012400007F19001204605F0A3FFF0E702460146B2
:10125000F8E76FF01500EEE7D0130220802300B509
:101260000F48A3B0019313F09CFF022815DD022163
:101270000B4801AB02AA13F071FF58B9019B22AAD7
:10128000134403F8800C02A805F024FFE23818BFCD
:101290004FF0FF3023B05DF804FB6FF01500F9E765
:1012A000D0130220802300B50F48A3B0019313F0A0
:1012B00078FF022815DD02210B4801AB02AA13F0CA
:1012C0004DFF58B9019B22AA134403F8800C02A8D1
:1012D00005F0E0FEFA3818BF4FF0FF3023B05DF89C
:1012E00004FB6FF01500F9E7D0130220802310B53E
:1012F0001548C2B0CDE9003313F053FF03281FDDBA
:1013000002AC6B46224602210F4813F027FFA8B912
:10131000009B0321E05422AA0B4801AB13F01EFFEF
:1013200060B9019B42AA134403F8800C22A920460D
:1013300005F076FEFA3818BF4FF0FF3042B010BD0E
:101340006FF01500FAE700BFD0130220802300B52C
:101350000F48A3B0019313F024FF022815DD0221EA
:101360000B4801AB02AA13F0F9FE58B9019B22AA5F
:10137000134403F8800C02A805F032FEFA3818BFB7
:101380004FF0FF3023B05DF804FB6FF01500F9E774
:10139000D0130220802300B51048A3B0019313F0AE
:1013A00000FF022817DD02210C4801AB02AA13F04E
:1013B000D5FE68B9019B22AA134403F8800C02A849
:1013C00005F0EEFD40F20113C01A18BF4FF0FF30D8
:1013D00023B05DF804FB6FF01500F9E7D01302208D
:1013E000802300B50F48A3B0019313F0DAFE022862
:1013F00015DD02210B4801AB02AA13F0AFFE58B96C
:10140000019B22AA134403F8800C02A805F09EFD5C
:10141000FA3818BF4FF0FF3023B05DF804FB6FF0CF
:101420001500F9E7D0130220402370B5A6B004934D
:1014300015232024ADF806304FF0FF334048CDE9A6
:101440000244059313F0ADFE0428054604DC6FF05A
:101450001504204626B070BD23460021029A06A836
:1014600014F055FB0221364802AB06AA13F076FEB3
:101470000446002831D0334A06AB10685168127A0E
:1014800003C31A70304B0EAA03F1100614461868F5
:101490005968083303C4B3422246F7D118681B7950
:1014A000206023710421264804AB16AA13F056FECF
:1014B00004460028CDD1049B26AA1344052D03F829
:1014C000400C22D1059ABDF8061016A805F038FB8D
:1014D000C8282CD06FF07104BBE706A8FBF7C8FC46
:1014E0000028C8D0029B26AA134403F8804C03218D
:1014F000134803AB0EAA13F031FE0028A7D1039BBB
:1015000026AA134403F8600CCCE705210C480DF122
:10151000060213F0FEFD40B9062DD3D0062108487F
:1015200005AA13F008FE0028CCD0044691E70EA9C6
:1015300006A805F0E1FBE62818BF6FF00C0488E769
:10154000D0130220AD860200B786020038B50546EA
:101550000C4610F09AFEC8B16300214628460D4A99
:101560009BB2FCF7D9FB011E04DD0A48BDE83840F8
:10157000FCF7EABC084B094A0948D21AD208920182
:1015800042F00202BDE8384011F042BA2146284636
:10159000ECE700BFDA6D0220006C0200386C02003C
:1015A000FB7C020010B520228024AAB0002102A8F2
:1015B000CDE9002414F0A3FA224600210AA814F071
:1015C0009EFA154813F0EDFD0228044619DD6B461E
:1015D0000221114802AA13F0C1FDD0B9009B2AAA2A
:1015E0001344032C03F8A00C0BD003210A4801ABD1
:1015F0000AAA13F0B3FD60B9019B2AAA134403F8A9
:10160000800C0AA902A805F035FCE23818BF4FF09B
:10161000FF302AB010BD00BFD0130220102370B5D8
:10162000264986B004460193FCF740FB002842D0CF
:1016300000212046224A13F06CFC014670B1214A79
:10164000214B2248D21AD208920142F0010211F035
:10165000DFF96FF01504204606B070BD204613F088
:101660005BFC01280446F4D1154813F09AFD0128CB
:10167000EFD92146124801AB02AA13F06FFD0446D0
:101680000028E8D1124D019B2E4606AA134403F808
:10169000100C696802A8FCF7E1FA30B10C2000FBDD
:1016A0000464A36898470446D5E701340F2C05F17C
:1016B0000C05EED1CDE76FF08504CCE7CD860200B6
:1016C000D0130220386C0200006C02006D7A020018
:1016D000DC6E020013B50A4B0A4C40F68C22002146
:1016E00000932046084B14F054FB2046FBF7C0FB48
:1016F0000146204602B0BDE81040FCF725BC00BF03
:10170000CD860200DA6D0220747B02000149024896
:1017100005F098BD4D150100A1230200032808B56E
:1017200006D911F08EFE092303604FF0FF3008BD8B
:10173000034B53F83030002BF3D00020F7E700BF05
:10174000E817022070B504460D461646FFF7E6FF7F
:10175000002809DB074B4DB103EBC4025268AA42D3
:1017600004D011F06EFE0660002001E053F8340052
:1017700070BD00BFE817022038B504460D46FFF7DC
:10178000CDFF0028A9BF054B002003EBC40252681F
:10179000A4BF53F834002A6038BD00BFE817022008
:1017A00010B500244FF0FF334FF0FF320C480EF01D
:1017B00001FA0C4B53F834206AB10134042CF9D1EE
:1017C00011F03FFE17234FF0FF34036004480EF082
:1017D00069FA204610BD012243F83420F6E700BF25
:1017E000B0070220E8170220034B43F8301003EB48
:1017F000C0004260704700BFE81702200022024B81
:1018000043F83020704700BFE81702202DE9F04F61
:101810002DED028B83B00E9C9A46012CB8BF01249B
:10182000012B0CBF302320231546064608EE103A44
:1018300001274FF00A080022DFF874B0B5FBFBF96E
:101840000AB9AB4520D809F130000091B047012218
:10185000013700990A2308F1FF38B8F1010F0BFB9B
:101860001955BBFBF3FBE9D105F130000091B047FE
:10187000BAF1030F009902D1E41B002C11DC03B074
:10188000BDEC028BBDE8F08F4445E3DBBAF1020FFB
:10189000E0D818EE100ACDE900120137B047019ADE
:1018A000D7E720200091013CB0470099E5E700BF51
:1018B00000CA9A3B014B1860704700BFA800022085
:1018C0002DE9F04F002705468B464FF0FF39B8460B
:1018D0001C468DB0531E0393002605E06EB92528E3
:1018E00000F071815946A847039B13F8010F039339
:1018F0000028F3D10DB0BDE8F08F7A280AD862280D
:1019000010D8302854D045D8252800F05A812D28E9
:1019100000F05F8159462520A8475946039B187857
:10192000A847D9E7A0F16303172BF3D801A252F817
:1019300023F000BFBB1B0100FF19010015190100B6
:101940001519010015190100E1190100FF19010025
:101950001519010015190100E119010015190100FF
:101960001519010015190100A11A0100151901002E
:10197000151901008B1B0100151901006F1A0100D8
:1019800015190100151901009D1901001519010013
:10199000E119010039281AD95828BBD1039B1B78BB
:1019A000702B40F0888054F8043B0022069390E0AE
:1019B000B9F1000F0EDAB8F1000F00F00D81A0F1BF
:1019C0003009B8F1000F08BF4FF002088CE7B9F1F9
:1019D000000FF4DB0A2303FB0909A9F13009F0E742
:1019E000682803D1682F06D148277DE76C2802D1EB
:1019F0006C2F00F0F480002F8CD1074674E77A2F0B
:101A000002D154F8046B21E06C2FFAD04C2FF8D19E
:101A1000073424F00704F4E80223CDE90423049BEF
:101A20004FF0FF3013F10041059B089143F1000195
:101A300009910021DDE90823994208BF904204D2B0
:101A40005946284610F0DEFC46E7049E002E05DAD3
:101A500059462D20A847764209F1FF3943463246C0
:101A6000CDF8009059462846FFF7D0FE34E77A2F8C
:101A700002D154F8042B0FE06C2FFAD04C2FF8D180
:101A800000214FF0FF30073424F00704F4E802236C
:101A9000994208BF9042D3D34346CDF80090E1E786
:101AA00059463020A84759467820A8474FF00809E2
:101AB0004FF0010872E76C2F3FF475AF4C2F7FF4A5
:101AC00072AFE31D23F007031C4654F8082B06925F
:101AD0005A68002110234FF0400A04910791AAF19F
:101AE000040A0699CAF1200EAAF1200C21FA0AF084
:101AF00002FA0EFE40EA0E0022FA0CFC40EA0C004C
:101B000010F00F0007D1079911B9BAF1000F25D1D4
:101B10004FF0300C05E009288CBF4FF0570C4FF008
:101B2000300C6044594640B20A920793A847049B80
:101B30000A9A01330493079BBAF1000F23D1B8F13D
:101B4000030F7FF4C9AE049BC3EB4906002E7FF759
:101B5000C3AE59462020A847013EF7E7591E9945D4
:101B60000A9107DBB8F1010F06D1594630200B92DC
:101B7000A8470B9A0A9BB2E7B8F1020FFAD159466F
:101B800020200B92F4E70796A9E754F8046BB246BD
:101B900053461AF8010B68B9B8F1030F21D19E1B07
:101BA000A9EB0606002E7FF797AE59462020A847DE
:101BB000013EF7E75946A847EAE7594654F8040BAF
:101BC000AEE65946ACE63746B0464FF0FF3901263F
:101BD0008AE64FF0030887E64FF0010884E64C27B9
:101BE00082E6064680E600BF30B5002585B0CDE927
:101BF0000101044601A905480395FFF761FEDDE9EF
:101C000002309842B8BF255405B030BD21240200EF
:101C10004FF02002EFF3118382F31188BFF36F8F2F
:101C20000121044AC2F8401583F31188BFF36F8F76
:101C3000002070470090034020B1034B800143F027
:101C400001031847704700BF306D020030B5002215
:101C500089B00F490F4813F0EEFD00220023002445
:101C6000CDE906230E230C4DCDE903344FF4407229
:101C70002846CDE90144094B094900940EF09EFC29
:101C80000849284613F062FD204609B030BD00BF68
:101C9000A91C01005812022038180220F920010066
:101CA000C0B002202887020001480EF0DFBB00BF51
:101CB00038070220F0B505460020012703460246FA
:101CC0000D4E15F8014B0CB18B4200D3F0BD252C05
:101CD00002D182F00102F4E7002AF2D014F806C023
:101CE0001CF0030FEDD0732C04BF07FA03F210436E
:101CF00001330022E5E700BF7397020008B500F04A
:101D000059FA094810F052FE0423342207490848C2
:101D100013F0FAFA074B084A4FF400401A60BDE886
:101D2000084000F091BC00BF1418022000F9022006
:101D30001C180220AC000220EB290200F8B5002597
:101D40000C4BD3E8EF7FC3E8E25F002AF9D10A4CDD
:101D50000A4E361B3611B54200DBF8BD63685B796D
:101D60002BB12368DB6813B139462046984701350B
:101D70001034F0E70C180220B86C0200C86C0200A6
:101D8000044BD3E8EF2F0132C3E8E12F0029F8D14B
:101D9000704700BF0C180220044A054B9B1AB1EB98
:101DA000D30F34BF52F8310000207047006C02009E
:101DB000B86C0200094B4268C31A1B11013310B5FD
:101DC000137101224368064C5A712278196012B9C6
:101DD00004480EF04BFB0123237010BDB86C0200C9
:101DE0004B9402203807022070B5144B144C1B1B77
:101DF0009F2B4FEA231606D94FF4F971114B124A63
:101E000012480EF087FE124BD3E8EF5F6A1CC3E85E
:101E1000E12F0029F8D10DB9B54200D170BD237B67
:101E200043B123685B6903B198470422002120462F
:101E3000FFF7C0FF01351034EEE700BFC86C0200A9
:101E4000B86C02005D870200ED8702003087020057
:101E500010180220144B73B59842044602D3134B5A
:101E600098421CD300220023114801A90DF074FDF3
:101E70000546B8B90122019BD3E8EF1FC3E8E02F64
:101E80000028F9D1019E2D22331D2146184613F05A
:101E9000DDFF7E22044686F8312086F83250204647
:101EA00002B070BD034CFAE73C690200F8980200EA
:101EB0001C1802209087020048B1054B984205D3B8
:101EC000D03398422CBF002001207047002070477B
:101ED00000F902202DE9F04F4A4B04461B7885B0EB
:101EE00003B940B34FF02003EFF3118683F3118859
:101EF000BFF36F8F444810F069FD054686F31188E3
:101F0000BFF36F8F58B1414BD3E8EF2F013AC3E8CD
:101F1000E12F0029F8D194B1284610F069FE24B9C8
:101F20003B4B1B680BB1FFF709FF374810F04CFD26
:101F3000041E18BF0124204605B0BDE8F08F354BC4
:101F40001B78CBB92B7ADB0716D410F060FE8046E5
:101F5000284610F02BFE01464046FFF7ABFE064632
:101F60002D4F2E4BDFF8D0B0DB1BDB0803932C4B3F
:101F7000DB1B4FEAD30A36B92A4E2B4F4FF000082D
:101F8000BF1B3F113AE0B6FA86F1C1F11F0949467D
:101F9000284610F00EFE254B0146984202D3244AF3
:101FA00090421AD30846FFF787FF0246A8B9214B93
:101FB000994212D06B890399C3F389138B4238BFBE
:101FC00057F833204FEA8A1343F00103ADF800308D
:101FD00049464346584610F04BFD012303FA09F1E8
:101FE00026EA0106C7E773685B7923B1336829469F
:101FF00030461B68984708F101081036B845F2DBF7
:102000008AE700BF4B94022014180220081802200F
:102010000C1802204C940220006C0200B86C0200E4
:10202000586C0200B86C0200C86C02003C690200E7
:10203000F898020090870200AA870200274B73B528
:102040001B68418104469847254DE060D5E8EF3F85
:102050000133C5E8E23F002AF8D14FF02003EFF347
:10206000118683F31188BFF36F8F1E48214610F04D
:10207000A1FC86F31188BFF36F8F1B4B1B7883B1D4
:102080004FF02003EFF3118483F31188BFF36F8FB8
:102090000020FFF71FFF84F31188BFF36F8F02B09A
:1020A00070BD124A2B681268002AF8D0012B0AD1A1
:1020B000002200230E48CDE900234FF40042002304
:1020C0000EF07AFCEBE70A2BE9D1094813F0BFFBCD
:1020D000084802B0BDE870400EF0C8B9AC0002205C
:1020E00008180220141802204C940220F018022034
:1020F000581202203807022010B5FFF775FE0EF0C7
:10210000AFF90C4B186030B10B4B1B68092B02DD8B
:102110000A480EF0ABF9094C0020FFF7DBFE00285F
:10212000FAD14FF0FF324FF0FF3320460EF0C4F9E2
:10213000F2E700BFF018022008180220380702203A
:10214000F8B50E4F3D7875B9FFF74EFE0C4C0D4EAD
:10215000361B3611B54207DB0020FFF7BBFE002817
:10216000FAD101233B70F8BD63685B791BB123682A
:1021700020461B69984701351034EBE74C94022048
:10218000B86C0200C86C020007B504380190D0E8B2
:10219000EF3F5A1EC0E8E12F0029F8D1012B03D1EF
:1021A000034801A90DF00AFC03B05DF804FB00BF71
:1021B0001C180220202302491A46024813F0A4B832
:1021C000D0F90220F4180220002337B5094D0193FD
:1021D0000120FFF77FFE0446FFF7D2FD0022002317
:1021E000284601A90DF0B8FB08B1002CF0D10198E8
:1021F00003B030BDF4180220002307B5002201937C
:102200000648002301A90DF0A7FB10B1FFF7DCFF82
:102210000190019803B05DF804FB00BFF4180220A0
:10222000F0B5037A457A85B00190D8074FEA1515C5
:102230001CD4DDB1002426463146019810F0B9FCCB
:102240000746FFF739FE70B134B9019B294618697A
:10225000FFF730FD044648B124FA06F3D90702D54A
:102260003846FFF791FF0136AE42E5D3019B1A7A5B
:10227000920704D55B69084C0393039B2BB906486E
:1022800001A90DF09BFB05B0F0BD1D68204603A918
:102290000DF094FB0395F0E7F41802200EB403B59B
:1022A00003AB53F8042B014604480193FFF708FBE6
:1022B000002002B05DF804EB03B070475B30020011
:1022C0002DE9F04F11F0020485B0064690469DF8C6
:1022D000387001F0010901F0080507D011F0440F32
:1022E00037D11A463249FFF7D9FF0446B9F1000F3A
:1022F0000AD0304B304653F827202F4B2F49002A65
:1023000008BF1A46FFF7CAFF3DB12D4B304653F8C0
:1023100027202C49FFF7C2FF0546B8F1000F44D033
:10232000012303FA07F7284B17F0100F274F18BFA8
:102330001F46BDF840109DF83C00FFF72DFD3946C3
:1023400002463046FFF7AAFF2844204405B0BDE806
:10235000F08F1F4A116831B31E4A4FF4616E146842
:102360004FF47A7CB3FBF4F3B3FBF1F4B4FBFEF26D
:102370000EFB124E01FB14340CFB04F4B4FBF1FB16
:102380004FF03C0A01FB1B440CFB04F4BEFBFAF3C8
:10239000B4FBF1F1CDE901B10AFB13E100910E4963
:1023A000FFF77CFFA1E708469FE7084FC1E700BFA2
:1023B00004880200906F0200F6870200298802005C
:1023C000A46F02002C88020000880200FB87020034
:1023D00010190220141902200D88020038B50C468D
:1023E000E107054603D5084A0849FFF757FFE2060B
:1023F00008D4A3062846BDE838404CBF0449054927
:10240000FFF74CBF38BD00BFF687020029880200E5
:102410005A850200598502002DE9F0471D46089BA8
:102420001746DA0604460E4605D499064CBF2B49DA
:102430002B49FFF733FF4FF00008DFF8AC90A845B9
:102440002DDB0025DFF8A480DFF8A490DFF898A04A
:10245000BD4232D249462046725DFFF71FFF01356B
:10246000102D23D120461F49FFF718FF0025DFF864
:102470007880DFF88090DFF880A0AF4229D9725DC4
:10248000514612F80930204613F0970F08BF2E224C
:10249000FFF704FF0135102D14D1BDE8F087494640
:1024A0002046FFF7FBFE08F10108C8E76A07CFD115
:1024B00051462046FFF7F2FECAE741462046FFF7A5
:1024C000EDFECCE76B07D8D141462046FFF7E6FE8C
:1024D000D3E741462046FFF7E1FEDBE75A850200DD
:1024E000598502003C8802003A88020038880200C0
:1024F00032880200739702003E8802002DE9F047FF
:102500008B7A174613F0070805460E460A7A8AB0FA
:1025100021D0D2434989C3F3C203C1F38911CDE964
:1025200000830291F368394602F00102FFF7C8FE0A
:102530008146347AE44314F001040ED02946304633
:1025400010F021FCB8F1000F2BD042463946284646
:10255000FFF744FF25E0C146EBE7B8F1000F26D1B5
:102560002746EB6806AA069330463B46A96810F05A
:10257000F6FB069A6B681A603AB1AB68134413F81D
:10258000014CA4F10A035C425C41284610F058FD5E
:10259000069B1F44002BE4D11CB128461349FFF7CA
:1025A0007DFE284610F04CFD0AB0BDE8F0873046AD
:1025B00010F02DFB0E4902462846FFF76FFE4FF044
:1025C000100A05AA2346304606A9CDF814A010F03B
:1025D000C6FB059A002AB8D04B462846009706A9A4
:1025E000FFF71AFF059B1C44EBE700BF4188020080
:1025F0002988020073B5D0E900435D6842F20F7389
:102600008B4228BF0B46684605210C4A0FF028FF75
:1026100006462B4620460B22094910F0A7FB2B4605
:1026200032466946204610F0A1FB2B461B2220466D
:10263000044910F09BFB02B070BD00BF6A84020029
:102640007F8802006388020001230021074A10B539
:10265000074C1360A04204D801B11360054B186009
:1026600010BD012140085B00F4E700BF14190220EF
:1026700040420F00101902200122014B1A707047CE
:102680005D94022008B5034810F0DAFC0122024BE9
:102690001A7008BDD06F02005E9402200148FFF757
:1026A000A9BF00BFD06F020010B50C46084610F05D
:1026B00074FA214604480F22FFF720FF2046BDE8A8
:1026C000104010F095BA00BFD06F0200054B1B7888
:1026D0001BB141F2883013F037B8A42000210DF06F
:1026E0009FBE00BF5E9402202DE9F84FDFF8909066
:1026F00007460E460424CA46DFF888B099F8003031
:1027000033B94FF0FF324FF0FF3358460DF052FA15
:1027100032463946002000F0D5FB9AF8003080465A
:1027200013B958460DF0BEFA144DB8F1000F18D089
:1027300001232B709AF8003033B93046BDE8F88F8A
:102740005CB92C704FF0FF34002000F03BFC0028F7
:10275000F3D02B78002BF3D1EFE7013CFFF7B6FF66
:10276000F2E72B7813B1013C04D12C702B78002BAD
:10277000C4D1E2E7FFF7AAFFF8E700BF5D940220AB
:102780005E940220C407022073B505460F4C104E1C
:10279000B44207D310F055FE6A2303604FF0FF30B8
:1027A00002B070BD2368AB4200D06BB928466368A5
:1027B000CDE900129847DDE9001228B12846A36848
:1027C00002B0BDE8704018470C34E1E7F46B02003A
:1027D000006C02002DE9F04F161E8046894699B024
:1027E0004EDB4FF4004440F2E73000214FF47A72A0
:1027F000C4FB06010023F9F7DFFE0025044620464E
:10280000294612F0EFFF4F46C346CDE903010DF113
:10281000240ACDF81CA0002F39D154EA050311D0A9
:102820006A1C08BFB4F1FF3F0CD00EF085F8039B83
:102830001C1A049B63EB0105002C75F10003BCBF5F
:10284000002400250799524BA1EB0A018910594336
:102850002B46224650460EF0FDF800F10B030B2BE1
:10286000064606D840F68107DF40FF4317F0010710
:1028700044D010F0E6FD764206604FF0FF362BE0C4
:102880004FF0FF344FF0FF354FF0FF36B7E7DBF87E
:10289000000000282EDB08A9FEF76EFF014648B3B2
:1028A00018AB019307AB40F20312009305905B460F
:1028B000089810F0EDFB10F1780F024618D010F1D7
:1028C000120F05990CD1CDE90096434640F205124E
:1028D000089810F0DDFB0646304619B0BDE8F08FD1
:1028E00040B1039210F0ADFD039A52420260C4E77A
:1028F000002400250BF1080B013F8CE7CB46434633
:102900003E46CDF81CA0BBF1000F17D1002FE3D03D
:10291000002EE1DC54EA0503DED06B1C08BFB4F1E5
:10292000FF3F8FD00EF008F8039B1C1A049B63EB4B
:102930000105012C75F1000384DACDE74FF00002A8
:102940001868DA8000281DDB08A90593FEF714FF3C
:10295000059B014618B92022DA80013612E007AA49
:10296000009208984FF48272059310F091FB10F1D9
:102970000B0F0246059B09D00028B2D1B3F90620FF
:10298000002AEAD108330BF1FF3BBCE70127F9E746
:10299000CDCCCCCC014B1860704700BF2C19022065
:1029A00010B4034C24682468A4465DF8044B6047C7
:1029B0002C190220014B1B685B6818472C19022058
:1029C0002DE9F04F85B01D4803A90CF033FE032319
:1029D00000261B4CDFF864A0DFF86CB0DFF86C80D9
:1029E0002380039B1FFA86F999454D4602DA238816
:1029F0000E2B02D905B0BDE8F08F1822DAF80030AE
:102A000002FB05352B695B450CD000270D4B53F8B5
:102A1000041B2868CDE90033FAF720FA009B18B9A7
:102A200028F817900136DCE70137032FEFD1238810
:102A30005A1C228028F81390F4E700BF30190220B6
:102A4000B06D0220E06F0200F7510200B26D02206B
:102A500008B50448FEF72EFF024801F0DDF800201B
:102A600008BD00BF692A01002DE9F3410446032592
:102A7000DFF85C80154E8DF807004FF0FF334FF004
:102A8000FF3240460DF096F801220DF107010020BB
:102A900000F064FA074640460DF004F92FB1012317
:102AA0003370204602B0BDE8F0813378002BF8D0B7
:102AB000013D08D012F042FE0028DED10021422064
:102AC0000DF0AEFCD9E73570EBE700BF5F94022054
:102AD000C40702202DE9F8434668D0F80CE0CFB2D5
:102AE0004AB10C237B435EF803309A4253D013B1B2
:102AF0001B68002BF9D14FF02003EFF3118C83F307
:102B00001188BFF36F8F0C257D430EEB05031C7AF4
:102B10000134E4B21C728CF31188BFF36F8F52B38F
:102B20004FF00308DFF878C0CCF8088393F809C0A9
:102B3000BCF1000F15D14FF02008EFF3118988F395
:102B40001188BFF36F8FC2F800C0D3F80480B8F1CA
:102B5000000F1CD15A604EF8052089F31188BFF38D
:102B60006F8F03250E4BC3F80453BCF1000F02D046
:102B7000D2E901329847012C07D106EBC706B3789A
:102B800003F1804303F5A0431C60002005E0C8F872
:102B900000205A60E1E76FF00F00BDE8F88300BF46
:102BA0000050004010B5002204460121052000F02D
:102BB000B3FA052000F08CFA0222074B0020C3F87C
:102BC00018250322C3F80423E368C3E90000E3687F
:102BD000C3E9030010BD00BF00500040F8B50C244D
:102BE000114F0546FB6804FB0034012363724FF06C
:102BF0002003EFF3118183F31188BFF36F8F2368F4
:102C00002BB166681A68B342226008BF626081F324
:102C10001188BFF36F8F03B9F8BD2946D3E901626C
:102C20003846B047E3E700BFB405022008B5104BB3
:102C30001A6862B10F4AD2F80423D10707D50022DF
:102C40001A600D4BDB68587A08B9FFF7C7FF0B4BCA
:102C50001A685AB1074AD2F80423920706D500220F
:102C600001201A60BDE80840FFF7B8BF08BD00BFEB
:102C70000051004000500040B405022004510040C3
:102C8000821C084B22F07F42C3F84025D3F804256C
:102C9000904200D17047D3F80405821C22F07F4295
:102CA000F2E700BF005001400022064B1A60064ABE
:102CB000D3F800041368C01A20F07F400344136067
:102CC0000DF0E6BD405101404C19022038B51448C2
:102CD0000CF08CFC00B38368002401211B6898472A
:102CE0004FF400120F4D104BC5F808451C600F4BF8
:102CF0000121C3F880214FF480332246C5F8043304
:102D0000152000F009FA152000F0E2F90123204611
:102D1000074A13602B6038BD4FF0FF30FBE700BF60
:102D2000BE880200005001404051014000E100E037
:102D300008500140F8B52C4B2C4CD3F804252C4BF3
:102D4000B0F1FF3F08BF20461968521A22F07F43B6
:102D5000120236D4013820EAE070A042A8BF204613
:102D600001331844A04294BF0C180C194FF4803062
:102D700000271D4B1F4EC3F80803D3F80415D3F8E2
:102D8000402521F07F45521A22F07F42012A376008
:102D9000C3F840551D46C3F8440303D10F2012F079
:102DA000D3FC37604FF40012134BC3F88021D5F8E1
:102DB0000405231A23F07F43012B04D1FFF760FFA2
:102DC0000BE00020CCE724F07F43C5F84035D5F870
:102DD0000405241A023C2302F0D44FF48032024B43
:102DE000C3F80423F8BD00BF00500140FFFF7F007F
:102DF0004C1902204051014000E100E04FF0200258
:102E0000EFF3118382F31188BFF36F8F064AD2F874
:102E10000405064A1268801A20F07F4083F3118867
:102E2000BFF36F8F704700BF005001404C19022064
:102E30004FF02003EFF3118283F31188BFF36F8FFC
:102E40000649074B0868D3F8043582F31188BFF3AD
:102E50006F8F1B1A23F07F43184470474C190220D0
:102E600000500140032310B5104C114AC4E904334B
:102E7000104BA261E3614FF4806322660E4A236225
:102E80006266002310220D49E01DA3626362E362C3
:102E90002367E3666367A26612F0A2FF2046084933
:102EA00012F09EFF2023A37110BD00BF5019022015
:102EB000E88802007094022060940220F1880200E9
:102EC000F58802002DE9F84F4FF0180B224F1446F9
:102ED0000BFB0072936A556A0646AB42884634D8AB
:102EE000D2F820A0AAEB050909F1FF32944211D8CB
:102EF0004FF0180906FB09933B44586822464146A7
:102F0000284412F0EFFD09FB06762C440120746280
:102F1000BDE8F88F13449C421BD800FB0BBBBB449D
:102F2000DBF804004A4628442C4412F0DBFDB4EBE5
:102F30000A0406D02246DBF8040008EB090112F06F
:102F4000D1FD182000FB0676E0E7013B5B1BA342A6
:102F5000CED20020DCE700BF50190220F8B51823BC
:102F6000174C00FB033503FB00402544C46A0F46A1
:102F7000012C16460FD0022C1AD0F4B9284610F0B6
:102F8000AFF9864205D832463946284610F0B6F9E0
:102F900034462046F8BD284610F0A2F98642344651
:102FA00028BF044639462246284610F0A7F9F0E724
:102FB0002846BDE8F84010F0BDB90024E9E700BF9D
:102FC000501902201822034B02FB0030836A406A2A
:102FD000C01A704750190220094A0A4993680968C3
:102FE000D866196708494B6843F080534B6000234B
:102FF00083F31188BFF36F8F9368186F704700BF1A
:103000007C6C0220C475020000ED00E026498A684D
:103010004FF030001044EFF3098C80E8F01F4FF0C0
:1030200010001EEA000F04D0D2F8B40020F0040013
:1030300007E002F1740080EC108AD2F8B40050F07E
:103040000400C2F8B400202080F31188BFF36F8F12
:10305000164F4FF000664A6A8A603E60D06E0023C9
:10306000D36680F31188D2F8B40010F0040F05D1B4
:103070000023E1EE103A5EF0100E05E02EF0100E87
:1030800002F1740090EC108AEFF3148323F0040330
:1030900083F31488BFF36F8F02F1300090E8F01FC4
:1030A0008CF30988704700007C6C022004ED00E07E
:1030B0001EF0040F0CBFEFF30880EFF30980816965
:1030C00011F8021C0229FFD001B510F067F901BD0B
:1030D00043B2002B08DB012200F01F0002FA00F0CF
:1030E000024A5B0942F82300704700BF00E100E09C
:1030F00043B2002B0DDB012200F01F0002FA00F0AA
:103100005B09044A203342F82300BFF34F8FBFF31B
:103110006F8F704700E100E043B2002B01F1010125
:10312000ACBF03F16043064B4FEA4111C9B2ABBFDC
:1031300003F5614300F00F0083F800131954704742
:1031400014ED00E008B572B6044B186A18B10022FD
:103150001A6212F052F862B608BD00BF7C6C022001
:10316000C0E918120A44203A22F007021360009BBB
:1031700008495360019B21F001019360029B91611A
:10318000D3604FF08073D36100230265C366C0F83B
:10319000B4307047A3240200F8B51D4606460C461D
:1031A00017460023E1EE103AEFF3148323F00403F3
:1031B00083F31488BFF36F8F00F080FB084BE21994
:1031C00022F007049E60284684F30988002163B634
:1031D00081F31188BFF36F8F002200230FF061F994
:1031E0007C6C0220014910220A60704710ED00E05B
:1031F00072B6404080F31188BFF36F8FBFF34F8FDB
:1032000030BF62B6BFF36F8F704700BF2DE9F04348
:1032100006460D468BB0002954D02E4B2E4C2F481D
:10322000E41AE408A40144F00104ADF80040D1E937
:10323000012309680FF01CFCADF80040D5E9042318
:10324000E96827480FF014FC2246E96925480FF089
:10325000DFFBA8460027DFF89890D8ED087AFCEE4F
:10326000E77ACDED037AD8ED097AFCEEE77ACDED79
:10327000057AD8ED0A7AFCEEE77ACDED077AD8ED3B
:103280000B7A0822FCEEE77A7B1C0493BB1C0693A6
:10329000FB1C02970893484623460DEB02010437B6
:1032A000CDED097A0FF003FC102F08F11008D4D1EE
:1032B0002246296E0C480FF0ABFB2246A9690B4849
:1032C0000FF0A6FB294630460CF0CAF90BB0BDE85A
:1032D000F08300BF006C0200906C0200FC880200CA
:1032E0002B8902005A890200AC890200BB890200C6
:1032F0006989020030BFFFF7FDBF00BF144A08B55F
:10330000144B22F07F029A60BFF34F8FBFF36F8F91
:10331000D3F8882022F47002C3F88820D3F88820DC
:1033200042F4A002C3F888204FF04042C3F8342290
:10333000BFF34F8FBFF36F8F0023E1EE103A0CF015
:103340000DFA0CF015FA00F085FA0CF04FFA00BFF8
:1033500000C0000000ED00E001B572B60B4A106A33
:1033600000281EBF0021116211F047FF62B6EFF383
:103370000580A0F110004FEAC0000549014409C9C9
:103380009847BDE801400349084700007C6C0220D3
:10339000EC690200093801000FF006FB202080F3E1
:1033A000118808484FF40061401880F30988EFF352
:1033B00014800221084380F31488BFF36F8FFFF756
:1033C0009DFF000000D10220EFF30880EFF3098198
:1033D000724601B500F03CF901BD00BF70B5274B46
:1033E000274C284DE41AE408A40144F001063146B4
:1033F00025480FF0FEFAAA6A920103D53146234808
:103400000FF0F7FAAB6ADB0104D5214844F0010163
:103410000FF0EFFA1B4DAA6AD60204D51D4844F0FE
:1034200001010FF0E6FAAB6A180304D51A4844F01C
:1034300001010FF0DEFA134DAA6A510304D51748B3
:1034400044F001010FF0D5FAAB6A9A0304D5144891
:1034500044F001010FF0CDFA0A4DAB6ADB0304D54D
:10346000104844F001010FF0C4FAAB6A00206FEA83
:1034700003436FEA1343AB6270BD00BF006C0200F0
:10348000906C020000ED00E0E9890200018A020070
:10349000148A02002E8A0200588A0200768A0200EC
:1034A0009B8A0200B58A02002DE9F041274B284C87
:1034B000284DE41AE408A40144F0010807460E462A
:1034C000254841460FF095FAAA6AD10603D5414630
:1034D00022480FF08EFAAB6A1A0704D5204844F050
:1034E00001010FF086FA1B4DAB6A9B0712D544F021
:1034F000010841461B480FF07CFA696BAB6A18065D
:1035000008D5424618480FF083FA1FB1AB6A23F082
:103510008003AB620F4DAA6AD20704D5134844F06A
:1035200001010FF066FAAB6A9B0604D5104844F01F
:1035300001010FF05EFA0020064B9A6A9A6A42F087
:10354000FF029A623070BDE8F08100BF006C02009B
:10355000906C020000ED00E0E08A0200F68A0200B2
:10356000298B02003C8B0200548B02006A8B020004
:10357000898B02002DE9F0412A4B2B4C2B4DE41A8C
:10358000E408A40144F0010807460E4628484146D5
:103590000FF02FFAAA6AD10403D5414625480FF04F
:1035A00028FAAB6A1A0504D5234844F001010FF04C
:1035B00020FA1E4DAB6A9B0512D544F00108414626
:1035C0001E480FF016FAA96BAB6A180408D54246DC
:1035D0001B480FF01DFA1FB1AB6A23F40043AB6226
:1035E000124DAB6A590504D5164844F001010FF09D
:1035F00000FAAB6ADA050DD5134844F001010FF06B
:10360000F8F90020094A936A43F47F4393623070CB
:10361000BDE8F081AB6A9B04F3D50C4844F001018E
:10362000EDE700BF006C0200906C020000ED00E0CE
:10363000B88B0200CE8B0200298B0200DF8B0200C8
:10364000F88B02000D8C0200288C0200898B02008E
:103650002DE9F0435A4B8146D3F804800F461446B7
:1036600000259DB0C8F3080685F31188BFF36F8F5E
:1036700002F07F43B3F17F4F23D1D00721D451060D
:1036800003D422070ED401250EE04E494E4B4F487D
:103690005B1ADB089B0143F001010FF0AAF914F05B
:1036A000040501D0B946002500238DF80730F31E2C
:1036B000092B6CD8DFE803F0075A5E3E6B6B6B6B2F
:1036C0006B62A946F0E74FF000083E4B3E4E404883
:1036D000F61AF608B60146F0010631460FF089F9F0
:1036E000374B8DF80780DC6A14F0020405D03146B0
:1036F00038480FF07EF900241FE0DB6A5B001CD520
:10370000314635480FF075F9344B1B782BB1012049
:103710000DF10701FFF7C8FE0EE0314B1B782BB10E
:1037200001200DF10701FFF725FF05E02D4B1B8858
:103730009BB213B1FFF752FE04469DF8073093B9D0
:103740006822494602A812F0CDF9099B9DB3C3F344
:10375000080222B96FEA53236FEA432309932046F4
:1037600002A9FFF753FD1DB0BDE8F08300200DF165
:103770000701CFE700200DF10701D4E71249114BF3
:103780001948C91AC908890141F00101B1E70D4A78
:103790000D4B16489B1ADB0818F4F87F4FEA831389
:1037A000134943F0010318BF0146A6F11002114866
:1037B0000FF045F99FE723F4FF7323F00103CDE7F2
:1037C00000ED00E0006C0200906C0200408C0200F2
:1037D000638C02007A8C02009B8C020028ED00E0D2
:1037E00029ED00E02AED00E0BA8C0200058D020010
:1037F000F08C02001E8D0200024A536943F0100350
:103800005361704700ED00E0074B9968586A8842A1
:1038100003D006494FF080520A6001B50CF08EFECD
:10382000BDE80140704700007C6C022004ED00E020
:10383000BFF34F8F0549064BCA6802F4E062134399
:10384000CB60BFF34F8F00BFFDE700BF00ED00E08E
:103850000400FA05002320210348C2180133412B3C
:1038600082F80013F9D1704700E100E038B5044652
:103870004FF02003EFF3118583F31188BFF36F8FAF
:103880000CF052FC0B4B9B68A3420DD10A4B5A68BB
:10389000C2F3080222B90CF051FE2846FFF79CFB48
:1038A0005A6842F080525A602846BDE8384011F00C
:1038B00045BE00BF7C6C022000ED00E010B50E4B51
:1038C00088B002930D4B0E4C03930E4B0E4A04939B
:1038D00002AB019301A82346012100F03DF900232A
:1038E00007930A4B0121E41A05A80593069400F0FA
:1038F0003DF908B010BD00BF00000220000000002C
:1039000000000420060001000000022080080220C0
:1039100010B50B680C7A23F01F0204F01F031A4342
:10392000CB68640923F01F03044943EA440343F0CE
:1039300001038860CA600B6110BD00BF90ED00E01C
:1039400008B5074A074B0146D21AD2089201064829
:1039500042F001020FF05CF86FF0150008BD00BFE7
:10396000786C0200006C0200358D02002DE9F04FEA
:103970000746884614460026564D85B0464535DA3A
:1039800057F82630D3F80490B9F1000F51D0B9F1AF
:103990001F0F1ED919F01F0F1BD1D3F800A01AF06A
:1039A0001F0F16D150460FF025FD834609EB0A0084
:1039B00001380FF01FFD83451CD06FF0150B464AF0
:1039C000464B5946D21AD2089201454842F00102AC
:1039D00008E03146404A414B4248D21AD20892018F
:1039E00042F001020FF014F86FF01504204605B004
:1039F000BDE8F08F1BF1160FE1D0631E5B45DEDBE7
:103A0000C5F808B0E868C5F808B02B6957F8261063
:103A100020F01F0043F01F0AD1E900321A449842F7
:103A200002F1FF3918D1CA4505D15FFA8BF00FF0CA
:103A3000C0FC0136A2E7C5F808B0EB6822F01F020F
:103A400003F01F031A43EA60E0B20FF0B2FC10F17A
:103A5000160FC9D0441CECE7C5F808B02A69013B31
:103A600023F01F0302F01F021343CA45E0B22B618B
:103A7000EBD00FF09EFC10F1160FB5D0C5F808B0D2
:103A8000EA689DF808300AF1FF3A62F304038DF802
:103A900008302B699DF808205B0863F3471257F83C
:103AA00026308DF80820D3E900130B44009323F04F
:103AB0001F03441C5344A3EB0903E0B223F01F038C
:103AC0000F28039302D9FFF73BFFC0E76946FFF7D2
:103AD0001FFFBFE790ED00E0786C0200006C020071
:103AE0007E8D02005B8D02000522034B5A60BFF3FE
:103AF0004F8FBFF36F8F704790ED00E0BFF35F8F84
:103B00000022014B5A60704790ED00E038B50E4C32
:103B10002568102D14D8FFF7F1FF00200B4B0C4A3D
:103B20001A63854205D10B4B1D70FFF7DDFF0020A6
:103B300038BD616801EB0011FFF7EAFE0130F0E7E4
:103B40004FF0FF30F4E700BF1070020090ED00E08E
:103B5000AAFF44007098022010B5034C2278FFF7AA
:103B600005FF207010BD00BF709802202DE9F74FAF
:103B7000264D8A4606464FF00008AB46244FD045F6
:103B80001BDAD6F80490B9F1000F39D03168084635
:103B900001910FF02FFC0199044609EB0100013857
:103BA0000FF028FC84424FF014021A4B08D06FF03B
:103BB000150302FB08F84BF8083003B0BDE8F08F9E
:103BC00014F1160F2C60F8D01978A142F5DD02FB34
:103BD00008B0BC60BC60FC6800F10801007B64F3C5
:103BE0000400087138690C79400860F347140C71BF
:103BF000F96821F01F016960396921F01F0129610D
:103C000008F1010814350C36B9E700BFF819022095
:103C100090ED00E070980220014B1860704700BFE3
:103C200064010220F8B506460D460024064FAC425A
:103C300008DA3B6898470A28305504F1010401D09E
:103C40000D28F4D12046F8BD60010220F8B50D46DC
:103C5000094F461EC0F10104A3199D4201DC28460C
:103C6000F8BD73780A2B02D10D203B6898473B685A
:103C700016F8010F9847EFE764010220052108B507
:103C80000148FFF7E3FFFEE7A18D020010B50446EF
:103C90004FF0FF324FF0FF330A480EF0F3FB0A49B2
:103CA0000B68E018094CC4F1005202F580229042E2
:103CB0002EBF4FF0FF34E418086002480EF0DDFB21
:103CC000204610BD980702200C1A02201013032072
:103CD00038B5074C074DAC4200D138BD23681B688E
:103CE0009B681BB11B680BB1204698472034F2E754
:103CF000400802206008022038B5084C084DAC424C
:103D000000D138BD23680C33D3E8AF3F1B0702D482
:103D100020460FF0B1FB2034F1E700BF400802203D
:103D20006008022000232DE9F04F022889B00746E1
:103D30001646CDE9063304913ED106A80591014609
:103D40001A4606E00C78013201340C70D4B2072C0C
:103D500004D8049C34F81240002CF3D00133082B13
:103D600001F10101ECD14FF0FF384FF001090023C0
:103D700010F8012B4A4588BF4FFA83F803F101037D
:103D8000DBB288BF9146082BF2D19B46B9F1010FF7
:103D90004FF03A0308BF4FF0FF3803930021344639
:103DA0000D465D4517DBB44208D00023012F0CBF40
:103DB00004F8013C237002E0012804D000263046BC
:103DC00009B0BDE8F08F2E234FF0040B4FF0FF3801
:103DD00081460393E2E7BBF1040F3BD1049B5A5D9C
:103DE0004AB93023204600F8023B039B637001353B
:103DF0000446EDB2D5E74FF0090E4FF0000ACDE9C9
:103E000001243A48DDF804C0F245BCFBF0F200FBA7
:103E100012C2019201DC844508D3BCFBF0FCF246DF
:103E2000029B0CF1300C03F801CB02930A220EF135
:103E3000FF3EBEF1FF3FB0FBF2F0E3D14FF00002D6
:103E4000029B1A701B1BDAB254FA83F3581C039BB3
:103E5000A354CCE7A84510D111B9B8F1000F02D195
:103E60003A2304F8013B3A23204600F8013B09F1CC
:103E7000FF331D440021EDB2B9E711B13A2304F834
:103E8000013B059B33F81530190241EA132111F467
:103E90007F4F0AB2C1F307235FFA81FA16D00F2BC6
:103EA000D9B20BD90023612220460FF016FB012363
:103EB000612251460FF011FB012198E75BB20929FD
:103EC00094BF30335733601C2370F0E7BAF10F0F03
:103ED00003D9612251462046ECE753B2BAF1090FEB
:103EE00094BF30335733601C2370E5E700CA9A3B18
:103EF0002DE9F0410D6890F87C403B4B3B4A07466A
:103F000090F87A00053504280CBF104618460D605D
:103F100088460FF087FCC4F34004034638B9D8E95B
:103F20000020904297F87A1004D16FF00B031846E6
:103F3000BDE8F081501CC8F800001170D8E900629B
:103F40009642F2D0721CC8F8002033704146B7F890
:103F500078000FF055FC03460028E8D107F148002F
:103F60000FF060FC03460028E1D1F86D6400D8B181
:103F700097F87C3044F0040403F0010344EA43144E
:103F8000037A4146DB0003F018031C430FF04AFCA0
:103F900003460028CBD13B6E41460BB318460FF0C9
:103FA00041FC03460028C2D1786D38B141460FF07C
:103FB00039FC03460028BAD144F08004B86D38B10A
:103FC00041460FF02FFC03460028B0D144F04004D6
:103FD000347042462946BDE8F04110200FF03DBC48
:103FE0000FF00EFCDDE700BF3870020040700200E9
:103FF000D0E900239B1A012B81BF054B1B8813803E
:10400000036883BF0233436000206FF00B007047EA
:10401000BE8D0200D0E900239B1A012B81BF054B06
:104020001B881380036883BF0233436000206FF056
:104030000B007047C08D0200142390F824205343D6
:10404000014AD358184700BF4870020030B4142505
:10405000034C90F8243005FB034330BC5B681847E1
:104060004870020010B4142490F82430034A04FB72
:1040700003235DF8044B9B68184700BF487002009B
:1040800070B41426044D90F8244006FB0454E468F0
:10409000A44670BC604700BF48700200142190F82D
:1040A0002430024A01FB03231B69184748700200B1
:1040B000C26808B542B1074B82689B689A4206D134
:1040C0000BF0F0FD002008BD6FF01500FBE74FF08E
:1040D000FF30F8E77C6C022013B50A4C206818B951
:1040E00009480BF083FA2060042283680DEB02017B
:1040F0001B689847002802DAFEF79AFE01900198A3
:1041000002B010BD101A0220CE8D020008B5094B76
:104110001A786AB90121312019700521FEF7FCFFD8
:104120003120FEF7D5FF4FF00042034BC3F80423C4
:10413000002008BD7198022000100340294BF0B503
:1041400046682948134083423DD00DD8062B15D030
:1041500005D89BB1022B38D06FF0150032E0B3F5D3
:10416000801FF9D1012309E0204883422FD0B3F505
:10417000A00F2ED0B3F5800FEED10223D0064CBF96
:104180000325C2F3401582F480749705C2F34020E2
:10419000C4F3002406D512F4006F77681BD0012207
:1041A0008A40BA60327A01F01F0141EA421140EAC6
:1041B0004402002042EA03230D4A43EA850380318A
:1041C00042F82130F0BD0723D8E70423D6E70523C2
:1041D000D4E70323D2E7520542BF01228A40FA60A6
:1041E000E0E700BF0600F0000600100002004000FB
:1041F0000025844070B543684C4C1A7A01F01F03C7
:1042000043EA42130022C668D4F80403C0B202F5A0
:10421000A27554F82550C5F30425AB426CD120FAA1
:1042200002F5ED0768D5900000F1804000F54430BC
:10423000D0F8105525F00105C0F81055012000FAFE
:1042400002F2C4F808233A4DF06805EB8305D5F86F
:104250000022C84022F4403210F00100C5F80022CC
:1042600049D03069C84010F0010044D0B069C8405E
:1042700010F001004AD0F2690025CA40D2074FBFB2
:1042800003227269CA4002F001025CBFC2F102025D
:10429000D2B205F5A27154F8210010F003002FD11D
:1042A000A90001F1804101F54431D1F810651B02EC
:1042B00003F4F85326F4473626F4407643EA0242E4
:1042C00005F14003C1F810659B00D1F810659BB261
:1042D00003F1804303F544333243C1F810251860DD
:1042E000D1F8103543F00103C1F81035012303FA6A
:1042F00005F5C4F8045370BD0132082A87D1A2E73E
:104300000135082DC5D16FF01200F4E77269D5F8B8
:104310000032CA4002F00102C2F1030223F440312C
:1043200041EA0242C5F80022E5E700BF0010034061
:1043300000258440B2F5A03F70B4C4680FD1456831
:104340002E7A01F01F0545EA46151D4E803556F8B8
:104350002550ED0707D56FF0850070BC7047B2F5AA
:10436000005FE56826D00125E6688D403543E560AD
:10437000012526698D40B2F5005F14BF2E43AE4380
:104380002661A669B2F5A03FE2690CBF2E43AE4399
:10439000B3F5C02F0CBF2A43AA43E2616269B3F5AB
:1043A000802F0CBF154322EA0505A661656170BC2C
:1043B000FFF720BF01268E4025EA0605D7E700BF9C
:1043C000002584404E492DE9F0410E68002E5ED054
:1043D0004C4B0025DA68D3F804C0D2E9030303404C
:1043E000D2E90604204323EA0003DCF80400526902
:1043F000046901205440DFF818E123EA04048BBB70
:104400000B60002301201F463F49404DD1F8042393
:1044100000FA03FC1CEA020F0DD055F8232052B11C
:1044200003F5A27251F8222045F82370C2F304224A
:1044300000FA02F214430133082BE7D14CBB7EB1E2
:10444000012400252F4B324FD8685E68D0E9032342
:104450001340D0E906210A4323EA0203002B33D19B
:10446000BDE8F08103420FD09CF8087005F01F02F0
:1044700042EA47120EEB8202D2F8007223EA0003EE
:1044800027F44037C2F8007201354000B7E73446E0
:10449000B7E71C48C76879680029D0D00D68804606
:1044A000002D38BF00258A683B6922401A4202D09D
:1044B00040464B689847002DC1D02B682946002BF9
:1044C00038BF00231D46EEE71C4216D0327A05F0B5
:1044D0001F0141EA4211426907EB8101D1F800C294
:1044E000EA4002F00102C2F103022CF4403C4CEA23
:1044F0000242C1F8002223EA040301356400ADE75B
:104500007C110340440602200010034000110340C8
:1045100000258440F0B54B79012B29D0032B24D101
:1045200010268B79032B20D1CC7924B1012C1CD1FE
:1045300043681B79CBB10A7912B1022A15D10E2238
:104540000B684568B3F5164F2D6864D02DD8B3F5C8
:10455000165F63D016D8B3F5966F61D00AD8B3F55D
:10456000967F60D0B3F5167F60D06FF0850051E084
:104570000026D6E7B3F5166F5BD0B3F5965FF4D19E
:10458000364B3CE0B3F5E14F56D007D8B3F5615F49
:1045900054D0B3F5964FE8D1314B30E047F61227AF
:1045A000BB42E2D14FF4000329E0B3F5613F47D0AD
:1045B00013D8B3F5963F46D009D84DF6C027BB4275
:1045C00043D0B3F5614FD0D14FF46B0317E0B3F58F
:1045D000E13FCAD14FF0EB7311E0B3F5612F37D053
:1045E00008D8204FBB4236D0B3F5E12FBDD14FF0F4
:1045F000E86304E01C4FBB42B7D14FF08053C5F8CD
:1046000024353443C368224303C9C5F86C2583E8C5
:1046100003000020F0BD4FF41D03F0E7134BEEE75D
:104620004FF49E23EBE74FF4A033E8E74FF41C333D
:10463000E5E74FF41D23E2E70D4BE0E70D4BDEE726
:104640004FF06C73DBE70C4BD9E74FF46503D6E70B
:104650004FF07063D3E74FF08063D0E700B01300F2
:1046600000A04E0090D0030040420F0000502700F1
:1046700000C0750000F03A0000903A01F0B54568BE
:104680006B792BB32B682D79D3F80C75D3F81425DF
:1046900007F18006D3F81045D3F80805164BC1B1D1
:1046A0000121B94099600321571C43F826101EBF11
:1046B0000021803243F8221055B1012282409A60D5
:1046C0000322803043F820200022803443F8242045
:1046D000F0BD022143F82610561C1CBF803243F85F
:1046E0002210002DF4D002228034803043F82420A0
:1046F00043F82020ECE700BF00258440F7B5C668EA
:1047000001F060444068B4F1005F00683CD1B468D7
:104710000C34D4E8EF5F002D03D1C4E8E72F002F5D
:10472000F7D134D10024B568A960C0F84415C0F8A9
:104730004825184AC0F82041C0F85841C0F8042361
:1047400001228260F279012A1BD15A1C19D04FF440
:10475000004040F2E736002723EAE371C0FB01671F
:104760004FF47A72002330463946F7F725FF0246A8
:10477000002000212346CDE9000105F110000CF0D6
:104780001BF9204603B0F0BD6FF08504F9E76FF028
:104790000F04F6E7000140002DE9F74301224368CA
:1047A000D0F80C80054603200F4609681C68644B4E
:1047B0008A409A6001F1800243F822007A68501C16
:1047C0001EBF002602F1800043F82060C4F80C15DB
:1047D000B968C4F814254E1C13D0FA68501C10D0C8
:1047E000012003269040986002F1800043F8206089
:1047F000002601F1800043F82060C4F80825C4F8C1
:10480000101541462846FFF785FE0646002840F071
:1048100083800123D8F80820C8F81030002A7FD000
:10482000EC68D5F80480A368D8F8007093F89D3040
:10483000CBB1444B08F10809CDE900306946484640
:10484000414A0AF037FE414B984244D0404B41491F
:104850004148C91AC908890141F001010EF0C9F89F
:10486000A36883F89D60A06890F89D30BBB1983034
:104870000AF0EAFD354B984211D0354B354937489F
:10488000C91AC908890141F001010EF0B2F80022ED
:10489000A36808F1080083F89D200AF073FEA3685E
:1048A00093F89D20F2B193F89820D8F8081042F0C0
:1048B0000042C7F8882193F8982042F00042C1F8DE
:1048C000882093F898000AF0DDFD204B98420CD028
:1048D0006FF0040620E048460AF03AFE484610F021
:1048E0007BFCC0E70423C7F804331D4BA068C7F85E
:1048F000043308230022C7F800351A49683010F045
:104900009AFFA368C3F89450A0680022164910309B
:1049100010F091FFA368DD63304603B0BDE8F0837B
:104920000822C4F800257A680132F5D008F1140194
:10493000C4F81001C4F83415C4F838352360EBE727
:104940000025844000010307C14402000000AD0BB4
:10495000006C0200B06C0200DC8D02001C8E0200B4
:1049600010020A006B4602005147020030B585B0C4
:104970006C460546084B0FCB84E80F00002201214E
:104980000820FEF7C9FB0820FEF7A2FB21462846B7
:10499000FFF702FF05B030BDD06C020030B585B026
:1049A0006C460546084B0FCB84E80F00002201211E
:1049B0000920FEF7B1FB0920FEF78AFB21462846B5
:1049C000FFF7EAFE05B030BDE06C020030B585B0FF
:1049D0006C460546084B0FCB84E80F0000220121EE
:1049E0000A20FEF799FB0A20FEF772FB21462846B3
:1049F000FFF7D2FE05B030BDF06C020043682DE930
:104A0000F0471D68C36804469B6888B093F89D20F2
:104A100062B9D5F8081149B1C5F80821D3F8982032
:104A20000132C3F8982008B0BDE8F087D5F82431EA
:104A30000BB30021C5F82411D5F880641422C5F801
:104A4000806403A811F05BF806238DF80C30F3079F
:104A500000F1D180B70700F1D080700700F1CF805E
:104A600006F00806204603A98DF810600FF046FDF9
:104A700020460FF070FED5F81031B3B10023E66880
:104A8000C5F81031B06890F89C30002B40F0B98028
:104A9000016C51B9142203A811F031F80523204606
:104AA00003A98DF80C300FF029FDD5F84C315BB31C
:104AB000002714223946C5F84C7103A8E66811F0A6
:104AC0001EF8032303A920468DF80C300FF016FDC5
:104AD000B668F36D591C17D04FF4004E40F2E73022
:104AE00000217366336E4FF47A7223EAE37CCEFBC7
:104AF0000C010023F7F760FD0246CDE900073B46B5
:104B000006F168000BF058FFD5F8443153B3002686
:104B10004FF00408E76814223146C5F8446103A841
:104B200010F0EDFF8DF80C80BB6820461B6C03A9CC
:104B300004930FF0E3FCBB681E64DB6C43B12046BA
:104B400003A904938DF80C800FF0D8FCBB68DE64D9
:104B50006368584A1B68C3F834250522C3F8382512
:104B60000122DA62D5F820319BB1D5F80433DA0599
:104B70000FD500234FF48071C5F820316368E268D7
:104B80001B689068C3F8081301211030D96010F039
:104B90005EFED5F85831002B3FF445AFD5F804330D
:104BA0005B027FF540AF0026E368C5F858619D6859
:104BB000AB68002B3FF437AF636831461B681422A3
:104BC00003A8D3F84C7510F09AFFAB684FF480023D
:104BD000CDE90437EB682046DB1B18BF01238DF8B5
:104BE0000C30AE606368EE601B6803A9C3F808234D
:104BF0000FF084FC17E7012634E7022632E704268B
:104C000030E763681F68012380F89E30683010F039
:104C10001EFEB368D7F83C25D3F84880996DA2EB07
:104C2000080222EAE27993F89D004944996508B99F
:104C3000C3F89810002A11DD0021142203A8D3F82C
:104C400040A010F05CFF0223204603A9CDE904A890
:104C50008DF80C30CDF818900FF050FC1422002184
:104C600003A810F04CFF04238DF80C30B3682046E5
:104C70001B6C03A904930FF041FCB368DA6C1A644F
:104C800082B11A6D5A640022C3E913229A64D7F8DC
:104C9000003223F02003C7F800320022B36883F803
:104CA0009E2002E70523204603A98DF80C300FF063
:104CB00025FCF2E7729802201FB500222A20114637
:104CC000FEF72AFA064A01AB07CA83E8070018462E
:104CD00008F034FB034B1860002005B05DF804FBBE
:104CE000006D0200341A022070B50D4C02460A25F0
:104CF000002620460B4B1B68016891420ED051B133
:104D00004168591AB142C4BF04460E46013D00F144
:104D10000800F1D12046013B0260436070BD00BF36
:104D2000441A0220381A0220684620F007018D46F6
:104D300019B50F4BD3E8EF2F0132C3E8E12F00295B
:104D4000F8D103F075F90B4B1C68002C38BF002418
:104D50002CB1201D0BF08AFB2468002CF8D1FEF743
:104D6000F1F9FEF751FDBDE819408546704700BFD7
:104D7000381A02203C1A02202DE9F04F0C4689B067
:104D800010F02EFD23688046002B8A4603D10BF0DD
:104D9000F9FA3C2091E0BCBF4FF0FF3323600122C1
:104DA000002102A810F0BAFC01AD4FF02003EFF390
:104DB000118B83F31188BFF36F8F0BF051FBFFF75B
:104DC00093FF464943680A68894693424FF00003BF
:104DD00008D10193424B5A68002A71D1C3E90055AA
:104DE000012300E042608BF31188BFF36F8F002B2B
:104DF00062D02068421C66D020EAE07C4FF4004E6E
:104E000040F2E730002100234FF47A72CEFB0C0110
:104E1000F7F7D2FB0023024602A80BF04DFB4FF040
:104E20002003EFF3118B83F31188BFF36F8F002002
:104E30002B4B1A685AB1AA424DD1019D002844D18A
:104E400059681D60914200D15D60002301930BF011
:104E500007FBFFF749FFD9F8003043608BF3118857
:104E6000BFF36F8F25686B1C26D010F0B9FC4FF490
:104E70007A7C8E46A8FB0C89A0FB0C010CFB0A99DE
:104E80000CFB0E114FEAD83242EA494252194FEA5E
:104E9000D93343EBE573C50B45EA4145561B4FEA51
:104EA000D13C63EB0C07002E77F10003B8BF00265E
:104EB0002660002E3FF46DAF002009B0BDE8F08FF2
:104EC00015605D608CE70346A5E70560596891426F
:104ED00008BF5860B9E710461268ABE7381A0220DD
:104EE0003C1A02203C28014608B500F38F800028B8
:104EF0000DDCB04BB04AB148D21AD208920142F050
:104F000001020DF085FD0EF09CFAAD4BBFE0431E93
:104F10003B2BEED801A252F823F000BF89500100CC
:104F200093500100F34E0100F34E01009B5001002D
:104F3000F34E0100F34E0100A3500100AB500100FD
:104F4000F34E0100F34E0100B3500100BB500100CD
:104F5000C3500100F34E0100F34E0100F34E010077
:104F6000F34E0100F34E0100F34E0100F34E010039
:104F7000CB500100F34E0100D3500100F34E01006D
:104F8000F34E0100F34E0100F34E0100F34E010019
:104F9000F34E0100F34E0100F34E0100F34E010009
:104FA000F34E0100DB500100F34E0100E35001001D
:104FB000F34E0100F34E0100AB510100EB50010034
:104FC000F3500100FB500100035101000B5101009F
:104FD000F34E0100135101001B510100F34E01007B
:104FE000235101002B51010033510100F34E010008
:104FF0003B510100F34E0100435101004B510100B0
:10500000F34E0100F34E010053510100A0F169037A
:10501000182B3FF66EAF182B3FF66BAF01A252F87C
:1050200023F000BF5B510100F34E0100F34E01007D
:10503000F34E0100F34E0100F34E0100F34E010068
:1050400063510100F34E0100735101006B510100E7
:10505000F34E0100F34E0100F34E0100F34E010048
:10506000F34E0100F34E0100F34E0100F34E010038
:10507000F34E01007B510100835101008D5101006D
:1050800097510100A15101000EF0DBF901230360EB
:1050900008BD0EF0D6F90223F9E70EF0D2F9052388
:1050A000F5E70EF0CEF90823F1E70EF0CAF909236F
:1050B000EDE70EF0C6F90C23E9E70EF0C2F90D2377
:1050C000E5E70EF0BEF90E23E1E70EF0BAF916237C
:1050D000DDE70EF0B6F91823D9E70EF0B2F90B238D
:1050E000D5E70EF0AEF92123D1E70EF0AAF96B2334
:1050F000CDE70EF0A6F96D23C9E70EF0A2F97B23E8
:10510000C5E70EF09EF97C23C1E70EF09AF95F2304
:10511000BDE70EF096F96A23B9E70EF092F9702315
:10512000B5E70EF08EF97323B1E70EF08AF972231A
:10513000ADE70EF086F97E23A9E70EF082F9682329
:10514000A5E70EF07EF97F23A1E70EF07AF9802320
:105150009DE70EF076F9742399E70EF072F9692352
:1051600095E70EF06EF9752391E70EF06AF9772353
:105170008DE70EF066F9782389E70EF062F98C234B
:1051800085E70EF05EF940F2D17380E70EF059F931
:1051900040F2D2737BE70EF054F940F2D37376E716
:1051A0000EF04FF940F2D47371E70EF04AF97A230A
:1051B0006DE700BF006C0200206C02007F8E0200D1
:1051C000ADBAADBA4FF08052014BC3F80021704721
:1051D00000E100E04FF08052014BC3F8802170479E
:1051E00000E100E04FF00052014BC3F8002170478E
:1051F00000E100E04FF00052014BC3F880217047FE
:1052000000E100E008B50023074AC2E90033074A7D
:10521000D2E8EF1FC2E8E03F0028F9D10FF03EFBD3
:10522000BDE808400FF02FBB3C1A0220381A0220BC
:1052300040F2022398425CD007DC012843D0B0F54D
:105240008D7F35D04FF0FF30704740F203239842F6
:10525000F8D101391329F5D801A353F821F000BF83
:10526000FF520100E3520100C3520100D35201007A
:10527000E7520100EB520100EF52010045520100DC
:1052800045520100455201004552010045520100BE
:1052900045520100455201004552010045520100AE
:1052A000455201004552010045520100D95201000A
:1052B00001390629C6D8DFE801F01416181A0C22A5
:1052C0000400032306E0142906D0192906D0042976
:1052D000B8D10423136002E01423FBE7116000201F
:1052E00070470223F6E70523F4E70623F2E70723D6
:1052F000F0E70229F5D00329E3D00129A2D1012347
:10530000E8E700BF2DE9F04FA1F5807391B00138B7
:10531000052B79D8DFE803F009787894030D6FF056
:105320005E04204611B0BDE8F08F08F049FA04464B
:10533000F7E74FF00008D2E900A90021D2F808B041
:105340006846402210F0DBFB6E4655465746444601
:1053500043463D49C14532DC002CE2DC5A46494611
:10536000684608F02DFB002304469945D9DD5AF81C
:105370003320002A20DB0DEBC302D288D70742BFBF
:10538000E98841F00101E980960742BFE98841F0D0
:105390000401E980500742BFE98841F00801E98033
:1053A000D10642BFE98841F02001E980120742BFDF
:1053B000EA8842F01002EA8001330835D5E7386800
:1053C000B3800028FB8005DA306008F10108083658
:1053D0000837BFE78622FCF7B5F900231A4978B1F0
:1053E00001383060B888C20742BFB28842F001027B
:1053F000B280420742BFB28842F00202B280E4E7C4
:1054000020220134FA80EDE703290AD0042910D1C3
:10541000126832F480430CD10121921308F0D2FAC1
:1054200085E70022022108F0CDFA800300F48044D1
:1054300077E70EF006F816234FF0FF34036070E7AD
:105440006FF011046DE700BF147102000122034BDD
:105450001860036802489A76FDF79CBA941A0220F5
:105460000C7102002DE9F0418AB007460C46154642
:10547000FCF796F90646002E07F1FF3005DA4FF0EB
:10548000FF3630460AB0BDE8F0811CB32DB32B685F
:105490006A46082B0CBF1023242301AF0093394622
:1054A00008F02AFAB0F10008E9DB64B15DB17B686D
:1054B000022B15D108232B60BDF80C30638001232B
:1054C0002380049B636030460C4A08F10101FCF71D
:1054D0008BF9D6E722462746E1E72A462F46DEE744
:1054E0000A2B06D1182320462B6001A90FF0CAFA17
:1054F000E9E73046FCF782F9C1E700BF147102000A
:105500002DE9F347074690460C4619B300231A4687
:10551000C868834228D1802A57D800254FF0FF322F
:105520004FF0FF332A480AF045FB2E46DFF8A490DF
:10553000E368AB421FD8636832460193236838465C
:105540000093244943460FF0EEFB054620480AF03D
:10555000A9FB05E00DF075FF16234FF0FF35036042
:10556000284602B0BDE8F087A16801EBC301496895
:1055700001330A44CDE7A16809EB060001EBC5033E
:105580005A6851F8351010F0ADFAA3684FEAC50A11
:1055900053445B6801351E44CAE7A16801EBC603AA
:1055A0005A6862B16368384601932368009351F8E2
:1055B000361043460FF0B7FB051ED1DBA944013678
:1055C000E368B342E9D84D46CAE70026B146F7E79B
:1055D000D807022077980220F8B506460D461746F0
:1055E000FCF7DEF8041E0DDBB0B20FF06EF910F11F
:1055F0006A0F064609D10DF024FF6A230360204696
:10560000FCF7FCF84FF0FF341BE0032D03D0042D12
:1056100008BF4FF4007538460FF073F910F17B0F97
:10562000024603D10DF00DFF7B23E7E72946304604
:1056300008F0B4F8011EE2DB2046034A0131FCF712
:10564000D3F82046F8BD00BF1471020007B50190E1
:1056500018B1D0F8983A0C309847034801A90AF0DD
:10566000ADF903B05DF804FBD806022008B540F29E
:10567000012202216620FDF787F8054B18600130F2
:1056800004D10DF0DEFE0068404208BD0020FCE7BA
:10569000981A02207FB504460D46F7F7E9FB204B28
:1056A0000646186800232146CDE9003332460DF046
:1056B00059FD431C04461CD11A4A1B4CA41A0DF078
:1056C000C0FEE408A40144F0010401682246174822
:1056D0000DF09EF90DF0B5FE03685B4202930123C5
:1056E0008DF80C3015B19DF80C302B70029804B079
:1056F00070BD4FF0FF324FF0FF330D4802A90AF0A2
:10570000FBF9A642EED0074A074B21469B1ADB085D
:105710009B013246074843F001030DF090F9E1E7A1
:10572000981A0220006C0200086C0200B88E020079
:1057300000080220DB8E020030B5164D89B02B78B0
:105740002BBBFFF793FF044668B1134A134B014686
:10575000D21AD2089201124842F001020DF058F913
:10576000204609B030BD00220023CDE906230A23DC
:10577000CDE90000CDE9020304900A4B4FF48062AA
:1057800009490A480AF01AFF01232B70E8E70024B0
:10579000E6E700BFF7980220086C0200006C0200E8
:1057A0000D8F0200B1570100C0B30220AC1A0220D5
:1057B0002DE9F04F7D4F7E4EB9467E4BDFF83C829F
:1057C000F61A87B0F60803A94FF0FF324FF0FF3307
:1057D00040460AF0C1F800230399386804938DF815
:1057E0001430C1F8983A40F68C220C31CDE90033E0
:1057F0000DF0E3FC011E46DAB4016F4844F00102EB
:105800000DF006F938680DF052FC60BBFFF72EFF73
:1058100048BB6A4844F003010DF0EBF801238DF812
:1058200014300DF00EFE03685B4204930399D1F827
:10583000983A002B40F09080404603A90AF0BEF849
:105840005F4B9B68002BBED19DF81420042ABAD070
:105850005C4A13604FF0FF324FF0FF3304A95A48FF
:105860000AF0F6F8AFE70DF0ECFD44F00104016832
:10587000224656480DF0CCF8D9F800000DF017FC80
:1058800007B0BDE8F08FDDF80CA0514491F80BB0E3
:10589000BBF1000F08D0B1014D4841F001010DF0FE
:1058A000A8F86FF06803C0E704230AF10C05284646
:1058B00048498DF8143010F003FB0446E8B18DF828
:1058C00014B0CDF810B00023621B013223709DF894
:1058D0001430042B56D0404D2B68002B5BD03F4C2E
:1058E0002068002857D093422CD303990C3110F034
:1058F000F9F800232B60236098E72846384910F018
:10590000DFFA044640B102230AF117008DF8143083
:1059100010F0C8F80490D6E72846324910F0D0FAC3
:10592000044608B10323EFE728462F4910F0C8FAD0
:105930000446002834D001238DF814306FF007039B
:105940000493C0E7B101294841F001010DF051F87D
:105950006FF079030493CCE7254B00224B600B4694
:105960000A6043F8082FD3E8EF2F42F00100C3E8A4
:10597000E40F002CF7D1D3073FF562AF1D480FF0BD
:1059800091FD5DE7002A3FF451AF1B4B1A68039B62
:10599000C3F8982A4AE7002A3FF448AF094BF5E7D5
:1059A0002846F7F765FA421C91E700BF981A0220D3
:1059B000086C0200006C02002F8F0200518F020061
:1059C000500702209C1A022000080220658F020066
:1059D0009C8F0200E78F0200A81A0220A41A02205E
:1059E000EA8F0200F68F0200029002000890020087
:1059F0004D560100BC6C0220A01A0220D8060220DD
:105A0000F7B504460E46154601930B4F4FF0FF3293
:105A10004FF0FF3338460AF04FFD084B20461E601A
:105A2000074B01991D60FFF735FE044638460AF022
:105A30001DFD204603B0F0BD50070220A41A02202D
:105A4000A81A022038B50E4C0546216859B181428A
:105A500009D00C4A0C4B0D48D21AD208920142F0E0
:105A600002020CF0D5FF4FF0FF324FF0FF33084831
:105A70000AF022FD25600648BDE838400AF0F6BC71
:105A8000A01A0220086C0200006C0200299002009B
:105A9000500702200F4B70B50446186870B10568B6
:105AA0000346002D284638BF002000255E688E4240
:105AB00005D19E68964202D11846256070BD002827
:105AC000FCD006681D46002E0346304638BF002035
:105AD000ECE700BF641B02200C4A08B513785BB1E9
:105AE0000B490C4B0C48C91AC908890141F0020145
:105AF0000CF07FFF002008BD01211170074A084803
:105B0000C2E90033FFF79EFFF4E700BFF8980220D8
:105B1000186C0200006C020059900200641B022005
:105B2000315B010001480AF0BDB800BFEC0702205C
:105B300038B505464FF0FF334FF0FF320D480AF0FD
:105B400039F80D4B1B681BB9BDE83840FFF7EABFB9
:105B50001C68002C38BF002429469A685868904772
:105B6000002CF1D022682346002A38BF00221446B8
:105B7000F2E700BFEC070220641B022073B5064663
:105B80000D4679B91D4A1E4B9B1ADB089B010A463C
:105B900043F0010301461B480CF051FF6FF0150064
:105BA00002B070BD4FF0FF324FF0FF3316480AF0DD
:105BB00001F82A46314601A8FFF76CFF044618B1E8
:105BC000FFF7B0FF0020EBE70C2009F021FF019068
:105BD00020B9FFF7A7FF6FF06800E1E70460019BC1
:105BE0000A4A446084601C605168C3E9016511B9C8
:105BF000C2E90033E4E70B605360E1E7006C0200A8
:105C0000186C02007C900200EC070220641B02204A
:105C100037B505460C4679B9204A214B9B1ADB085B
:105C20009B010A4643F0010301461E480CF007FFA2
:105C30006FF0150003B030BD002301934FF0FF3229
:105C40004FF0FF33184809F0B5FF2246294601A856
:105C5000FFF720FF68B91249104B1448C91AC90848
:105C6000890141F002010CF0C4FEFFF75BFF002048
:105C7000E0E7019A01680E4B4AB95A6819609042F0
:105C800000D15960002303600FF071FBEDE7116054
:105C90005968884208BF5A60F4E700BF006C0200F0
:105CA000186C02007C900200EC070220AD9002000C
:105CB000641B0220064BC35C03F00303022B08BFE6
:105CC00020384138C0B219288CBF0020012070470D
:105CD000739702002DE9F0430568A3B000952B7877
:105CE00080460F461646002B00F0C880654B1C7896
:105CF000062C10D16B1C0093009A1078FFF7DAFF86
:105D000030B9531B2A46394630460FF0BCF91BE028
:105D100001320092F0E7072C24D168460FF0EBF82F
:105D2000009A1078FFF7C6FFA8B9531B39462A46D8
:105D300030460FF0A8F9009B1A783D2A0ED15A7808
:105D40003F2A01D1023300930020009BC8F80030A5
:105D500023B0BDE8F08301320092E1E73F2AF3D19E
:105D60000133F0E7082C03D110460FF067F9EBE799
:105D7000022C11D1009A117808460FF0B3F818B927
:105D800011B101320092F5E7531B2A4639463046DD
:105D90000FF079F9009BE3E7032C09D1009B1A78F7
:105DA000222A03D012B101330093F7E75B1BECE723
:105DB000012C3CD128460A2201A90BF0B7FC019B1B
:105DC000314D0290009300980378292B28D03BB3E3
:105DD0002C3BDBB20130112B009003D825FA03F3E2
:105DE000DB0708D4A14604E0019BB9F1200F009322
:105DF00015D04C46E7E70A2201A90BF097FC22AB2D
:105E000004F1010903EB840444F8800C0098F7F7CF
:105E10002FF804460198F7F72BF88442E4D14C465A
:105E200039463046A30002AA0FF050F9B2E7042C1D
:105E300015D10A22284602A90BF078FC029BB0F586
:105E4000803F0246009305DA82B2394630460FF0B1
:105E5000E2F879E7394630460FF002F974E7052C8D
:105E60007FF472AF0949009B1A78525C12F0440F1C
:105E700001D15B1B46E701330093F4E74FF0FF309D
:105E800066E700BFF9980220014002007397020004
:105E900010B50446F6F7ECFF012822D92178134B00
:105EA000CA5C02F00302022A08BF203941291A46BF
:105EB00017D16378D25C02F00302022A08BF203BAC
:105EC000542B0ED1A278252A0DD002F0F703232BF4
:105ED00009D010460FF006F810B9B2FA82F0400966
:105EE00010BD0020FCE70120FAE700BF7397020015
:105EF00070B5046800290546227841D12B2A294E25
:105F000001D0252A04D10623337000202C6070BDF7
:105F10002046FFF7BDFF88B30723F5E7222A06D006
:105F2000282A09D101221F4B14441A70EDE70322DD
:105F30001C4B01341A70E8E710460EF0D3FF70B125
:105F400018490878042808D114F8010F0EF0CAFF88
:105F50000028F9D105230B70D7E70828D5D02C3AB3
:105F6000D2B2112A07D8104B23FA02F2D30702D576
:105F700008220C4B13E04FF0FF30C8E70223C3E7C1
:105F800003DD2B2AF7D0252AF5D0084BD35C59071F
:105F900003D42D2A01D02B2AC0D10422014B1A7020
:105FA000B3E700BFF9980220014002007397020096
:105FB0002DE9F74F884616461F46044600287ED036
:105FC000002A7CD05368002B79D0002510460FF0B2
:105FD00004F801942C463368DFF8EC909F4228BF08
:105FE0001F46384BDFF8E4A01D70019B1A78002A89
:105FF0004BD0A74249D912F8092001A8110748BF80
:106000000133214648BF0193FFF772FF421C3CD089
:106010003246214601A8FFF75DFE431C35D0019BA7
:106020001A782C3AD2B2112A1AD82AFA02F2D107D7
:1060300016D558780EF056FF78B10134BC4239D0ED
:10604000214601A8FFF754FF421C1ED032462146CC
:1060500001A8FFF73FFE431C17D0019B01330193BA
:10606000019A10780EF03EFFF8B101321178934694
:10607000084601320EF036FF0028F7D119B12B295E
:1060800001D0252911D1CDF804B0019BA5B91A780A
:10609000002A0CBF00206FF00A00B8F1000F01D0F9
:1060A000C8F8003003B0BDE8F08F0134BC4208BF2F
:1060B00001259AE70546E8E76FF00600EDE76FF087
:1060C0001500EFE7F99802207397020001400200E3
:1060D00008B5002304481A461946FFF791FC00282A
:1060E00018BF6FF0040008BD1A91020010B50446F5
:1060F000094A084623780021FFF75AFF10F10B0FD9
:1061000000D040B904480FF04CF82378984294BF6F
:1061100000206FF00A0010BD6C1B022015289DBFE7
:10612000024B53F82030987AEA2070471072020030
:10613000002330B50D46A1B004467C22194601A8C3
:1061400000930FF0DCFCE5B1114A52F82440A27A2A
:10615000032A16D00023802269462068FFF750FCEE
:1061600090B9694604F10900FFF7C0FF38B92A4623
:10617000217A08480EF0CDFF002808BF022021B088
:1061800030BD6FF01500FAE76FF00400F7E700BFCD
:10619000107202006C1B02202DE9F04F00250E4604
:1061A000A5B08046914629467C2205A804950FF0AB
:1061B000A6FC0395002E00F0E480B9F1000F00F07A
:1061C000E080744B802253F828A004A92B46DAF80B
:1061D0000000FFF715FCB8F1020F04460CD10DF1D9
:1061E000190130460FF0FCFD3046F6F741FE01463E
:1061F000084625B0BDE8F08FB8F1090F38D0002C63
:1062000040F0C2802746DFF8B0B10094009A04AB9A
:10621000B8F1090F13440FD118465F4901930FF0ED
:106220004FFE002800F0B3800021019B24AAC01A71
:10623000471C3A4402F8801C19460AF10900FFF78E
:1062400055FF0146B8B1554A554B0090D21AD208B5
:106250009201544842F001020CF0DAFB0099C7E7C2
:106260000130013539460FF02BFE0028F8D1C6E782
:10627000494F04A8F6E79AF80A30012B1ED19AF884
:10628000081058460DF10A020EF043FF014648B1CE
:10629000424A434B0090D21AD2089201424842F03F
:1062A0000102D9E749463046BDF80A303F4A0BF0B3
:1062B000EDF8484515D96FF0790199E7032B10D116
:1062C000A9EB04039AF808100393584603AB32195C
:1062D0000EF044FF014600288AD1039B4B45EAD2C9
:1062E000F054B8F10E0F21D134463046F6F7C0FD18
:1062F000A31CA41BA0420FD8039B142B06D1F37C34
:10630000462B03D10023F37413230393039900292D
:1063100008BF6FF085016BE713F8022C13F8011C1E
:106320001C4603F8021C03F8012CDEE7B8F1090F44
:10633000ECD1002DEADD331918461D4901930FF009
:10634000BFFD30B10022019B02701846F6F790FDA8
:106350000390039B012D1C440ED0A9EB0401154AA8
:10636000301900910BF092F80028A4DD00998142C9
:10637000A1D37B1C02340093013D7FF447AF03940B
:10638000C4E76FF0150133E76FF0040130E76FF0F9
:106390000D012DE71072020059850200686C0200A1
:1063A000006C020092920200AB9202006A8402002A
:1063B0003A880200C69202006C1B02200A210148A2
:1063C0000EF0F8BD6C1B022038B5054690F86C0045
:1063D000FFF7A4FE032818D1642295F86C00A91CCD
:1063E000FFF7DAFE041E02DB0024204638BD114A06
:1063F000114B95F86C109B1ADB089B0122460F4845
:1064000043F001030CF01BFBEFE70128ECD1294618
:1064100095F86C00FFF78CFE041EE5DA054B064A82
:106420002146D21AD2089201054842F001020CF02E
:10643000EFFADAE7006C0200706C0200C992020009
:10644000E7920200002846D0012380F86C30022336
:1064500080F8DC30032380F84C31052380F8BC3110
:10646000062380F82C32072380F89C32082380F81A
:106470000C33092380F87C33042380F8EC330F239A
:1064800080F85C34102380F8CC34112380F83C353C
:10649000142380F8AC35152380F81C360A2380F8C5
:1064A000A4360E2380F81437122380F884370D2386
:1064B00080F8F4370B2380F86438132380F8D4383D
:1064C000064BC0F8D838064BC0F8DC38054BC0F88E
:1064D000E038002070476FF015007047029302000B
:1064E000149302001B9302002DE977440446002810
:1064F00000F0CE80FFF768FF054604F17000FFF75B
:1065000063FF054404F54470FFF75EFF054404F59E
:106510006070FFF759FF04F5A8730544184601930E
:10652000FFF752FF054404F52870FFF74DFF04F113
:10653000E00A05445046FFF747FF054404F57C7028
:10654000FFF742FF054404F58C60FFF73DFF05446B
:1065500004F59A60FFF738FF054404F5B660FFF7CD
:1065600033FF054404F5A860FFF72EFF019B0544A7
:1065700004F5E07104F50C72002B50D000294ED0C8
:10658000002A4CD0B4F8523104F5E170A4F8C231BD
:1065900094F854310A228370B4F855310021A4F8DC
:1065A000323294F8573104F2322684F834320BF048
:1065B00039F80021A4F8C0010A2230460BF032F865
:1065C0000021A4F8300210220D4404F2A220002180
:1065D0000BF028F8F5F786FF04F5C466C6E900015C
:1065E000BAF1000F1ED000261022314684F8E66072
:1065F00004F1E2000BF016F8A4F8E000A91914D099
:10660000254A264B2648D21AD208920142F00102AE
:106610000CF0FEF96FF00A0003B0BDE870846FF073
:106620001501D0E76FF01506E8E704F5C760FFF73E
:10663000CBFE054604F5D560FFF7C6FE054404F51C
:10664000E360FFF7C1FE291808D0134A134B154821
:10665000D21AD208920142F00102D9E704F5F160A2
:10666000FFF7B2FE054604F5FF60FFF7ADFE0544F7
:1066700004F66800FFF7A8FE2818CDD0064A074B9D
:106680000146D21AD2089201074842F00102BFE740
:106690006FF01500C0E700BF706C0200006C0200D4
:1066A00028930200469302006093020008B5FBF7AE
:1066B00047FD064B06490748C91AC908890141F038
:1066C00001010CF096F90020FDF7B2F8006C020011
:1066D000306C02008F93020070B50C4601212D4DE5
:1066E00086B02B6806460493ADF8141042F210727F
:1066F00004A8FCF76FF8002812DC274A274CA41ADC
:106700000CF09FFEE4080168A40144F00104244851
:10671000224649420CF07CF96FF0730006B070BD60
:10672000286800231F494FF41072CDE900330CF0A4
:1067300044FD011E13DA184A184CA41A0CF081FE0D
:10674000E4080168A40144F00104224616484942C5
:106750000CF05EF90CF075FE00684042DEE715D0E3
:106760001EB16B690F4889B29847062200210F4B72
:10677000009402A80FF00DFB0A4802A90FF0A0FB3D
:10678000002814BF20464FF4FA70C7E76FF0670087
:10679000C4E700BF741B0220006C0200406C0200C2
:1067A000AC930200FA980220C4930200DC9302002A
:1067B000014600F10803D3E8EF2F42F00100C3E8DF
:1067C000EC0FBCF1000FF6D1D30702D401480EF054
:1067D00069BE7047E81B02200148FFF7E9BF00BF10
:1067E000C40302202DE9F341002406460D46274646
:1067F000DFF85C80A54201D800201DE0D8F8000039
:106800000023CDE900772A1B31190CF0ABFC031EE5
:1068100015DA0C4A0C4CA41A0CF013FEE4080168BB
:10682000A40144F001042246084849420CF0F0F863
:106830000CF007FE0068404202B0BDE8F0811C4445
:10684000D8E700BF006C0200406C0200E093020039
:10685000741B022008B506210448FFF7C3FF20B9C6
:10686000BDE80840C821FFF737BF08BDF693020016
:10687000F0B5524989B00FF023FB514901300FF0B8
:106880001FFB4F4901300FF01BFB4D4901300FF04A
:1068900017FB4B4901300FF013FB451C28464849B4
:1068A0000FF00EFB1022044600210DEB02000FF04A
:1068B00026F91023621B0DEB030029460FF0D9FACD
:1068C00004A80FF0EFF8013406463E4920460FF0C9
:1068D000F7FA1022054600210DEB02000FF00FF928
:1068E000102321460DEB03002A1B0FF0C2FA04A867
:1068F0000FF0D8F8344F00EB06203B6986B2002B2E
:106900004FF00101D4BF06224FF481720846FBF715
:106910003BFF0028044610DA2C4A2D4DAD1A0CF02E
:1069200090FDED080168AD0145F001052A462948B2
:1069300049420CF06DF80CF084FD3B69002B23DD1F
:1069400003930423012200934FF48D71204603AB7F
:106950000CF06AFCC0B11D4A1D4DAD1AED080CF0DB
:1069600070FDAD0145F001052A4601681A4849420B
:106970000CF04EF820460EF029FC0CF062FD046885
:106980006442204609B0F0BD300240EA16267E81FE
:106990000822204611490CF0B1FB0028F1DA0B4A1D
:1069A0000B4DAD1A0CF04DFDED080168AD0145F041
:1069B00001052A460A484942DAE700BF038D020072
:1069C000FD930200AB900200741B0220006C0200D9
:1069D000406C0200FF930200857F02007C1B0220B6
:1069E0001794020030B5ADF5157DFFF741FF051E88
:1069F0002DDB0123274C0295ADF80C3042F21072CA
:106A0000012102A8FBF7E6FE00280FDC224A234CF6
:106A1000A41AE4080CF015FDA40144F00104224678
:106A200001681F4849420BF0F3FF0DE0BDF80E303E
:106A3000DB070FD41949184B1A48C91AC90889012C
:106A400041F003010BF0D5FF28460EF0BFFB0DF51A
:106A5000157D30BD002304A94FF410722846CDE9FE
:106A600000330CF0AAFB011E0DDA0B4A0B4CA41AE2
:106A70000CF0E7FCE4080168A40144F0010422469C
:106A800009484942CFE7DFD0A36989B204A89847F3
:106A9000B4E700BF741B0220006C0200406C0200CF
:106AA0003094020048940200559402002DE9F3410D
:106AB000047B012C08D10D30FFF794FF1B4802B076
:106AC000BDE8F04109F0D2BC64BB076DB0F854607A
:106AD0000D30FFF7CDFE051E20DBA046B4421AD2D2
:106AE00000232846CDE90088321B39190CF03AFB07
:106AF000002815DA0E4A0F4CA41A0CF0A2FCE40888
:106B00000168A40144F0010422460B4849420BF0FD
:106B10007FFF0CF096FC28460EF058FB0748CEE7A6
:106B20000444DBE702B0BDE8F08100BF6807022043
:106B3000006C0200406C02006D940200800702208D
:106B40002DE9F04198B080460E46174600215022AC
:106B500004A80EF0D4FF01215B4D06912B797BB187
:106B60005A4B5B495B48C91AC908890141F00101C8
:106B70000BF03FFF6FF01504204618B0BDE8F08120
:106B8000002FD4BF06224FF481720846FBF7FCFDAC
:106B900028602B68002B10DA4C4A4D4CA41A0CF0DC
:106BA00050FCE4080168A40144F0010422464A486C
:106BB00049420BF02DFF0CF044FC002F22DD286829
:106BC00003970423012200934FF48D7103AB0CF063
:106BD0002BFBB0B13D4A3E4CA41A0CF032FCE40849
:106BE0000168A40144F001043C48224649420BF0EC
:106BF0000FFF28680EF0EAFA0CF023FC04686442E8
:106C0000BAE72F610021404603AB04AA0CF03CFA1E
:106C1000044608B9039B73B92D4A2C4B2146D21A5E
:106C2000D20892012E4842F001020BF0F1FE2868D2
:106C30000EF0CCFAA0E701279B6976BA5B6828685A
:106C40002F816E81EB60082226490CF057FA00284C
:106C500014DA1E4A1E4CA41A0CF0F3FBE408016877
:106C6000A4013C43224649421F480BF0D1FE28684C
:106C70000EF0ACFA03980CF009FABDE703980CF09B
:106C800005FADC213846FFF727FDDC280446CED183
:106C9000164B4FF41072002100931548154B0FF05E
:106CA00078F81348F6F7E4F801461148FFF79AFD23
:106CB00004460028BBD1C8213846FFF70DFDC8287F
:106CC00004463FF459AFB2E7741B0220006C020087
:106CD000406C02008394020099940200857F0200B8
:106CE000B19402007C1B0220D4940200F7940200AD
:106CF000FA980220ED94020037B5224B4FF410723F
:106D000000900D46204800210FF043F81E48F6F78A
:106D1000AFF801461C48FFF765FD044678BB40F21A
:106D20004B110120FFF7D8FC40F24B139842044668
:106D300015D14FF410720021144B134800950FF039
:106D400028F81148F6F794F801460F48FFF74AFD76
:106D50000446A0B9E6210120FFF7BEFC0446E62C5C
:106D60000DD101220A4B1A714FF4F0120023094889
:106D7000CDE900234FF40042002309F01DFE204618
:106D800003B030BDFF940200FA980220099502007A
:106D9000741B0220A806022038B506210B48FFF715
:106DA00021FD044638B9DD210120FFF795FC04469A
:106DB00007480EF04CFD074D28680EF007FA002337
:106DC0002B714FF0FF3320462B6138BD1395020025
:106DD000A8060220741B022008B506210E48FFF702
:106DE00001FD18B9D7210120FFF776FC06210B48D9
:106DF000FFF7F8FC30B9D3210120FFF76DFCD32851
:106E000001D1D32008BDD3210120FFF765FC10F18B
:106E1000740FF4D1F6E700BF1A9502002195020025
:106E200008B550B908210948FFF7DCFC60B9BDE896
:106E30000840C8210120FFF74FBC012802D10821DA
:106E40000348F1E76FF0150008BD00BF2895020068
:106E50003195020008B505210548FFF7C3FC30B99C
:106E6000BDE8084040F201110120FFF735BC08BD24
:106E70003A950200F0B506460D462E480621A3B00D
:106E8000FFF7B0FC0746002850D1E3210120FFF7AF
:106E900023FCE328044630D1274C4B22274904F138
:106EA0000D000EF0A5FF012330462373F5F7E0FF38
:106EB000044628465CB3F5F7DBFF014600B38022A9
:106EC0003946CDE900651E4B02A80EF062FF02A80C
:106ED000F5F7CEFF014602A8FFF784FC04461648EA
:106EE000FFF766FC4CB9E2210120FFF7F5FB10F13A
:106EF000740F044601D0E228F5D1204623B0F0BD3E
:106F00008022104B009602A80EF043FFDFE7F5F752
:106F1000AFFF20B1802221460A4B0095F3E70A4BD0
:106F200018689B880290ADF80C30D0E76FF004042D
:106F3000E3E700BF40950200901B0220FA98022070
:106F400047950200549502005E95020013B5104962
:106F50000446F5F783FF58B906210E48FFF742FCB7
:106F6000A0B9FA21012002B0BDE81040FFF7B4BB80
:106F700000214FF41072084B084800940EF009FFEE
:106F80000648F5F775FF01460448E7E702B010BD73
:106F900065950200689502006F950200FA9802203C
:106FA00007B50D4B00214FF4107200900B480EF006
:106FB000F0FE0A48F5F75CFF01460848FFF712FCAF
:106FC00038B940F20111012003B05DF804EBFFF77E
:106FD00083BB03B05DF804FB78950200FA980220A9
:106FE00007B50D4B00214FF4107200900B480EF0C6
:106FF000D0FE0A48F5F73CFF01460848FFF7F2FBD0
:1070000030B9FA21012003B05DF804EBFFF764BB4F
:1070100003B05DF804FB00BF81950200FA980220DE
:1070200013B54FF41072184B00900C46174800210E
:107030000EF0AFFE1548F5F71BFF01461348FFF7AA
:10704000D1FB20B94FF4AF710120FFF745FBB0F53C
:10705000AF7F16D100214FF410720D4B0B480094F6
:107060000EF097FE0948F5F703FF01460748FFF7C2
:10707000B9FB30B9FA21012002B0BDE81040FFF79A
:107080002BBB02B010BD00BF8A950200FA98022007
:107090009495020007B50D4B00214FF4107200903B
:1070A0000B480EF076FE0A48F5F7E2FE0146084866
:1070B000FFF798FB30B9FA21012003B05DF804EB2B
:1070C000FFF70ABB03B05DF804FB00BF9E9502000A
:1070D000FA98022070B506210646A2B02548FFF7AF
:1070E00081FB054600283FD1E3210120FFF7F4FA98
:1070F000E32804463AD1204C4B22204904F10D00EC
:107100000EF076FE01232946237380221C4B009645
:1071100002A80EF03EFE02A8F5F7AAFE014602A85C
:10712000FFF760FB00BB2046FFF742FB154D4FF019
:10713000FF334FF0FF32144809F0BEF902216B69AA
:1071400012489847E2210020FFF7C6FA10F1740FA9
:1071500004460BD0E228F5D108486D69F5F788FEA2
:1071600081B20648A84701E06FF00404204622B02F
:1071700070BD00BF40950200901B0220FA980220CB
:10718000A8950200741B022068070220598502009E
:107190002DE9F041804615460E46A2B0C9B1C2B1F4
:1071A00006212348FFF71EFB074600283CD1E321B8
:1071B0000120FFF791FAE328044631D11D4C4B2200
:1071C0001D4904F10D000EF013FE27732665A4F887
:1071D000545080220021194BCDF8008002A80EF0F7
:1071E000D8FD02A8F5F744FE014602A8FFF7FAFA17
:1071F000044656B14DB10F48FFF7DAFA4FF0FF32AF
:107200004FF0FF330E4809F057F94CB9E221012045
:10721000FFF762FA10F1740F044601D0E228F5D1AD
:10722000204622B0BDE8F0816FF00404F8E700BF0B
:1072300040950200901B0220FA980220B2950200AD
:107240008007022010B5B8B1B1B100244FF0FF3271
:107250000B4BC3E904201A6099614FF4006209489E
:107260001C7109490E2309F037FA2046074B084ADA
:107270001C60C3E9012410BD6FF01500FBE700BFDF
:10728000741B0220E81B0220C0B70220901B0220C2
:10729000AD6A01002DE9F0430025214C214E54F840
:1072A000048CDFF8889085B0A84503D8002005B08D
:1072B000BDE8F083636A96E807001F6801AB83E8C6
:1072C00007000C22194638460EF0FEFB90B98FB12C
:1072D000636A21691B681A6991420BD19A69A16995
:1072E000914207D8E169914204D962695B6932EA47
:1072F00003030AD0276A67B10B480BF0A4F840409B
:1073000080F311884FF0040002DFE36801351C446C
:10731000CAE748460BF097F8636A1F60F5E700BFBD
:107320003CC200000C6D0200C7950200F0950200FF
:1073300010B50446006804F0D9FCA06818B1BDE897
:10734000104007F0A7BA10BD30B53B4B85B01D68A3
:10735000002D4CD048F20203994253D01CD948F278
:10736000030399425AD049F20103994247D10024BC
:1073700043680268CDE90244CDE90023E869694623
:1073800003685B68984701304ED020462B6843F471
:1073900080332B6005B030BD48F2010399422ED1F5
:1073A000C368002B35D1286810F480003ED02B68CC
:1073B0009BB2012B05D12B681B0C1B0443F002036D
:1073C0002B601E4B1A7802F0FF01002A31D01C4AB4
:1073D000117809B901211170002018702B6823F46D
:1073E00080032B602B6843F400032B60D2E7006816
:1073F0000028CFD004F07AFC284605B030BD00202C
:1074000005B030BD2B6813F480030BD0C068002892
:10741000E4D00E2300206B6005B030BDC368012BA3
:10742000A5D1F6E71846B5E70220B3E70E236B6057
:10743000B0E7034A1170CFE7BC1C02203A9B022040
:107440003B9B0220002310B50848094C09490A4A11
:10745000237003600B70136004F00CFC18B9012258
:10746000064B1A7010BD4FF0FF3010BDBC1C02203F
:107470003B9B02203A9B0220B81C02203C9B02202E
:107480002DE9F04700245B4B84B01B780194002B5E
:1074900000F09F806628804640F08F800229894650
:1074A00040F08B8040F205239A42924640F085805E
:1074B000514F3D68002D40F08680504A01A807F0EA
:1074C00011FD019B0646002B00F08D802946042209
:1074D0004B483B600EF013FB019C2946C4E903892D
:1074E000C4F814A002A804F0CBFB002842D101226A
:1074F0000421029B434D58739873D8735872987245
:10750000D87219722A701A732268184642F48002DF
:10751000226047F2010104F0CBFB68BB616A4FF4C3
:107520000002002908BF4FF0FF3104AB43F8041DEF
:107530003046114607F088FD044610B3019A002E2C
:10754000136843F400331360019A136823F4800333
:107550001360019A136823F4000313603FDA0023D9
:1075600020463B604FF0FF36FDF7BCFC304604B0D0
:10757000BDE8F0870C24E1E7029804F0AFFB052496
:10758000DCE7304607F0E0FD20B1446814B1002389
:107590004360D3E73046019A136843F40033136025
:1075A000019A136823F480031360019A136823F48B
:1075B0000003136004B0BDE8F0871620FDF792FCCD
:1075C0004FF0FF36D2E70120FDF78CFC4FF0FF367D
:1075D000CCE70520FDF786FC4FF0FF36C6E73046C6
:1075E00007F0E4FCBBE71820FDF77CFC4FF0FF360A
:1075F000BCE700BF3C9B0220BC1C02203173010091
:10760000B81C02203A9B02202DE9F04387B00029E4
:107610006BD0002A174668DD1D4680460E4607F0EF
:1076200093FD0446002866D04DBBE069AA070368B5
:10763000DB682DD59847013047D02368E06913F403
:10764000803344D0002123682A4623F4803323600A
:10765000CDE90411CDE90267036802A99B68984748
:107660000546E0690368DB689847013003D023686A
:1076700043F480332360284607B0BDE8F08315F05B
:107680002A0FD2D12D20FDF72DFC4FF0FF35F2E768
:10769000226812F08059CDD19847431CCDD1226A7F
:1076A00006AB002A18BF10464FF4803243F8140D81
:1076B0001146404607F0C8FC58B14FF0FF35FDF7C2
:1076C00011FC284607B0BDE8F0832320F5E71D46EE
:1076D000C8E7404607F038FD03460028ADD04068B3
:1076E0000028AAD0C3F80490E7E71620FDF7FAFBBC
:1076F0004FF0FF35BFE70920FDF7F4FB4FF0FF35F2
:10770000B9E700BF2DE9F04182B000296BD0042A0F
:1077100069D11F4606460D4607F016FD04460028AF
:1077200074D0E7B1B8076BD523689B0364D50027F5
:107730002368002123F4003323606846D5F80080D5
:1077400004F09EFA98B10C20236843F400332360C0
:10775000FDF7C8FB4FF0FF3002B0BDE8F0810368D1
:10776000D900E1D403689A0348D50127E0E704254E
:10777000009B47F20301C3F80C8058729872D872CC
:107780001D72184604F094FA804618BBD7B1616A9E
:107790004FF48032002908BF4FF0FF3102AB43F8AD
:1077A000041D3046114607F04FFC20B1236843F416
:1077B00000332360CCE7304607F0C6FC034608B12F
:1077C0004068B0B92846236843F40033236002B010
:1077D000BDE8F081009804F081FA2368052043F4A5
:1077E00000332360B4E71620FDF77CFB4FF0FF3039
:1077F000B2E7C3F80480D9E77320A9E70920A7E717
:107800002D20FDF76FFB4FF0FF30A5E70920FDF7B6
:1078100069FB4FF0FF309FE7F0B5012985B06DD0CF
:107820001E4640F20523994240F0A08007461546C7
:1078300007F08AFC0446002800F0C380012D19D00F
:10784000022D10D02A25036823F4800323602368C7
:10785000284623F400032360FDF744FB4FF0FF3577
:10786000284605B0F0BD16B10A9B012B4ED0236807
:107870001625E9E7002EFAD00A9B042BF7D1002148
:1078800003A804F0FDF90546002875D103980822E5
:1078900029460C300EF033F9039831460A9A0C3021
:1078A0000EF020F90823039847F202010372457293
:1078B0008572C572236843F48003236004F0F8F9ED
:1078C000002878D1616A4FF40002002908BF4FF008
:1078D000FF3104AB43F8081D3846114607F0B4FBEE
:1078E0000546002840D1384607F02EFC00284ED02F
:1078F0004368002B4BD045601D4635E00A9C009440
:1079000007F04AFC0546284605B0F0BD002102A854
:10791000357804F0B5F978BB012D08BF2C4B4FF03A
:10792000040208BF1D700023029847F20101437250
:10793000C5608372C3720272236843F480032360BC
:1079400004F0B6F9064680BB616A4FF400020029D4
:1079500008BF4FF0FF3104AB43F8041D3846114611
:1079600007F072FB054650B123686DE72A20FDF74A
:10797000B9FA4FF0FF3573E723680C2564E7384602
:1079800007F0E2FB40B1456835B14660ECE73146AF
:10799000042210480EF0A6F8236823F48003236025
:1079A000236823F4000323605AE7029804F096F951
:1079B0000525236848E7039804F090F90525236816
:1079C00042E70920FDF78EFA4FF0FF3548E700BF88
:1079D0003A9B0220B81C0220F0B5012983B0089E12
:1079E00030D01F4640F20523994234D1154607F0A6
:1079F000ABFB002837D0012D15D0022D0BD187B35A
:107A0000336873B30023012218461A490978397084
:107A1000326003B0F0BD0920FDF764FA4FF0FF3388
:107A2000184603B0F0BDE7B13368032B19D93846C7
:107A3000042211490EF056F8002304221846326041
:107A400003B0F0BD009607F0EDFB03460028E3D13C
:107A5000184603B0F0BD2A20FDF744FA4FF0FF337B
:107A6000DEE71620D8E70920FDF73CFA4FF0FF3398
:107A7000D6E700BF3B9B0220B81C022010B504468D
:107A800007F062FB38B1204607F090FA0023054A60
:107A90001846136010BD0920FDF724FA4FF0FF309F
:107AA00010BD00BFBC1C022000F0DABE00F05ABFBF
:107AB00000F0C0BF00F0AEBD00F064BA014B18602A
:107AC000704700BFCC1C0220F0B56E4B83B01B7812
:107AD000002B00F0D3806C4B1C6824B1A368626853
:107AE000934240F08C80694B1C681CB1A3686268AB
:107AF000934246D1664B1C681CB1A36862689342EE
:107B000001D103B0F0BD4BF6EF62ADF80020227852
:107B10006E468DF804206268052193422ABF2769CA
:107B2000D71AFF1A934294BF0025E568BFB288BFF9
:107B3000521B304688BF95B2ADF802700CF0B9FE0A
:107B4000BDF80210A0680CF0B4FEA36822691F44BF
:107B5000974208BFE368A76008BFA360002DD0D09C
:107B600005213046ADF802500CF0A3FEBDF802101E
:107B7000E0680CF09EFEBDF80220E3681344A360A9
:107B8000BFE74BF6EF62ADF8002022786E468DF825
:107B900004206268052193422ABF2769D71AFF1A79
:107BA000934294BF0025E568BFB288BF521B3046A0
:107BB00088BF95B2ADF802700CF07BFEBDF80210E4
:107BC000A0680CF076FEA36822691F44974208BFA4
:107BD000E368A76008BFA360002D8BD00521304665
:107BE000ADF802500CF065FEBDF80210E0680CF034
:107BF00060FEBDF80220E3681344A3607AE74BF609
:107C0000EF62ADF8002022786E468DF8042062689D
:107C1000052193422ABF2769D71AFF1A934294BFBE
:107C20000025E568BFB288BF521B304688BF95B2B9
:107C3000ADF802700CF03DFEBDF80210A0680CF02B
:107C400038FEA36822691F44974208BFE368A76013
:107C500008BFA360002D3FF446AF05213046ADF8C4
:107C600002500CF026FEBDF80210E0680CF021FE78
:107C7000BDF80220E3681344A36034E7FDF7BAFAC5
:107C800029E700BF3D9B0220C81C0220C01C022027
:107C9000C41C022000222DE9F04FB24B83B01B68B8
:107CA00019695C69187C1A74587C5A74987C9A74A7
:107CB000D87CDA74187D1A75587D5A75987D9A7536
:107CC000D87DDA75A9B10139032912D8DFE801F0AE
:107CD0007CA902140125032000226FF05F01A24C51
:107CE00025701C7A1872587A5A72987A9A72DA7ACF
:107CF000D97203B0BDE8F08F042100226FF05F005D
:107D00001C7A1972597A5A7297499C7A9A72DC7A5B
:107D1000D8720A700B78002B00F09F80934B1C6880
:107D200024B1A3686268934240F0D980904B1C68EC
:107D300024B1A3686268934240F092808D4B1C6826
:107D4000002CD6D0A36862689342D2D04BF6EF6283
:107D5000ADF8002022786E468DF804206268052177
:107D600093422ABF2769D71AFF1A934294BF00256E
:107D7000E568BFB288BF521B304688BF95B2ADF8E8
:107D800002700CF096FDBDF80210A0680CF091FD99
:107D9000A36822691F44974208BFE368A76008BF31
:107DA000A360002DA5D005213046ADF802500CF09F
:107DB00080FDBDF80210E0680CF07BFDBDF80220EC
:107DC000E3681344A36094E7674A117809B100217E
:107DD0001170A568002D3BD04FF0000CDFF890A18A
:107DE000DFF888B16349E14666466246D1F800E0B3
:107DF000DAF80080DBF8007008E0632916D061290A
:107E000004BF074601260132AA4213D0911C04EB9D
:107E10008101486801786229EFD180464FF001095D
:107E2000F1E7FDF7DFF903B0BDE8F08F86464FF0CC
:107E3000010CE8E7002E40F09180B9F1000F01D06D
:107E4000CAF80080BCF1000F02D04A4AC2F800E034
:107E5000012000226FF05F0143E7FDF7CBF95DE7FA
:107E60004BF6EF62ADF8002022786E468DF80420C4
:107E70006268052193422ABF2769D71AFF1A9342E5
:107E800094BF0025E568BFB288BF521B304688BF4B
:107E900095B2ADF802700CF00CFDBDF80210A068B0
:107EA0000CF007FDA36822691F44974208BFE368EE
:107EB000A76008BFA360002D3FF440AF0521304606
:107EC000ADF802500CF0F5FCBDF80210E0680CF0C3
:107ED000F0FCBDF80220E3681344A3602EE74BF6E4
:107EE000EF62ADF8002022786E468DF804206268BB
:107EF000052193422ABF2769D71AFF1A934294BFDC
:107F00000025E568BFB288BF521B304688BF95B2D6
:107F1000ADF802700CF0CDFCBDF80210A0680CF0BA
:107F2000C8FCA36822691F44974208BFE368A760A2
:107F300008BFA360002D3FF4F9AE05213046ADF82F
:107F400002500CF0B6FCBDF80210E0680CF0B1FC79
:107F5000BDF80220E3681344A360E7E6CBF80070A5
:107F60006BE700BFCC1C02203D9B0220C81C0220F6
:107F7000C01C0220C41C0220014B1878704700BFAF
:107F80003D9B022010B50E4B0446D3E90023134459
:107F900098420DD282420BD800F01CFD58B1094A1C
:107FA00084600260FFF780FDBDE81040FDF70AB96C
:107FB000204606F085FCBDE81040FDF703B900BF80
:107FC000D01C02200100020088B110B582B001AAC5
:107FD0006946044600F05AFB024648B1124B283469
:107FE00094E8030083E80300104602B010BDFEE7EA
:107FF000DDE90012204600F0FBF902460A4B04F1CD
:10800000280103C983E80300002AEDD14FF4806002
:10801000A36B06495B01DBB281F82A33C1F8840106
:108020004860104602B010BDD01C022000E100E004
:108030002DE9F84FFDF7CEF8DFF8D480DFF8D4B0A3
:10804000DFF8D4A008F1080958F8047B396861B357
:10805000002402E001348C4227D2E600BD19AA6850
:10806000002AF7D06A68D2B2012AF3D16868BBF857
:108070000020B2EB104FEDD1A8684168C9B20229C7
:108080002CD0012915D00436B959013221F0FF0155
:1080900041F00301B951ABF80020FDF793F858F80F
:1080A000047C013439688C42D7D3C145CCD1BDE8BA
:1080B000F88F0168090C02F0BBFD012814D010D321
:1080C000022807D00322114B1046CAF800201A607C
:1080D00005F062F958F8047C3968BBE702F0C0FD8E
:1080E000EBE7BBF80020CEE76A68BBF8001022F08F
:1080F000FF0242F002026A604A1CABF80020FDF762
:1081000061F858F8047C3968A4E700BFD81C022045
:10811000E01C0220D06D0220E81C0220F0B54FF4D4
:1081200080669F4D9F4CC5F88461D4F80C3395B0A0
:1081300018060BD5FFF7AEFDFFF71EFF002858D13C
:10814000994BC4F81C011B680193019B954CD4F812
:108150000C5315F001051ED1D4F80C3313F0400375
:108160004CD1D4F80C2351070ED5904AC4F80831ED
:1081700012688F4B0692069A1A68022A00F0F28063
:108180001A68012A00F0D380864BD3F80C23D2065C
:1081900023D415B0F0BD002148F20202854BC4F88B
:1081A00000111B680293029BD4F81436934200F02E
:1081B000E28000F2A080002B00F0D780022B40F27A
:1081C000AB8048F20102934240F0CF8003200722A7
:1081D0007749794B08601A60DBE70021774AC3F8DA
:1081E000101113680793079B15B0BDE8F040FCF72A
:1081F000E9BFE02385F82A336E60CAE7704BC4F804
:1082000018511B680593059B00F01EFC10200122ED
:108210000A216C4BC4F8A0551B6803936A4B039E5C
:10822000C4F808031868694B049004980895C3F8CB
:108230001026D3F8100608900898C3F81426099160
:10824000099B2BB1099B013B0993099B002BF9D199
:1082500000224FF0010C042710265C49514BC1F855
:10826000142601F51531C3F89025402501F5C87194
:10827000096880240A9156490A98C3F89825096824
:108280000B9150490B98C3F8A025096805200C9163
:108290005049DDF830E0C3F8A82509680D914E4932
:1082A000DDF834E0C3F8AC2509680E914649DDF8E5
:1082B00038E0C3F808C3D1F800C0CDF83CC0DDF801
:1082C0003CC0C3F808730F681097109FC3F8086389
:1082D0000E681196119EC3F808530D681295129DF1
:1082E000C3F808430C68324B13943C49139C0A8032
:1082F000186015B0F0BD3A4A93422AD8B3F1886F9E
:108300002AD848F2030293422FD10320042228499D
:10831000294B08601A603CE7032318462449264A83
:108320000B60136015B0BDE8F04005F035B82D4A7C
:108330002D4811688A6802604968416012B309B328
:108340001268102A24D80A68102A21D802221A603A
:108350001AE7264A934208D103201549164A0860B5
:10836000136016E7FCF72EFF0EE703231049124AAD
:108370000B6013600DE7032006220D490E4B0860C9
:108380001A6006E7032010210B4A18601160FBE613
:1083900003204CF20601084A18601160F4E600BFA1
:1083A00000E100E000A002401CA1024008A1024040
:1083B000E81C022000A10240D81C022010A10240AB
:1083C00018A10240A0A5024008A3024000500040AE
:1083D00098A50240A8A50240ACA50240D06D02209D
:1083E00004004004EC1C0220E01C022001005005A7
:1083F000002800F0F7802DE9F04F056895B0002DBA
:1084000000F0E6808368002B00F0E2800669002E11
:1084100000F0DE80846A002C00F0DA8044681B2CB7
:1084200040F2DB80C4680B2C40F2D780D0F814C037
:10843000BCF1170F40F2D18000270446DFF8C4A139
:10844000806BDFF8C481DFF8C4B1DFF8C491CDE9F7
:108450000012CAF80000624639463046CBF80030B8
:10846000C8F80070C9F800700DF049FBE3693046A8
:108470003360A3697360FFF721FB01224FF0040C06
:108480005A4B5B49C3F8105609688020049159493A
:10849000DDF810E0C3F8147609682F7003916F704F
:1084A000EF70AA700399A16ADBF800E06960E16AE5
:1084B000019CA960EC60009C4F49AE61C5F814E0D6
:1084C0002C61C3F890250C68A1F592610594059C78
:1084D000C3F898C5D1F898444FF480660694069C7A
:1084E0001024C3F8A045D1F8A044444D0794079C3C
:1084F0004024C3F8A845D1F8A8440894089CC3F8C0
:10850000AC05D1F8AC0409900998C3F8007108686B
:108510000A900A98C3F8087188680B900B98C3F802
:10852000107108690C900C98C3F8187188690D9047
:108530000D98C3F81C71C86901F501710E900E9871
:10854000D3F804031043C3F804030C682C480F94B9
:108550000F9CD3F8044344EA0C04C3F804430C68AA
:108560001094109CD3F8044344F01004C3F804435F
:108570000C681194119CD3F8044344F04004C3F8F0
:1085800004430C681294129CD3F8044344F0800412
:10859000C3F80443DAF8003009685B011391DBB2D9
:1085A0001399C8F8002080F82A33C0F88461466027
:1085B0000297C5F81076D5F810360293029BD8F8CA
:1085C0000030012BFBD0D9F8000015B0BDE8F08FCA
:1085D0004CF20E0015B0BDE8F08F4CF2090015B05A
:1085E000BDE8F08F4CF20E00704700BF00A00240C3
:1085F00010A6024014A6024090A502400050004080
:1086000000E100E0DC1C0220E81C0220EC1C02203F
:10861000D81C022070B4174E31680D68ADB18B685C
:10862000834224D000230133DA009D4201EB02048F
:108630000BD0A468A042F6D104328B5823F0FF037C
:1086400043F003038B5070BC704771680D68002DB8
:10865000F9D08B6883420AD000230133DA009D42AF
:1086600001EB0204EFD0A468A042F6D1E4E70422B3
:10867000E3E700BFE01C0220034B1868A0F10500EF
:10868000B0FA80F040097047E81C0220002800F092
:10869000B880002900F0B580002A00F0B2802DE9F2
:1086A000F04F046A85B0002C00F0A680406A0028D4
:1086B00000F0A28042F687454FF0000A554EA842CE
:1086C00086F800A040F2A0800827DFF880912046BD
:1086D00016460D4644225146C9F800400DF00FFAE7
:1086E000D9F8002004F14403DFF8648182F801A086
:1086F00082F802A082F803A017701846442251465F
:10870000C8F800300DF0FBF9D8F8002004F1880318
:10871000DFF840B1177082F801A082F802A082F859
:1087200003A018464FF400725146CBF800300DF00C
:10873000E6F9394B04F5227CC3F800C05146604687
:108740004FF400720DF0DBF94FF4205C06214FF07E
:10875000010E4FF401304FF48832304B04F5916430
:108760005C602F4CC3F808C09981A3F800E019465B
:108770001C612C4BDFF8E0C020612B48636003F5DF
:10878000C073A060C4F800C02848E360626105F0CF
:108790005DFF002832D14FF0020C2024D9F80010E0
:1087A000DBF8002029601C4BD8F80010DFF8ACE0A3
:1087B0001F4D3160CEF800201B681E4902F5007283
:1087C0002A601D4E1D4A1E4D0B6003F500731D49A6
:1087D00033602880C2F814C509681B4B03910399C4
:1087E000C2F81C7519683B4402910299C2F82445ED
:1087F0001B680193019B01E04CF2070005B0BDE846
:10880000F08F4CF20E0070474CF2040005B0BDE84A
:10881000F08F00BF3E9B0220181D0220041D022085
:10882000281D02208000040000010400F01C02202A
:10883000FC1C0220F81C0220F41C022000A00240B4
:10884000D26D022014A502401CA50240241D022066
:108850001C1D0220201D022040000800001D0220D7
:10886000002861D0F0B4344B82B01A68334B824296
:108870001ED81B6832498342096803D8314C2468EA
:10888000844249D881420ED92F4B1B78002B4ED100
:10889000831A2E499F099B060A682D4D4FF0030449
:1088A0004FF0020614D04CF2100002B0F0BC70473A
:1088B0001B689842F7D3234A12689042F3D20124EE
:1088C000C31A244A9F099B0626461268224DEAD104
:1088D0004168C9B28E4222D1202002EBC7031F4952
:1088E0005A680E8892B242EA06425A605A6822F0EA
:1088F000FF0242F001025A6000BF0138FCD10122A0
:10890000174B43F824202A680B880192019A0133FF
:108910000B8002B0F0BC70478142D0D9B4E74CF272
:10892000070002B0F0BC70474CF20E0070474CF2EA
:108930000F0002B0F0BC7047001D0220F81C02209E
:10894000FC1C0220F41C02203E9B0220241D02205D
:108950000CA002401C1D022004A00240D26D022087
:1089600000A00240184B1B7863BBF0B4174A03F019
:10897000FF001468164B25681E68A5B10746C100A4
:1089800063185A68D2B2032A04D19F605A6822F051
:10899000FF025A605A6812F0FF0F01D19B682BB199
:1089A0000130A842EBD10020F0BC704706EB8010EC
:1089B00021448860436823F0FF0343F002034360CF
:1089C000F0BC7047002070473E9B0220241D02200F
:1089D000201D0220F0B4154A154B14681E68256846
:1089E000ADB100200746C10063185A68D2B2032A0D
:1089F00004D19F605A6822F0FF025A605A6812F050
:108A0000FF0F01D19B682BB101308542EBD10020D3
:108A1000F0BC704706EB801021448860436823F067
:108A2000FF0343F001034360F0BC70471C1D0220AC
:108A3000181D0220034B1B780BB905F037BF00202F
:108A4000704700BF3E9B02200122014B1A70704705
:108A50003E9B0220F0B4164A164B14681E68256827
:108A6000ADB100221746D00023185968C9B20329B6
:108A700004D19F60596821F0FF015960596811F0D5
:108A8000FF0F01D19B6823B10132AA42EBD1F0BCA8
:108A9000704792010444B018A0604368064923F06F
:108AA000FF0343F001034360B150F0BCFFF7D8BEB1
:108AB0001C1D0220181D0220010003002DE9F047B3
:108AC0004FF0FF3C0C460B68464F23F400330B601D
:108AD0000B68C60023F480130B6007EB060A84B012
:108AE000DAF80430896947F281020546D4F800803B
:108AF000CDE902CC00F0FCFC00286DD0DAF80420AF
:108B00008146002A5DD1384B711903EB8101242283
:108B100009F114000CF0E6FFD9F808304946243377
:108B2000C9F8083022684346120C120442F00A02C7
:108B30002260204647F2810200F0FAFC034668B941
:108B40002368DB000ED403AB4FF6FF720B212846DF
:108B500000F002FD034650B1C4F80080184604B08E
:108B6000BDE8F0877323184604B0BDE8F0874FF0E6
:108B7000806202AB1146284600F0EEFC034630BB93
:108B800057F8350038B1019305F084FE019B3E444F
:108B9000736047F835301846226822F08062226000
:108BA0002268120C120442F00C022260226842F485
:108BB00000322260226842F48012226004B0BDE8D4
:108BC000F08757F8351000680CF08CFF9BE7732B8B
:108BD000C4D0C4F80080C1E70C23184604B0BDE837
:108BE000F08700BF841E0220401D02200020704735
:108BF00038B54B1E012B08D8144662B101292DD07F
:108C0000B2F5877F08BF02220DD02920FCF76AF950
:108C10004FF0FF3520E001290BBF012202224FF463
:108C200082744FF4877400F0C9FC051E1BDB0F4BE8
:108C300005EBC50003EB800024220D490CF052FF28
:108C4000284606F081FA0368446123F48013036028
:108C5000036823F400330360284638BDB2F5827FF1
:108C6000D3D10A46DFE74FF0FF35F5E7401D02207C
:108C7000A472020038B5044606F066FA80B10B4DC6
:108C800055F8340038B105F005FE002305EBC402A9
:108C900045F8343053602046BDE8384000F054BDFC
:108CA0000920FCF71FF94FF0FF3038BD841E022069
:108CB0002DE9F0470D46DDE9088916461F460446B2
:108CC00006F042FA00283BD003689BB20C2B39D047
:108CD00003689BB20B2B11D1204B04EBC40413F897
:108CE0002430022B38D00369012B14BF39202A20ED
:108CF000FCF7F8F84FF0FF30BDE8F0870369012B6F
:108D00000BD0022B01D03920F2E703689BB2022B73
:108D100007D003689BB2042B03D003689BB2052BDA
:108D2000F1D10E4B04EBC40213F82230022BEAD12E
:108D300001462046FFF7C2FE002803D0D8DCD9E761
:108D40000920D5E7CDE908893B4632462946204629
:108D5000BDE8F04700F06ABD2320C9E7401D0220AE
:108D60002DE9F0470D46DDE9088916461F46044601
:108D700006F0EAF9002838D003689BB20C2B0FD01C
:108D800003689BB20D2B0BD00369012B1AD0022B69
:108D900010D02320FCF7A6F84FF0FF30BDE8F08795
:108DA000CDE908893B46324629462046BDE8F047D2
:108DB00000F0A2BE03689BB2022B07D003689BB2EF
:108DC000042B03D003689BB2052BE2D1084B04EBC4
:108DD000C40213F82230022BDBD101462046FFF7F4
:108DE0006DFE0028DCD0D5DCD6E70920D2E700BF35
:108DF000401D02202DE9F04782B00E461746054679
:108E000006F0A2F9002869D0036804469BB2022B41
:108E100058D13A463146284601F058F8002848D142
:108E2000EE002F4F731917F82330012B02D002B038
:108E3000BDE8F0874FF0FF3CDFF8A8A047F28102C1
:108E40000AEB0609D9F80430A1692846CDF804C018
:108E500000F04EFB804600283ED0D9F80420AABB83
:108E6000711907EB8101242208F114000CF03AFE7D
:108E7000D8F8083041462433C8F808302268042363
:108E8000120C120442F00A022260204647F28102CC
:108E900000F04EFB68B92368DB0015D4284601AB0F
:108EA0004FF6FF720B2100F057FB0028BFD00423C0
:108EB00023600028BBDDFCF715F84FF0FF3002B04F
:108EC000BDE8F0872D20F6E77320F4E75AF8351057
:108ED00000680CF007FEC3E70C20ECE70920EAE786
:108EE000401D0220841E0220F8B50E461746044697
:108EF00006F02AF9E8B1134B04EBC40213F8223050
:108F0000022B1CD1036805469BB2022B03D00368D9
:108F10009BB2042B13D13A463146204600F014FF91
:108F200010B1002806DCF8BD29462046FFF7C6FD33
:108F3000F7E70920FBF7D6FF4FF0FF30F8BD2D20F3
:108F4000F8E700BF401D02202DE9F04F85B00191E8
:108F5000054606F0F9F800287CD003690446012B89
:108F600076D103689BB2042B62D023689BB20B2B93
:108F70006ED1EE00384F731917F82330012B67D1EB
:108F800001224FF0FF3CDFF8D4907319EE0007F890
:108F9000232009EB0608A169D8F8043047F28102C2
:108FA0002846D4F800A0CDF80CC000F0A1FA834602
:108FB00000284BD0D8F80420002A41D1711907EBC2
:108FC000810124220BF114000CF08CFDDBF8082049
:108FD00059462432CBF8082022685346120C12045A
:108FE00042F00A022260204647F2810200F0A0FA15
:108FF00060B92368DB000ED403AB4FF6FF720B2180
:10900000284600F0A9FA70B1C4F800A0002803DCDB
:1090100005B0BDE8F08F7320FBF764FF4FF0FF3021
:1090200005B0BDE8F08F0199284600F0F1FFEDE7AB
:10903000EE00094F731917F82330022B95D19FE7E3
:1090400059F8351000680CF04DFDB7E70C20E3E748
:109050002D20E1E70920DFE7401D0220841E0220C9
:109060002DE9F04182B00E461746984605464FF06E
:10907000FF3406F069F8019400283CD0006880B203
:10908000062838D143463A463146284601F038F89A
:10909000044628B1002C2FDC204602B0BDE8F08148
:1090A000284606F051F80368184F23F40033036094
:1090B000036805EBC50523F480130646036007EB40
:1090C0008501242238460CF00DFD02233B703368E5
:1090D00020461B0C1B0443F00B0333604FF6FF725A
:1090E00001AB0C2100F038FA04460028D4D000204F
:1090F00000F02AFBCEE7092420464FF0FF34FBF7AF
:10910000F1FE204602B0BDE8F08100BF401D022004
:109110002DE9F041B1F58D7F069E1ED11F46054613
:10912000002B00F08C80904606F00EF800287BD0D3
:109130000468A4B2022C07D003689BB2042B03D0AE
:1091400003689BB2052B6FD108F1FF32042A7CD84B
:10915000DFE802F0244E32410700BDE8F04101F0A3
:1091600011B93B4C54F8350038B105F093FB00229F
:1091700004EBC50344F835205A6030464EB305F081
:109180007FFB44F83500002857D004EBC504324675
:10919000394666600CF0A6FC00201AE0042E4AD185
:1091A0003868002839D0012845D12A4A05EBC50482
:1091B00002F8240000200CE0012E3CD13A78002077
:1091C000003218BF0122234B05EBC50403EB8404D6
:1091D0006270BDE8F081042E2DD13A68022A2AD8A7
:1091E0001C4B05EBC50403EB8404A2700020F0E7E0
:1091F0005FEA960C1FD016F003041CD105EBC505E1
:10920000AD00144B281D18442B443246394683F8D0
:1092100003C00CF067FC2046DBE702210D4A05EB9A
